:020000040000FA
:040000006FD00400B9
:101000006F00907E00000000000000009020002093
:10101000AA220020A9BDF9F56C23002000000000E1
:10102000000000006C230020902000200000000041
:101030000000000090200020000000009020002010
:101040000000000090200020902000209020002030
:101050009020002090200020582F00209424002071
:101060000000000090200020902000201E2400207E
:1010700090200020D22300209020002090200020EB
:101080009020002090200020902000209020002020
:101090009020002001A04111B7170040985F3AC688
:1010A000945F3247E39CE6FE3245410182800111A4
:1010B00013078008F337078093F787083EC20100C3
:1010C0000100B7170040930570052380B70413068D
:1010D00080FA2380C7040100010083C6B70493F699
:1010E000F60DA385D704238007049246F3A6068055
:1010F0000100010093760502D5CEF336078093F602
:10110000860836C4010001002380B7042380C70489
:1011100001000100B70614007D89558D88C70100C4
:1011200001000100010023800704A246F3A6068007
:101130000100010073370780137787083AC6010062
:1011400001002380B7042380C704010001000100CF
:1011500001003727004093061005A303D7802380A2
:101160000704B247F3A70780010001009307800836
:10117000F3B7078093F787083ECE01000100B71749
:101180000040130770052380E704130780FA2380CB
:10119000E7040100010003C7B70413670708A3852C
:1011A000E70423800704F247F3A70780010001004A
:1011B0000561828093760504BDC6F336078093F6F9
:1011C000860836C8010001002380B7042380C704C5
:1011D00001000100B7061400938606047D89558D31
:1011E00088C7010001000100010023800704C246F6
:1011F000F3A6068001000100733707801377870884
:101200003ACA010001002380B7042380C70401000B
:1012100001003727004093062005A303D7802380D1
:101220000704D24781B773370780137787083ACC12
:10123000010001002380B7042380C70401000100DE
:1012400098471367070C98C723800704E24719BF24
:101250000111814601468145114506CE97000000E7
:10126000E780605893078008F3B7078093F78708F3
:101270003EC601000100B717004013077005238028
:10128000E704130780FA2380E7040100010003C785
:101290006704136717002383E70423800704B2471A
:1012A000F3A7078001000100F2400561828041112F
:1012B000814601468145114597000000E780A05214
:1012C00013078008F337078093F787083EC40100AF
:1012D0000100B7170040130670052380C70493066A
:1012E00080FA2380D70401000100FD552396B70240
:1012F00023800704A245F3A5058001000100733790
:101300000780137787083AC6010001002380C704CD
:101310002380D7040100010003C767041367170087
:101320002383E70423800704B247F3A70780010063
:10133000010001A0BD473305F50201007D1575FDD3
:101340008280411122C426C206C6AA8401446317C2
:101350009400B24022449244410182800504130566
:10136000803E420497000000E78000FD4180C5B741
:101370009305000273A04580824573901534924016
:101380002242B2424243D2436244F2440255925551
:101390002256B2564257D2576258F25806499649D9
:1013A000264AB64A464BD64B664CF64C065D965DD1
:1013B000265EB65E465FD65F09617300203041113C
:1013C000B7170040985F3AC6945F3247E39CE6FE49
:1013D000324541018280B71700401307000323887C
:1013E000E702854717170000232EF74673002030C9
:1013F000411122C42D6426C24AC006C637190040D6
:101400001304A4AAB704002023208900977000E0E9
:10141000E78020AA9C408297977000E0E78060A94F
:10142000E5B737370040834747009146BD8B639E41
:10143000D702B73600401306F00F973500009385AA
:10144000651E9737000083D7E72D03C7A6001377E3
:10145000F70F1DE3B7E70400BC4F09468945171590
:1014600000000345A5F7829731A099466394D70001
:10147000834757007300203003C786001377F70FA8
:10148000E365F6FC13851700AE9717380000231BA1
:10149000A8282380E70075B7B787004003C7670017
:1014A000098B6309071003C77700930600031377BE
:1014B0000703630DD708173800000348F87717367D
:1014C0000000130666740547B30606012380E60094
:1014D00083C577001737000013070775429793F508
:1014E000F50F2300B70003C58700973500009385EB
:1014F000A572C2951375F50F2380A5000347070059
:1015000089451377F703630CB70C63E7E50A6306B5
:10151000071A8545630CB7129737000083C7D77148
:101520003307F600034707001377F70F19CB85073A
:1015300093F7F70F3D476363F71A17370000A30DC2
:10154000F76EB787004009472383E700B78700405D
:1015500083C77700E207E18763DE0704973700005F
:1015600083C7976D173700001307076A3E978546B4
:101570002300D700173700001307076B3E97930629
:1015800000032300D700173700001307E7683E97D2
:10159000A14685072300D70093F7F70F3D47636403
:1015A000F71417370000A309F768B7870040094709
:1015B0002383E70073002030930610026300D70EE8
:1015C000930620026305D70693060002E316D7F4BC
:1015D00003C727021377C70F13672700D5A803C7D0
:1015E00067001377070465CB03C7A702173800000D
:1015F00013080843173500001305453A1347070839
:101600002385E70203C7A7021377370F1367870005
:101610002385E702814713070004B305F5008C41D9
:10162000B306F80091078CC2E399E7FEF5B503C74E
:10163000A702134707042385E70203C7A70213770E
:10164000C70F136727002385E702F9B503C76700B3
:101650001377070449C303C767021738000013084C
:10166000E82F1735000013052527134707082383A4
:10167000E70203C767021377370F136787002383D7
:10168000E702814713070004B305F5008C41B30658
:10169000F80091078CC2E399E7FEBDBD03C767025E
:1016A000134707042383E70203C767021377C70FB3
:1016B000136727002383E70285B503C76700137705
:1016C000070411CB03C727021377370F136787006F
:1016D0002381E70291B5238006003DBD97370000C6
:1016E000A38C0754B9BD97370000A387075475BD75
:1016F0002303048015472303E48001002302A48010
:10170000828083076480E3CE07FE23030480828007
:1017100083076480E3CE07FE03454480828083070D
:101720006480E3CE07FE2302A4808280411126C498
:101730004AC24EC006C61377F50BAD47AA892E895B
:101740009544630CF700194597000000E78080FA84
:1017500097000000E78020FB8D444E859700000035
:10176000E78040F9FD59FD1463983401B240A2446A
:101770001249824941018280135509011375F50F01
:1017800097000000E780E0F92209F1BF011126CCA3
:1017900006CEB704080097000000E780C0F61545A4
:1017A00097000000E78000F597000000E78080F6D2
:1017B00097000000E78000F62AC697000000E78047
:1017C00080F432459377150089EB13651500137586
:1017D000F50FF240E24405618280FD14E9F0014515
:1017E000CDBF397126DC4ADA4ED852D656D45AD2F9
:1017F0005ED006DE62CE66CCB7E700E07D5783AAF6
:10180000070022C603AA470023A0E71823A2E7186F
:10181000B7170040130770052380E704130780FA09
:101820002380E70483C74704930B75FFB684E20760
:1018300093FBFB0F8546AA892E8B32893724004003
:10184000E187015763FA76016308D50089461307DB
:1018500000026313D5000157D98F93F7F70FB71C18
:1018600000402382FC0411472303E4801305F00F9A
:1018700097000000E78000E8094C97000000E7802F
:1018800080E863657C15B7050700DA9537870700A0
:10189000795563FEE504B3879500636AF704370B57
:1018A0000800A94733EB65016395F90881E8814495
:1018B00097000000E78020E5268515A8DA85094510
:1018C00097000000E780C0E605090345F9FFFD1415
:1018D000050B97000000E780C0E481C49377FB0FFD
:1018E000E5F797000000E780A0EA69F17D55B7179A
:1018F0000040130770052380E704130780FA238054
:10190000E70403C74704418B2382E704F250B7E79B
:1019100000E023A0571123A24711E2543244525948
:10192000C259325AA25A125B825B724CE24C21615C
:101930008280A547639BF90685691309F00FB306FA
:101940009900B3742B01B6941349F9FFB37499004D
:10195000856B33796901416B9387F9FFB3F72701F1
:1019600099E363FC340193D94900C147E3E637FFAB
:101970003DBF0569C1697D19D9B71305800D63881D
:101980006901130500026384790113051008CA85F3
:1019900097000000E780C0D997000000E78040DF93
:1019A00031D54E99B38434416DBFDA852D4597000A
:1019B0000000E780E0D7CA94E30B99EE0509970091
:1019C0000000E78020D5A30FA9FEFDB79387F9FF9C
:1019D00093F7F70F636DFC0C83C71C0413073008E3
:1019E0006315F706370708006361EB06B3079B0032
:1019F000B706100063FBD704334BEB0089476399AC
:101A0000F9068980D549E38404EADA850945970017
:101A10000000E780E0D111090327C9FF9147232087
:101A2000E48003076480E34E07FE23033481FD173F
:101A3000EDFBFD14110B81C49377FB0FE9FF9700B9
:101A40000000E780E0D461F155B5B717004003C747
:101A50005704B70708001377070219E3B787070091
:101A60007955E376FBE833079B00E3F9E7F841B5E6
:101A70008547E380F9F0DA852D4597000000E7807F
:101A800020CB9389F4FFE38404E297000000E78011
:101A900060C893F7390091EB83260480032709007F
:101AA00093074900E396E6E03E89CE84D9BFB54767
:101AB0006399F9001305900B97000000E78080C33D
:101AC000FDB3B1471305B00AE388F9FE9947639760
:101AD000F904B7050800B365BB002D459700000069
:101AE000E78000C581448D4BA14997000000E78045
:101AF00060C263967401832704802320F900850463
:101B0000E39534FF8327048013172B0163550700E7
:101B10002312F90069BB2322F90051BB9D47639F43
:101B2000F90281451305B00497000000E78040C02A
:101B3000BD442320090023220900FD59970000001D
:101B4000E78040BD93F77400CA9703C70700FD14F0
:101B5000398D2380A700E39334FF91BBA14763979E
:101B6000F90697000000E780A0C28144630D0B00D6
:101B70008D479304C0036308FB00930400056304CE
:101B80008B01930440041375C507E30295D21945F0
:101B900097000000E78000B697000000E780A0B63D
:101BA000054597000000E780E0B426859700000017
:101BB000E78020B7094597000000E78080B69700CE
:101BC0000000E780E0BCE31405CE0DB39147639FAE
:101BD000F9001305600697000000E780A0B19700A8
:101BE0000000E78040B213059009F9B5E38109CC04
:101BF000F1547DB9BD660147173600001306063063
:101C0000938606A685458347060093F7F70F91C391
:101C100082800507E3F9E6FE973700002380B72EA0
:101C2000DDB77D166206618693178601E18763D46E
:101C3000070001458280931726003307F500AE9711
:101C400018439C4363E7E7007D16E37FF7FC7D556F
:101C5000828005458280FD15E205E18513978501A7
:101C6000618793F7F50F63480700FD15139725006B
:101C70002A97584365D713851700620561858280CE
:101C80003308B5021C4283A80600B335B502C297DB
:101C900033B50701AE98469585486367B5006394F0
:101CA000A50063E3070181480C43C6950CC388C2B5
:101CB0001CC2828081471397870161876343B70005
:101CC0008280139727002A97232007008507E5B70E
:101CD0008147014793968701E18663C5B6001335B6
:101CE0001700828093962700AA9694428507558F05
:101CF000D5B793D755408A07AA979C430545331516
:101D0000B5007D8D828017F3FFDFE702833D2A84D3
:101D100097000000E78060F405C5931725003E9406
:101D20000327C4FF814711EB7D1516053E9542053B
:101D3000418517F3FFDF6700033D05838507E5B79E
:101D40000145C5BF81471397870161876343C7007A
:101D5000828013972700B386E50094422A9785076F
:101D600014C3D5B77D1662066186014793178601B5
:101D7000E18763D50700133517008280931726008B
:101D8000B306F500AE9794429C437D16B58F5D8FE8
:101D9000F1BF8A05AA9501476363B500828083A6D7
:101DA000C5FFF11593D71600D98F9CC11397F60183
:101DB000E5B72A830148014701456343D700828084
:101DC000B387050183A80700B30706019C43C697A4
:101DD000AA976384F80033B517010507B308030118
:101DE000620723A0F80061871108C1BF2A83014759
:101DF0008147014563C3D70082803388E50083288B
:101E00000800330EE600032E0E003388A840330886
:101E1000C8416384080133B508018507B308E300AE
:101E2000E20723A00801E1871107E9B717F3FFDFF5
:101E3000E702232B0111B286B2842E86AA850A8579
:101E400097000000E780C0FA2A84A6850A859700DB
:101E50000000E78020E833348000060413351500C5
:101E6000018D056117F3FFDF6700E32917F3FFDF3B
:101E7000E702A3244111AA89AE8A328BB68402C23A
:101E800002C402C60144131C8401135C8C416349E3
:101E90009C02939B1400FD1B0549138CF4FFF15C1D
:101EA00033048901620461846340740792478E049D
:101EB000CE9423AEF4FE410117F3FFDF67006323E6
:101EC00013192400B30B2B01014A93172A00D6974C
:101ED00083A50B0088437800340050009700000071
:101EE000E78040DA050A93178A01E187F11BE35E78
:101EF000FCFC92474E9905042320F900A2473EC2FC
:101F0000B24702C63EC441B7131A8901135A8A4127
:101F1000131D240093178A01E18763CF970092472E
:101F20000A044E941CC0A24705091379F90F3EC25A
:101F3000B24702C63EC4ADB7B3079A0313152A00D1
:101F400056950841780034005000050AEA97DA9760
:101F50008C4397000000E780E0D26DBF197106C284
:101F600012C416C61AC81ECA22CC26CE2AD02ED219
:101F700032D436D63AD83EDA42DC46DECAC0CEC2C9
:101F8000D2C4D6C6DAC8DECAE2CCE6CEEAD0EED2F9
:101F9000F2D4F6D6FAD8FEDA971500009385058CB0
:101FA0008841E700050092402242B2424243D243B8
:101FB0006244F244025592552256B2564257D257C5
:101FC0006258F25806499649264AB64A464BD64BBD
:101FD000664CF64C065D965D265EB65E465FD65F45
:101FE0000961730020300000972100209381810156
:101FF000175100201301018117F5FFFF1305C500DC
:102000009705002093850500171600201306C6FDCE
:1020100063FAC5008322050023A055001105910530
:10202000E3EAC5FE170502001305856C971500202D
:102030009385C5FB171600201306C66563FAC50015
:102040008322050023A0550011059105E3EAC5FE92
:102050001715002013050564974500209385053664
:102060006377B500232005001105E36DB5FEFD4241
:10207000739002BC8D4273904280B722000093821D
:10208000828873900230970200209382A2F793E235
:1020900032007390523097520000938222B57390B1
:1020A00012346FB0F47573002030397101436EC67D
:1020B00019A0397141536AC866CA62CC5ECE19A0B4
:1020C000397101535AD056D252D44ED64AD826DA54
:1020D00022DC06DE33016140828241114AC026C201
:1020E00022C406C68282B24D4101024D924C224C5E
:1020F000B24B4101024B924A224AB2494101024984
:1021000092442244B240410182803D432A87637356
:10211000C3029377F700BDEFADE5937606FF3D8AE6
:10212000BA960CC34CC30CC74CC74107E36BD7FE30
:1021300011E28280B306C3408A0697020000969699
:102140006780A6002307B700A306B7002306B700E1
:10215000A305B7002305B700A304B7002304B70005
:10216000A303B7002303B700A302B7002302B700FD
:10217000A301B7002301B700A300B7002300B700F5
:10218000828093F5F50F93968500D58D9396050182
:10219000D58D61B7939627009702000096968682A8
:1021A000E78086FA9680C1171D8F3E96E374C3F8C8
:1021B000A5B73367B500FD530D8B79E7B7877F7FF0
:1021C0009387F7F710419441B372F6003363F6003A
:1021D000BE92B3E262006397720C6318D606504158
:1021E000D441B372F6003363F600BE92B3E26200EC
:1021F0006398720A631BD60410459445B372F600C7
:102200003363F600BE92B3E262006391720A631E0A
:10221000D6025045D445B372F6003363F600BE9241
:10222000B3E26200639A72086311D60210499449BE
:10223000B372F6003363F600BE92B3E262006393BA
:1022400072085105D105E30FD6F6131706019397CF
:102250000601631CF7001357060193D706013305E7
:10226000F7409375F50F91E982804183C18333056F
:10227000F7409375F50F91E182801377F70F93F78D
:10228000F70F3305F74082800346050083C605003B
:10229000050585056313D60065FA3305D6408280AF
:1022A00011059105E312D6FE014582802105A105A5
:1022B000E31CD6FC014582803105B105E316D6FC4E
:1022C000014582804105C105E310D6FC01458280AD
:1022D000B717004003C777051377E70FA38BE70411
:1022E000130700F8A38DE7043D47238CE704130789
:1022F0005003A38CE70403C7A7051377D70F238DDB
:10230000E7048280B717004003C7E7020D89411137
:102310001377C70F498F93068008F3B6068093F6AC
:10232000860836C601000100930670052380D70495
:10233000930680FA2380D704010001002387E70277
:1023400023800704B247F3A7078001000100410181
:10235000828041112A83014E930E407E130F001993
:10236000930F400663E56E129308001913034006AD
:10237000B3781503854E0D4FA14F337365020D8958
:102380001335150063EFBE121308F6FF79467298F5
:102390004208135808013307C70213D61700BE07B7
:1023A00032976146B3F6C60213068070B386C60242
:1023B0003697A166F58F42075D8FB716004083C739
:1023C000F60293F70708A303F1000346710083C7E1
:1023D000F60293F70708E394C7FE83477100B71628
:1023E000004093F7F70F6388071293078008F3B74D
:1023F000078093F787083EC401000100B71700402B
:10240000930670052380D704930680FA2380D704AF
:102410000100010023AA070383C6170393E60608F9
:10242000A388D70223800704A247F3A707800100EF
:1024300001001166B71700407D16D45BC85F938515
:102440004703A98EF18EF5FA93068008F3B606804D
:1024500093F6860836C601000100930670052380B6
:10246000D704930680FA2380D7040100010098C1A5
:1024700003C7170313670704A388E7022380070431
:10248000B247F3A7078001000100410182807D135C
:102490003368E3039308E016630E08003368F30320
:1024A0009308D016630808009378330093B8180097
:1024B0009388D81633081E01131E0801135E0E01FF
:1024C00055B56393E5030548638608000148630337
:1024D00003002A8871087298FD15131E0801C205B1
:1024E000135E0E01C18179BD13F8150063F4BF00BE
:1024F0007908D5B713381800E5BF83C7F60293F7FC
:102500000708A303F1000346710083C7F60293F79F
:102510000708E394C7FE8347710093F7F70FF1DFD5
:10252000E9B531714AD966CB06DF22DD26DB4ED70D
:1025300052D556D35AD15ECF62CD6AC96EC7AA8C26
:1025400002D897100000E78020B12A8993078008FD
:10255000F3B7078093F787083EDA01000100B71749
:102560000040130770052380E704130780FA2380D7
:10257000E7040100010003C7F7021377770FA38771
:10258000E70203C7F70213678700A387E7022380E8
:102590000704D257F3A70780010001000545970003
:1025A0000000E78060D6130780C13347E902116A53
:1025B00093070AE893065002BD69930BA004814A71
:1025C000014B13048008930470057D1AB347F90288
:1025D0003307D7023EC0FD873ECC938709A69309F7
:1025E000803E3347F7023AC27D873AC43347390306
:1025F0008549B399990193D93940B306D702B30BF2
:102600007703B3C6F602B3CBFB0236C6FD8636C8E7
:1026100093D6FB4136CEB7460F0093860624334946
:10262000D9028566938606FAB3969601B389E902C4
:10263000130760553309D90293060010B389E902E4
:102640003349D902B3C9F9029316390036CA37198A
:102650000040FD8636D0930D090493D7F9413ED250
:10266000F336048093F6860836DC010001009307F8
:1026700070052380FD00930680FA2380DD000100B1
:1026800001008346390593F6860FA309D9048346D2
:10269000390593E61600A309D90423800D00E256FC
:1026A000F3A6068001000100130C80FA116DF336C9
:1026B000048093F6860836DE01000100930770055A
:1026C0002380FD0023808D01010001008346390530
:1026D000216693E60602A309D90483560905B3E6E9
:1026E000A6012318D90483560905D18E2318D904CD
:1026F00023800D00F256F3A60680010001008346F8
:10270000390593F606026381061A03463905218AC4
:102710006DDE081897100000E7800098733604807B
:1027200013768608B2C20100010023809D00238039
:102730008D0101000100B717004003C6370513766D
:10274000F60DA389C70403C6370513660602A389DD
:10275000C704835609052166B3E6A6012318D904E8
:1027600083560905D18E2318D90423800D0096467F
:10277000F3A60680010001008346390593F60602A0
:10278000638B061483463905A18AEDFE970000206D
:10279000E7806090AA8636D497000020E780A08F5B
:1027A000A256E30AD5FE835609054255B3E6A601B3
:1027B0002318D90497100000E780C08F834639059D
:1027C000A18AEDDE03560905834629058247337643
:1027D000CA00B306DA0293D5F641B296B388F64042
:1027E000E24733B8C6002E983308F840A247B3B684
:1027F00016013308D84063C70701631DF8009247EC
:1028000063FA1701C247634FF80E63950701B24799
:1028100063EAF80E894663E9660FF24693151800DD
:1028200013D3F8015E8613951800B365B30042D642
:1028300046D497C00100E78080493258050B137BCE
:10284000FB0F63470001631A0838A25863870838F2
:1028500013081500B336A800B69513D6F5013298C3
:10286000B336C800AE9613581800FE06B3E606014C
:102870007336048013768608B2C6010001002380F7
:102880009D0023808D01010001000356C902B2960C
:10289000C206C1822316D90223800D00B646F3A6D4
:1028A00006800100010021B5F336048093F6860806
:1028B000B6C00100010023809D0023808D0101002E
:1028C00001008346390593E60602A309D904238053
:1028D0000D0086460DB5F336048093F68608B6C41F
:1028E0000100010023809D0023808D010100010073
:1028F0008346390593E60602A309D90423800D0017
:10290000A646BDB5E30B0BF0F336048093F68608BC
:10291000B6C801000100930680FA23809D00238041
:10292000DD00010001008346390593F5FC0F93F6A5
:10293000860FA309D90483463905CD8EA309D9048E
:1029400023800D00C646F3A6068001000100130592
:1029500080FA03463905930639051D8A631C9629BA
:102960007336048013768608B2CC0100010013068A
:1029700080FA23809D002380CD000100010003C662
:1029800006001376F60D2380C60003C60600136604
:1029900006022380C600835609051166D18E2318CE
:1029A000D904835609052166D18E2318D9042380C2
:1029B0000D00E646F3A6068001000100130680FA2A
:1029C0008346390593F60602638006268346390559
:1029D000130C3905A18AFDDA081897000000E7807A
:1029E000A06BF336048093F68608B6D00100010090
:1029F000930680FA23809D002380DD000100010002
:102A000083460C00116693F6F60D2300DC00834626
:102A10000C0093E606022300DC0083560905D18EE4
:102A20002318D904835609052166D18E2318D904A9
:102A300023800D008656F3A60680010001001306D0
:102A400080FA8346390593F60602638A0620834698
:102A50003905A18AEDFE97F0FF1FE780C0632A8C3D
:102A600097F0FF1FE7802063E30C85FF835609057D
:102A700011664255D18E2318D90497000000E780D3
:102A800060638346390513063905A18AFDDAF336FA
:102A9000048093F68608B6D401000100930680FAFC
:102AA00023809D002380DD00010001008346060095
:102AB00093F6F60D2300D60023800D00A656F3A64C
:102AC0000680010001008356090503462905D24707
:102AD000B376DA003306CA021305800C9355F6412B
:102AE0003696330DF6408257333CD6002E9C333653
:102AF000A601330CFC40330CCC40330885039256BE
:102B00004E86B335A5033305A503C29597C00100D2
:102B1000E780E01B63468001631E0C16630C0D16F4
:102B2000130615003335A6002E959356F5013696FB
:102B3000B335D600AA959396F50105828585D18E89
:102B40006346B000639D051A638B061A0356C902DB
:102B500015823305D6003336C500B2956348B00000
:102B6000639105241306F00F637DA622894663F363
:102B7000561593078008F3B7078093F78708BED6EA
:102B80000100010037170040930770052300F70488
:102B9000930780FA2300F704010001008356C7025F
:102BA00089678117D58FC207C1832316F7022300D7
:102BB0000704B657F3A7078001000100FA506A54D2
:102BC000DA544A59BA592A5A9A5A0A5BFA4B6A4C49
:102BD000DA4C4A4DBA4D296182801308F5FF33352E
:102BE000A800FD152E951356F5013298B336C8008E
:102BF000AA9695B9F336048093F68608B6CA010002
:102C0000010023809D002380AD0001000100834668
:102C10003905CD8EA309D90423800D00D646F3A62D
:102C200006800100010035B3F336048093F6860870
:102C3000B6CE0100010023809D002380CD0001005D
:102C400001008346390593E60602A309D9042380CF
:102C50000D00F646F3A606800100010095B3F33699
:102C6000048093F68608B6D20100010023809D00FF
:102C70002380CD00010001008346390593E606025A
:102C8000A309D90423800D009656F3A606800100FF
:102C9000010045BB9306F5FF33B5A600FD152E9543
:102CA0009355F501AE96B3B5B600AA951396F50106
:102CB000858269B5F336048093F68608B6D801009C
:102CC0000100930680FA23809D002380DD0001002F
:102CD00001008356C9020566011693F6F60FD18EE0
:102CE000C206C1822316D90223800D00C656F3A660
:102CF000068001000100850A93FAFA0F95B233E6C7
:102D0000B60045C20356C9023305D0403338A0008F
:102D1000B305B040B385054115826345B000D1E1EC
:102D20006371A608894663F0560593078008F3B7D8
:102D3000078093F78708BEDA01000100B71700404B
:102D4000130770052380E704130780FA2380E70444
:102D50000100010003D7C7027D8B2396E702238081
:102D60000704D65781BDF336048093F68608B6DC97
:102D700001000100930680FA23809D002380DD007E
:102D8000010001008356C9020566011693F6F60F8D
:102D9000D18EC206C1822316D90223800D00E656C9
:102DA000B9B793078008F3B7078093F78708BEDEAB
:102DB0000100010037170040930770052300F70456
:102DC000930780FA2300F704010001000356C702AD
:102DD00093975600B297C207C1832316F7022300C8
:102DE0000704F657C1BB914763EEB70217E701002E
:102DF0001307478C8A05BA959C41BA978287B71703
:102E0000004003A7470B1345F5FF698F23AAE70A84
:102E100003A7070B698F23A8E70A03A7070A798D81
:102E200023A0A70A8280B717004083A6470B134749
:102E3000F5FFF98E23AAD70A83A6070B558D23A881
:102E4000A70A83A6070A758F23A0E70A8280B7170F
:102E5000004003A7470B498F23AAE70A03A7070BE4
:102E60001345F5FF45BFB717004083A6470B13472F
:102E7000F5FF758F23AAE70A03A7070A598D4DB7F7
:102E8000B717004003A7470B498FEDB7914763EE93
:102E9000B70217E70100130727838A05BA959C41FB
:102EA000BA978287B717004003A7470D1345F5FF70
:102EB000698F23AAE70C03A7070D698F23A8E70CE6
:102EC00003A7070C798D23A0A70C8280B7170040B9
:102ED00083A6470D1347F5FFF98E23AAD70C83A6C7
:102EE000070D558D23A8A70C83A6070C758F23A06B
:102EF000E70C8280B717004003A7470D498F23AA2C
:102F0000E70C03A7070D1345F5FF45BFB7170040B2
:102F100083A6470D1347F5FF758F23AAE70C03A778
:102F2000070C598D4DB7B717004003A7470D498FC0
:102F3000EDB7797122D43714004026D24AD0035914
:102F400024028354040206D64209C2044ECE52CC57
:102F500056CA13590901C1802DE11379F9F793F489
:102F6000F49F4209C20413590901C18093078008E4
:102F7000F3B7078093F787083EC401000100930769
:102F800070052300F404930780FA2300F404010081
:102F90000100231124032310940223000404A247F8
:102FA000F3A7078001000100B25022549254025945
:102FB000F249624AD24A45618280B7F507008146EC
:102FC0003000B105194597000020E7808081A247B5
:102FD00013972701E34A07FC1369090893E40440A7
:102FE00093098008F3B7098093F787083EC0010072
:102FF0000100930A700523005405130A80FA230088
:10300000440501000100231124032310940223002E
:1030100004048247F3A7078001000100294597F0C7
:10302000FF1FE7802031F3B9098093F989084EC268
:1030300001000100230054052300440501000100A4
:103040008357040293E707202310F40223000404AB
:103050009247B9B7B7170040884742054181937737
:10306000050491EB9377F5013755E80113050580C9
:103070003345F50282809377050C130700046397AC
:10308000E7009377F50137459C1CCDB72165130503
:1030900005D0828037E700E01C435443A183E20659
:1030A000D58F1CC1FD572320F7182322F7188280E3
:1030B00013178500B7E700E023A0E710618123A282
:1030C000A7108280B7F700E08847CC47828081470D
:1030D00037370040A14663C4C7003285828003456C
:1030E000B740E38EA6FE3385F5000345050085074E
:1030F0002304A740CDB797070020938727EF9C4371
:10310000173700201307872B3E95636EE5001737AE
:1031100000201307273F6368A70017070020232715
:10312000A7EC3E858280FD57EDBF8280411122C40D
:1031300006C62A8497000000E78000F22947B307FB
:10314000E502B2408D83B3D7870222449507B3D7F7
:10315000E70237370040C207C1832316F700410159
:103160008280411137150E0006C697000000E780E7
:1031700020FCB7370040130770F82381E7000D47A4
:10318000A381E70013070004A380E7000547238716
:10319000E700B24041018280373700408347270073
:1031A0001A0593F7F703C98F93F7F70F2301F70079
:1031B0008280B737004003C7170019C9D98DA38093
:1031C000B70003C70700136787002380E7008280EA
:1031D00093C5F5FFF98DA380B7008280AE872A875B
:1031E000B736004021463738004089E71703000012
:1031F0006700E3F383C8B600E30916FF05078348B9
:10320000F7FFFD17C20723041801C183F9BF41115D
:1032100022C406C62A8497000000E780E0E329471D
:10322000B307E502B2408D83B3D7870222449507E6
:10323000B3D7E70237370040C207C1832316F740F0
:1032400041018280716541111305052006C6970072
:103250000000E78000FCB7370040130770F82381B7
:10326000E7400D47A381E74013070004A380E74030
:1032700005472387E740B24041018280CC4141119C
:1032800006C6328503C6150083C5050022064D8E8D
:1032900042068D654186138875A2630C0611634B47
:1032A000C804138845A26300060D634AC8009385CD
:1032B00035A26301B6082390060029464DA0138865
:1032C00055A26305060D938565A2E316B6FE8D45EE
:1032D0001D4663E6E5081146198E63F3C7003E8676
:1032E000B7E704002390C600FC4797D501009385FB
:1032F000E53F9DA0138895A263030611634E060D5A
:103300001388A5A263000613938505A5E315B6FAF5
:1033100099451D4663E5E504198E63F3C7003E86B3
:10332000B7E704002390C600FC479705002093856B
:1033300025D61DA09D451D4663E3E5022146198E55
:1033400063F3C7003E86B7E70400FC472390C6003E
:103350009705002093858534BA9582970146B2403F
:10336000328541018280AD451D46E3EAE5FE3146E6
:10337000198E63F3C7003E86B7E704002390C600AA
:10338000FC4797D501009385E538F9B7B1451D464F
:10339000E3E7E5FC3546198E63F3C7003E86B7E7E1
:1033A00004002390C600FC4797D50100938585371C
:1033B00065B78D451D46E3E4E5FA1146198E63F3C2
:1033C000C7003E86B7E704002390C600FC4797D5A8
:1033D00001009385653249B78D451D46E3E1E5F867
:1033E0001146198E63F3C7003E86B7E704002390A9
:1033F000C600FC4797D5010093858534B1BFA5452C
:103400001D46E3EEE5F42946198E63F3C7003E86B8
:10341000B7E704002390C600FC4797D501009385C9
:10342000652E1DBFB5451D46E3EBE5F23946198E05
:1034300063F3C7003E86B7E704002390C600FC474D
:1034400097D501009385852901BFB7E7040003A341
:103450000713970600209386A6C24146A545170587
:1034600000201305E5B802832D455DE703C505007F
:103470000947631FE50803A84500411106C6034735
:10348000180032850346080022074168518F9308CF
:1034900028FE6307170563E9E800051863030703BF
:1034A00023900600294591A8130648FE630AC70425
:1034B0001518E31707FF15463E87637BF60015478F
:1034C00001A8130600023E876374F600130700028A
:1034D000B7E704002390E600FC471316070111A884
:1034E0003E8691C30546B7E70400FC472390C6001B
:1034F0004206CC45418282970145B240410182801B
:10350000130600083E87E375F6FC13070008C9B7E9
:103510002390060005458280828041677917630405
:10352000E504411122C406C685472A84639FF5003D
:10353000B7E7040022852244B24003A3871397050E
:1035400000209385E52F4101028389476399F500A7
:10355000B7E7040083A7070B8545829771D9B2406E
:103560002244410182808280797126D252CCAE847D
:103570002A8A97D501009385A51E17D5010013054A
:10358000A52006D63AC622D44AD0368432894ECEF9
:1035900097C00100E780E0BEA28517D501001305A2
:1035A000A51F97C00100E780C0BD294597C0010055
:1035B000E78000C283C7840093F70702F9E383C959
:1035C00004008947054532476396F908D44083C70C
:1035D000160083C60600A207D58FC166138616FEA5
:1035E000638CC7028D16638FD7068D6693862690EF
:1035F00029456391D706B7E70400A286225403A3A6
:103600004714B250F2494A86A6850259925452850F
:10361000624A8547456102832D450DEF93070002FD
:10362000354563E98702B7E70400FC47C844130641
:103630000002CA8582978149970700209387072156
:103640009C43014581CB9C4391C74E852286CA8508
:1036500082970145B250225492540259F249624A6B
:10366000456182802D457DF79307700F3545E3E373
:1036700087FEB7E70400FC47C8442286CA858297C4
:1036800065BF2145C1BF411122C437E4040083272F
:10369000841326C2AA84416506C697050020938537
:1036A000251A7D1582978327C40A17050000130584
:1036B00005E78588829795C0032304132244B2400E
:1036C000924497060020938626AE4146C5451705CD
:1036D00000201305659C41010283B24022449244BC
:1036E00001454101828019C59707002023A0A71634
:1036F00001458280454582801147636AA70A97D6B3
:1037000001009386A6040A0536951841411106C6A4
:103710003697AE87B2850287130700026145639D25
:10372000E700B7E70400FC47130600021705002076
:10373000130545F782970145B24041018280054754
:103740006145E39BE7FEB7E70400FC470546170524
:103750000020130525F7F9BF1307700F6145E39D9E
:10376000E7FCB7E70400FC471306700F17050020BD
:10377000130585F5C1B7130700086145E39EE7FA15
:10378000B7E70400FC4713060008170500201305DF
:1037900025034DB715476145E390E7FAB7E7040005
:1037A000FC471546170500201305C50961B70945F3
:1037B0008280411126C2B7E4040083A7C41322C447
:1037C0004AC006C62E8497050020938565072A897E
:1037D0008297058905C5970700209387E78B83D7D4
:1037E000A70BA28503A3440D2310F4002244B2408A
:1037F00092444A850249014641010283B240224473
:103800009244024949454101828097070020238163
:1038100007049707002023AF0702B717004003A74C
:10382000070CB706C0FFFD16758F23A0E70C03A792
:10383000070DB7064000558F23A8E70C03A7070C18
:103840003D9B23A0E70C03A7070D1367070123A8DF
:10385000E70C8280B717004003A5470C83A7470CED
:10386000598113451500C18B058999E3136525001E
:103870009707002083C7C7FD6380A7029707002032
:103880002388A7FC11C9970700209387A7FC03A3EF
:1038900007006303030002838280114517F3FFFFD3
:1038A000670063C8011122CC06CE3714004026CA37
:1038B0004AC84EC652C483447405034AB4058349BA
:1038C00084050349940597F0FFFFE780A0A0834794
:1038D000A40593F4F40F137AFA0F93E71700230D5E
:1038E000F40493F9F90F1379F90FB717004003C7E0
:1038F000A705058B6DFF03D5C705A38D4705238C51
:103900003705A38C2705A38B9704F2406244D24469
:103910004249B249224A05618280411193970501CB
:1039200022C406C626C2C1872E8463DC0700B7E422
:103930000400FC54829719C1BC5482972165218DE3
:1039400015A893F7150013C515008DE793F725000B
:103950009DC797000000E78020F0B7E70400BC4F48
:103960001306000A894517050020034525EF8297B5
:1039700013452400B240224492444101828093972F
:10398000250163D80702B7E4040083A7C41E829709
:1039900097000000E780A0F0BC4C375607001306E4
:1039A0000630896517050020034545EB82970965B8
:1039B00079B7939715010145E3DE07FA17D50100A2
:1039C000130585E597C00100E7808093B7E7040001
:1039D000BC4F13060064916517050020034505E8F8
:1039E00082971165A9BF1D71A2CC37E404005C5C0D
:1039F000485886CE494697D50100938565DD829764
:103A000011E917D501001305E5DD97C00100E78036
:103A1000208F01A0B7F600E0795798CAFD57DCCA9D
:103A20000567B7E700E023A0E7101306F00290C295
:103A300023A0E718010001003707002018471306EC
:103A4000000481459706002023A8E6E04157A38A99
:103A5000E7403C4408088297970700209387077C3B
:103A60003EC8856713870740938757D1231AE10023
:103A70002312F1021307B00F97F7FFFF9387C76474
:103A80002310E1023ED81547970700009387C7E14E
:103A9000B7F50700A30FE1003EDC054797070000DC
:103AA0009387E7DF81463000E10519452301E102F4
:103AB0003EDE97F0FF1FE780C0D218088147994685
:103AC00030003E960346060085070507A30BC70096
:103AD000E398D7FEC24791C70357410185676373D7
:103AE000F70001A0B7E7040083A7470A08088297F8
:103AF000AA8511C917D50100130505D097B001009B
:103B0000E780206801A0F64066442561828041116B
:103B100026C2B7E4040083A7040806C622C417051A
:103B200000001305C5DF829717040020130404D397
:103B30002300A40097000000E780800297000000A7
:103B4000E780E0CC03450400224403A38405B2408F
:103B5000924413060032896541010283797106D6C9
:103B600022D413078008F337078093F787083EC2F3
:103B700001000100B7170040930570052380B704CA
:103B8000130680FA2380C7040100010083C6F702F0
:103B900093F6A60FA387D702238007049246F3A6C5
:103BA00006800100010073370780137787083AC445
:103BB000010001002380B7042380C7040100010035
:103BC00003C7F70213672700A387E70223800704D0
:103BD000A247F3A7078001000100054597E0FFFF1A
:103BE000E780807297000000E78060CB0147814644
:103BF0008147054685451305407E97E0FFFFE78036
:103C0000807537E404003C44680051468145829742
:103C1000B707C0A83EC8B787E803938707D03ECA56
:103C200097E7FF1F9387A7793EC67C586800829765
:103C3000B250225445618280411197D5010093858D
:103C4000A52217D50100130525B406C697B00100BB
:103C5000E780205317D501001305053A97B00100FE
:103C6000E7802052B2402945410117B301006700A7
:103C70002356411197D501009385452017D50100A2
:103C8000130585B006C697B00100E780804F17D5B1
:103C900001001305253597B00100E780804EB24042
:103CA0002945410117B3010067008352411122C425
:103CB00006C6834705002A849DC797D501009385D2
:103CC000A52117D50100130525AC97B00100E780A9
:103CD000404B4C4017D501001305454797B00100F4
:103CE000E780204A3DA058410DEF97D5010093850C
:103CF000A51E17D50100130525A997B00100E7807F
:103D0000404817D501001305E54597B00100E7804D
:103D100040472244B2402945410117B301006700E2
:103D2000234BA1679386D7036313D70297D501006E
:103D30009385851A17D50100130505A597B00100D5
:103D4000E780204417D501001305C5427DBFED076C
:103D500097D501009385451817D501001305C5A215
:103D6000631BF70097B00100E780A04117D5010061
:103D70001305854159BF97B00100E78080404C4052
:103D800017D501001305454291BF411197D5010098
:103D90009385051017D501001305059F06C697B03A
:103DA0000100E780003EB2402945410117B3010000
:103DB00067000342397122DC26DA4AD82E842A8928
:103DC0008145B2844808714636C606DE97E0FFFF9B
:103DD000E780E03397F7FF1F9387075EDC4783D7C1
:103DE0000700231C2101231BF10097500000E780EE
:103DF0006055B246230DA10091E285469307001954
:103E00003ECE2686FD57A2854808A30DD100230289
:103E1000F10297500000E780C055F2506254D2542E
:103E20004259216182808546170300006700C3F86C
:103E30004111972700202396078E97170020238F84
:103E4000077C06C6170700200347C72D9307F00A13
:103E50006315F7029307F0F889451705002013054D
:103E6000652C17070020230FF72A97070020A38B44
:103E7000072A97600000E780200E97600000E78027
:103E8000E03A97600000E780203C81453705040058
:103E90009707002023AE07269707002023890726CF
:103EA000970700202398071E970700202396071CDA
:103EB00097070020239B072497070020239C0724B3
:103EC00097400000E780E09F014597600000E78091
:103ED000A01197D50100938525FE17D50100130584
:103EE000A58A970700202393072297B00100E78057
:103EF000402917D501001305653197B00100E7800F
:103F00004028B2402945410117B301006700432C06
:103F10004111814617F6FF1F1306464785451705D1
:103F200000200355251506C697D00000E78020978E
:103F300015C997D501009385E5F817D5010013053C
:103F4000A58497B00100E780C02317D501001305B1
:103F5000E51B97B00100E780C022294597B001001A
:103F6000E780002797D501009385C5F517D5010097
:103F70001305858197B00100E780A02017D50100C7
:103F80001305051A97B00100E780A01F294597B0D7
:103F90000100E780E02397F7FF1F9387E741DC47A5
:103FA000054797D501009385E5F12390E70017C5F4
:103FB00001001305657D97B00100E780801C17D5CF
:103FC00001001305251797B00100E780801BB24060
:103FD0002945410117B301006700831F411122C425
:103FE00097D50100938585F02A8417C50100130534
:103FF000A57906C697B00100E780A0184C4017D5F8
:1040000001001305250E97B00100E78080172945B0
:1040100097B00100E780C01B034704009307F00F2F
:10402000631FF70297D50100938545EC17C5010082
:104030001305857597B00100E780A0144C4017D593
:1040400001001305250B97B00100E780801322447F
:10405000B2402945410117B3010067006317B24020
:10406000224441018280411122C426C22A84AE84A6
:1040700017C501001305457197D501009385C5E269
:1040800006C697B00100E780C00F17D501001305E1
:10409000651697B00100E780C00E294597B0010072
:1040A000E780001397D50100938505E0970700206E
:1040B000239287FC17C501001305056D054497077A
:1040C0000020239797FA97070020239487FA9717E1
:1040D00000202398976497B00100E780800A971525
:1040E000002083D5056417D501001305251197B06D
:1040F0000100E7800009294597B00100E780400DE5
:1041000097170020238C875097F7FF1F9387C72AA4
:10411000DC4717F5FF1F0345E57403D70700C167A8
:10412000FD17631EF700B7E7040003A38705130616
:10413000000A85452244B240924441010283B7E718
:10414000040003A387051306001493050010DDB7D0
:10415000B1C1411122C417C501001305E5622E84C7
:1041600097D50100938585D306C697B00100E780F7
:104170004001A28517D501001305050797B001007E
:10418000E78020002244B2402945410117B30100D5
:10419000670003048280B7E70400FC471171A2DDC9
:1041A000CAD986DFA6DBCED72E8432892E86AA8591
:1041B00017050020130505F782971707002013073E
:1041C00067F683470700930680029387E70793F714
:1041D000F70FE3ECF610BA898A0717C70100130737
:1041E000E763BA979C43BA9782878D4797D50100BA
:1041F000938545D517C5010013050559630FF400D4
:1042000097B00100E780E0F717D50100130545924C
:1042100097B00100E780E0F6BDA497B00100E78009
:1042200040F617D501001305259297B00100E780ED
:1042300040F5294597B00100E78080F9930720F801
:104240001146970500209385E5ED4A851707002064
:10425000230AF7EC97070020A38707EC97000000DC
:10426000E780A0BC2A841DC997D50100938585CD20
:1042700017C501001305455197B00100E78060F0B4
:10428000A28517D501001305E58F97B00100E780DF
:1042900040EF294597B00100E78080F397D50100F2
:1042A000938545CA17C501001305054E97B0010057
:1042B000E78020ED17D501001305058E97B00100AA
:1042C000E78020EC294597B00100E78060F0416568
:1042D000930730FA0546970500209385A5E47D15E0
:1042E000170700202300F7E497000000E780E0B301
:1042F0002A841DC997D501009385C5C417C501003F
:104300001305854897B00100E780A0E7A28517D57F
:1043100001001305258797B00100E78080E6294555
:1043200097B00100E780C0EAB7E70400BC4F05661C
:10433000130606C8A14517F5FF1F0345A55282972E
:10434000FE506E54DE544E59BE5911618280914721
:104350006303F40297D501009385C5BE17C501001C
:104360001305854297B00100E780A0E117D5010051
:104370001305C58571BDB7E70400FC4F914517F5DE
:10438000FF1F0345254E829797D50100938585BB76
:1043900017C501001305453F97B00100E78060DEB7
:1043A00017D501001305458497B00100E78060DD53
:1043B000294597B00100E780A0E197500000E78011
:1043C000600F914535A485476303F40297D501003A
:1043D000938545B717C501001305053B97B001004C
:1043E000E78020DA17D501001305858115B59707F9
:1043F0000020239127CBB7E704000566BC4F1306C6
:1044000006C8C1450DBF8D476303F40297D501006F
:10441000938545B317C501001305053797B0010013
:10442000E78020D617C501001305457FD5B3930754
:1044300040F81146970500209385C5CE4A85170799
:1044400000202301F7CE97070020A38E07CC97000A
:104450000000E780809D2A84E30405EE97D50100E3
:10446000938545AE17C501001305053297B00100CD
:10447000E78020D1A28517C501001305A57097B06C
:104480000100E78000D0294597B00100E78040D4C3
:1044900045BD9147E31CF4F6B7E70400FC4F9305D4
:1044A000000217F5FF1F0345E53B829797D50100F2
:1044B000938545A917C501001305052D97B0010087
:1044C000E78020CC17C501001305C576F1BD8947EB
:1044D00063E3870297D501009385C5A617C5010040
:1044E0001305852A97B00100E780A0C917C5010010
:1044F0001305857531BB9704002083C4C4C2970798
:10450000002083C737C297D501009385A5A3A204D5
:1045100017C5010013054527DD8C97B00100E78022
:1045200040C6A28517C501001305457397B0010069
:10453000E78020C5C204294597B00100E78040C943
:10454000C1849305D4FF93960401C1824A8693F5F2
:10455000F50F17050020130515BD97300000E78003
:10456000003AE35F90DC930750F817070020230B15
:10457000F7BA83C73900228697050020938585BA4C
:1045800085074A8517070020A30FF7B8970000009A
:10459000E780A0892A84E30505DA97D50100938591
:1045A000659A17C501001305251E97B00100E78025
:1045B00040BDA28517D50100130505C2C9B58947BD
:1045C00063E3870297D501009385C59717C501005E
:1045D0001305851B97B00100E780A0BA17C501003D
:1045E0001305856935B197500000E780A0ECA285DE
:1045F00017050020130505B397600000E780C095FC
:1046000081B38D476303F40297D5010093858593A9
:1046100017C501001305451797B00100E78060B684
:1046200017C5010013050567E5B6B7660200014628
:10463000B7750200054597E0FF1FE780801A9307D2
:1046400060F817070020230FF7AC97070020A38C12
:1046500007AC93070006170700202307F7AC89472C
:1046600017070020A302F7AC97070020238F07AAA3
:1046700097070020A38B07AAC1471707002023072D
:10468000F7AA930720F917070020A301F7AA3146DC
:1046900097070020A38DA7A897050020938585A8DC
:1046A0004A8597070020238407A897F0FFFFE7803B
:1046B000C0772A84E30605C897D5010093858588CD
:1046C00017C501001305450C97B00100E78060ABEA
:1046D000A28517C501001305655D55B3B147630396
:1046E000F40297D501009385E58517C501001305F0
:1046F000A50997B00100E780C0A817C50100130500
:10470000A55C39B6B7E70400FC4F9305000417F524
:10471000FF1F03452515829797500000E78080D939
:10472000B145F9B5914763E3870297D501009385B9
:10473000658117C501001305250597B00100E780C5
:1047400040A417C501001305E559D9B4970400200A
:1047500083C4849D9707002083C7F79CA204DD8C47
:104760008E04B77702006D14BE942286A68517C505
:1047700001001305655897B00100E78080A0B7E7F6
:104780000400FC472286970500209385F5992800B0
:10479000829793160401C1823000A685094597E0EF
:1047A000FF1FE78000042A8409C917C5010013050B
:1047B000655697B00100E780A0B4930770F81946DA
:1047C00097050020938505964A8517070020230B3F
:1047D000F79497070020A389879497F0FFFFE7805D
:1047E000C0642A84E30E05B497C5010093858575DE
:1047F00017C50100130545F997B00100E7806098DF
:10480000A28517C501001305E55195B99947630BBA
:10481000F41297C501009385E57217C501001305D1
:10482000A5F697B00100E780C09517C501001305F4
:10483000E550F9BA914763E3870297C50100938574
:10484000657017C50100130525F497B00100E780D6
:10485000409317C501001305E54F5DBA970400208A
:1048600083C4848C9707002083C7F78BA204DD8C58
:104870008E04B77702006D14BE942286A68517C5F4
:1048800001001305654E97B00100E780808FB7E700
:104890000400FC472286970500209385F5882800B0
:1048A000829793160401C1823000A6850D4597E0DA
:1048B000FF1FE78000F32A8409C917C5010013050B
:1048C000654C97B00100E780A0A3930780F81946D4
:1048D00097050020938505854A8517070020230347
:1048E000F78497070020A381878497F0FFFFE78074
:1048F000C0532A84E30605A497C501009385856407
:1049000017C50100130545E897B00100E7806087EF
:10491000A28517C501001305254895B6994763037D
:10492000F40297C501009385E56117C501001305E1
:10493000A5E597B00100E780C08417C50100130505
:104940002547F9B0B7E70400FC4F9305000417F5BD
:10495000FF1F034525F1829797500000E78080B53F
:10496000994579B18D476303F40297C5010093859A
:10497000655D17C50100130525E197B00100E780CB
:10498000408017C501001305254459B017C5010023
:104990001305854497B00100E78080961305C01287
:1049A00097E0FF1FE780E099014597E0FFFFE78070
:1049B000A06E0D4597100000E780C038294597E0AC
:1049C000FF1FE780009897E0FF1FE78060888DBA9F
:1049D00099476303F40297C501009385A55617C54F
:1049E0000100130565DA97A00100E780807917C5FB
:1049F00001001305253F29B817F7FF1F0347D7729A
:104A000097F7FF1F83C7477222075D8F9166BA969B
:104A1000C2061166C1821306F6EF8D476365D602A2
:104A200097F7FF1F938747999C4B17F6FF1F034685
:104A3000966F9386C7002DC203D6070069CA8907FF
:104A4000E39CD7FE89471307A0F8114697F5FF1F8F
:104A50009385456D4A8597F6FF1F2385E66C17F70A
:104A6000FF1FA302F76C97F0FFFFE780003C2A844A
:104A7000E308058C97C501009385C54C17C5010057
:104A8000130585D097A00100E780A06FA28517C508
:104A9000010013056536E5B203D60700630EE60A8A
:104AA0008907E39BF6FE8D4779BF91476304F402C3
:104AB00097C501009385054917C501001305C5CCAD
:104AC00097A00100E780E06B17C50100130545348E
:104AD0006FF00FF4B7E70400FC4F9305000817F5DB
:104AE000FF1F034525D88297C9B897C50100938554
:104AF000654517C50100130525C997A00100E7808A
:104B0000406817C50100130525326FF06FF0239040
:104B1000E70017F5FF1F1305258A97400100E7807E
:104B2000C09297C501009385E54117C501001305A3
:104B3000A5C597A00100E780C06417C50100130553
:104B4000A52F97A00100E780C063294597A0010029
:104B5000E78000688147C5BD2390070017F5FF1F58
:104B60001305858597400100E780208E97C50100D9
:104B70009385453D17C50100130505C197A00100A8
:104B8000E780206017C501001305852C5DBF01116A
:104B900022CC06CE26CA4AC8834705002A849DC770
:104BA00097C501009385C53517C501001305C5BD1F
:104BB00097A00100E780E05C4C4017C50100130599
:104BC000E56897A00100E780C05BE1A05841B70706
:104BD000CF009387777D631DF7060359C50085478E
:104BE00004450356E5009716002083D686B363FC80
:104BF000270383C7040003C71400A207D98FC20785
:104C00007177C1871307C755639FE7006305D60C0B
:104C10006244F240CA8526854249D244056117E3C1
:104C2000FFFF6700E35B630AD600CA85268532C6AC
:104C300097E0FFFFE780C05A32466244F240CA85DF
:104C400026854249D244056117F3FFFF6700E3540C
:104C5000B707CC009387777D6317F70497C50100EA
:104C60009385052A17C50100130505B297A0010019
:104C7000E78020511C448356E4008355C40003C6DA
:104C8000070017C501001305E55D97A00100E78047
:104C9000404F6244F240D24442492945056117A37E
:104CA00001006700E352B707CE009387777D630466
:104CB000F70297C501009385A52417C501001305C8
:104CC000A5AC97A00100E780C04B4C4017C5010080
:104CD0001305854DFDB5F2406244D2444249056159
:104CE0008280B7E70400FC4741112E8606C622C425
:104CF00026C24AC02E842A89AA8517F5FF1F1305EC
:104D00006542829797C501009385852517C50100E7
:104D1000130585A797A00100E780A04697F5FF1F20
:104D200083C5454017C50100130585CB97A0010039
:104D3000E7802045294597A00100E780604997F466
:104D4000FF1F9384243E83C70400414793870706CF
:104D500093F7F70F636AF75E17C70100130747B6AB
:104D60008A07BA979C43BA9782879D476307F402E4
:104D700097C501009385C51E17C501001305C5A081
:104D800097A00100E780E03F17C501001305C5C5E6
:104D900097A00100E780E03E69AC97F7FF1F83C74B
:104DA0007738DDCB17F7FF1F0347F73797F7FF1F5C
:104DB00083C7673722075D8F97F7FF1F83C7C73603
:104DC000C2075D8F97F7FF1F83C71736E207D98F9A
:104DD00017F7FF1F232EF73283C7640097C5010022
:104DE0009385051817C501001305059A17F7FF1FCE
:104DF000230FF73097A00100E780A03897F7FF1F37
:104E0000938707318C4317F6FF1F0346463017C5BB
:104E10000100130525BF97A00100E78080362945D2
:104E200097A00100E780C03A97F7FF1FA38C072ED9
:104E30002244B24092440249930700F817F7FF1F3B
:104E40002302F72E9D4517F5FF1F1305A52D4101E0
:104E5000175300006700431097700000E78000E0E0
:104E600097F7FF1F2381A72C9357850017F7FF1F84
:104E7000A30BF72A935705012A8417F7FF1F230571
:104E8000F72A93578501014517F7FF1FA30EF7284F
:104E900097700000E780E0E097F7FF1F2387A728BF
:104EA00097C501009385C50B17C501001305C58D76
:104EB00097A00100E780E02C17F6FF1F0346E626C7
:104EC000A28517C50100130565B5B1B7CD476303CA
:104ED000F40297C501009385A50817C501001305C5
:104EE000A58A97A00100E780C02917C50100130516
:104EF00065B479BD97F7FF1F83C7E72317F7FF1F37
:104F000003475723A207D98FC207C18717F7FF1F8F
:104F1000231EF71E6345F004B7A71C81B7060001E6
:104F20000147938757DC17F5FF1F1305E593938619
:104F300036191946B305E50083C505000507AD8F91
:104F4000B387D702E318C7FE2167130707E0B3F75B
:104F5000E7029387072017F7FF1F2319F71AB7E710
:104F6000040003A387051306000A89452244B240C2
:104F70009244024917F5FF1F0345C58E4101028384
:104F80008D476303F40297C50100938565FD17B54E
:104F900001001305657F97A00100E780801E17C5FB
:104FA00001001305E5B8EDB317F4FF1F0344A41780
:104FB00097F7FF1F83C7171797C50100938545FA19
:104FC000220417B501001305257C5D8C97A0010014
:104FD000E780201BA28517C50100130525A797A010
:104FE0000100E780001A294597A00100E780401ED4
:104FF0000D4697F5FF1F9385E512228597F0FFFF79
:10500000E780A0E2AA8421C197C50100938545F5F8
:1050100017B501001305457797A00100E7806016DA
:10502000A68517C501001305A5A397A00100E78079
:1050300040152244B240924402492945410117A338
:1050400001006700E31897F7FF1F23958704B7E770
:105050000400116603A38705130606E8914539B7D6
:105060008D476303F40297C50100938565EF17B57B
:1050700001001305657197A00100E780801017C536
:1050800001001305A5B929B317F4FF1F0344A409B0
:1050900097F7FF1F83C7170997C50100938545EC54
:1050A000220417B501001305256E5D8C97A0010041
:1050B000E780200DA28517C501001305A59B97A0C9
:1050C0000100E780000C294597A00100E78040100F
:1050D0000D4697F5FF1F9385E504228597F0FFFFA6
:1050E000E780A0D4AA841DC197C50100938545E738
:1050F00017B501001305456997A00100E780600816
:10510000A68517C501001305259805B797F7FF1F5A
:10511000239487F6B7E70400116603A387051306F7
:1051200006E89305000299B5894763E3870297C5AE
:1051300001009385E5E217B501001305E56497A02A
:105140000100E780000417C501001305E5AF89B130
:1051500097F4FF1F83C424FD97F7FF1F83C797FCB5
:1051600097C501009385C5DFA20417B5010013059B
:10517000A561DD8C97A00100E780A000A68517C57A
:1051800001001305E59197A00100E78080FF294504
:1051900097A00100E780C003228697F5FF1F938543
:1051A00065F8268597F0FFFFE78020C82A84630E04
:1051B000051A97C501009385A5DA17B501001305F7
:1051C000A55C97A00100E780C0FBA28517C5010080
:1051D0001305458E99BD854763F9871883451900E6
:1051E0002244B24092440249B335B00097F7FF1F02
:1051F000238CB7EA17C501001305058D410117A3DC
:105200000100670003F8A2852244B24092444A8517
:105210000249410117130000670003B9994763036E
:10522000F40297C501009385A5D317B501001305B6
:10523000A55597A00100E780C0F417C5010013052C
:1052400065BAB9B617F4FF1F0344E4ED97F7FF1FE3
:1052500083C757ED97C50100938585D0220417B504
:105260000100130565525D8C97A00100E78060F195
:10527000A28517C501001305A58697A00100E78048
:1052800040F0294597A00100E78080F4194697F582
:10529000FF1F938525E9228597F0FFFFE780E0B89F
:1052A000AA841DC197C50100938585CB17B5010060
:1052B0001305854D97A00100E780A0ECA68517C5D2
:1052C00001001305E58295B397F7FF1F239487E448
:1052D000B7E70400116603A38705130606E89305E4
:1052E000000869B1854797C50100938565C717B563
:1052F000010013056549630BF40097A00100E780E6
:1053000040E817B501001305E57F59B497A00100E7
:10531000E78020E717C501001305458097A001002D
:10532000E78020E6294597A00100E78060EA224453
:10533000B2409244024997F7FF1F239907DC4101CD
:10534000177300006700038297C50100938545C16C
:1053500017B501001305454397A00100E78060E2FF
:1053600017C50100130545AC25B4B2402244924450
:10537000024941018280411106C622C426C239C1B8
:105380002A8497F00000E7800006AA8411EDB7E7B1
:105390000400BC474146814522858297B2402244A1
:1053A000268592444101828041657D1597F0000079
:1053B000E7804004B7E7040001E9BC474146814566
:1053C000228582978144D9BF0347E501FC479305B5
:1053D000900819E393050003AA9541462285829718
:1053E00085446DBF411106C622C426C24AC097F04B
:1053F0000000E78040FF55CD97700000E780C08631
:105400002A8497100000E7804046AA8422856373AF
:1054100094002685B7D7B0009387F75E63F3A702A1
:10542000B7E7B000130514009387F74F63E3A708AD
:105430002244B240924402494101177300006700C0
:1054400063838567938707F13E956364A400330502
:10545000F40097700000E780E08197700000E7801B
:10546000A0802A8963F6A40097100000E780A0427C
:1054700097C50100938545B017B501001305C530E8
:1054800097A00100E780E0CFA6864A86A28517B5DF
:1054900001001305254797A00100E78080CE224434
:1054A000B240924402492945410117A30100670017
:1054B00023D2B24022449244024941018280011128
:1054C00022CC37E404005C5C06CE354697C501006B
:1054D0009385C5B317D5010013054587829711E958
:1054E00017B501001305053097A00100E78040E1E2
:1054F00001A097E7FF1F9387A7373EC4B7F50700C2
:10550000856793870780814617E6FF1F1306C63518
:10551000E10519453EC697D0FF1FE780802C7C44EB
:10552000194697E5FF1F9385253417F5FF1F1305CF
:10553000A5B68297340017E6FF1F1306E63297C51B
:1055400001009385A5F517C501001305A5F6976021
:105550000000E78040262A841DCD97C50100938571
:10556000259C17B501001305252297A00100E780AF
:1055700040C1A28517C50100130545AA97A00100E7
:10558000E78020C0294597A00100E78060C4F24071
:1055900062440561828097E00000E780808B17C538
:1055A00001001305A59E97500000E780801A9750D0
:1055B0000100E780C04417E5FF1F130565DC975025
:1055C0000100E780602D17C501001305259D975048
:1055D0000100E78040452A8497600000E780408111
:1055E00097000100E780A01C97800100E780C0B50C
:1055F00097700000E78020DD97600000E78040F7AB
:1056000097300100E78000DE97C501009385459142
:1056100017B501001305451719C897A00100E780C9
:1056200040B6A28517C50100130585A181BF97A0CB
:105630000100E78000B517C501001305A5A297A0DA
:105640000100E78000B4294597A00100E78040B839
:1056500097300100E780E0B997F00000E780A0D81C
:1056600069CD97E7FF1F9387A7C483D707008545B8
:1056700037050400170700202315F70A97200000BC
:10568000E780202497C501009385858917B501001F
:105690001305850F97A00100E780A0AE17C5010094
:1056A0001305C59D97A00100E780A0AD294597A0EF
:1056B0000100E780E0B18547170700202300F7F6D7
:1056C00097E7FF1F938747CFDC4703D70700C167E2
:1056D000FD176316F70097F0FFFFE780A0839700A0
:1056E0000000E78060D097100000E78020EC1705ED
:1056F00000200355050397400000E780605B0545E7
:1057000097500000E780408E97500000E780C0B3BC
:1057100097C501009385C58017B501001305C5061F
:1057200097A00100E780E0A517C501001305459A81
:1057300097A00100E780E0A4B1B597B5010093857B
:10574000257E17B501001305250497F7FF1F239F3A
:10575000079A97A00100E780C0A297C50100938532
:10576000259417C501001305259497A00100E78033
:1057700040A1294597A00100E78080A501459750E9
:105780000000E780608669B7411122C437E4040055
:105790008327041A06C6829797400000E7800055C9
:1057A000832704081705000013050503829797E770
:1057B000FF1F2389A70A17E5FF1F1305E5BF9740C1
:1057C0000000E780E0052244B240410117030000D9
:1057D000670023CF011122CC06CE26CA4AC84EC686
:1057E00093F715002E84B5CB97E0FFFFE78080721A
:1057F000930710F817F7FF1F2306F79297F7FF1F7D
:1058000083D7078717F7FF1FA30EF7909145A18352
:1058100017F5FF1F1305059117F7FF1F2305F790D5
:1058200097F7FF1FA381079097400000E780C072A1
:10583000B7E70400BC4F130600149305001017E5EA
:10584000FF1F03452502829713451400F24062446E
:10585000D2444249B2490561828093F70510B1C72D
:10586000054597400000E780207817050020035584
:1058700045EB97400000E780A04397000000E780D9
:10588000A0B697100000E78060D297F7FF1F83C78C
:10589000B79889E797500000E7804099975000003B
:1058A000E780809A1345041055B793F72500E9CF98
:1058B00017F7FF1F0357878569C7AD64B719004005
:1058C0009384A4AA23A0990097F6FF1F9386468489
:1058D000944297C701009387679517F6FF1F034609
:1058E0000683814517C501001305459597600000A3
:1058F000E780601723A0990097E7FF1F2392A79CDA
:105900002A8941C197B501009385856217B50100C9
:10591000130585E797A00100E780A086CA8517B523
:1059200001001305E50097A00100E7808085294567
:1059300097A00100E780C08997E7FF1F2398077CA5
:10594000930710F817E7FF1F230EF77C97E7FF1F59
:1059500083D7077217E7FF1FA306F77CA18317E71A
:10596000FF1F2302F77C91458D4717E5FF1F1305A5
:10597000657B17E7FF1FA308F77A97400000E780D1
:10598000A05D13452400D9B593F74500D1C397B561
:1059900001009385E55917B501001305E5DE9790E1
:1059A0000100E780007E17B50100130525FA9790E6
:1059B0000100E780007D294597A00100E780408134
:1059C000930720F817E7FF1F230EF77497E7FF1FD1
:1059D00083D7476C17E7FF1FA306F774A18317E768
:1059E000FF1F2302F774854717E7FF1FA30DF77208
:1059F00097400000E78000AC17E5FF1F1305857294
:105A0000914597400000E7802055134544003DBD77
:105A100093F78500A9C797B501009385655117B520
:105A20000100130565D697900100E780807517B5D2
:105A300001001305E5F297900100E7808074294585
:105A400097900100E780C07897E7FF1F2390076CCD
:105A500097600000E780001113458400C5BB93F7F1
:105A60000501D1C3854517E5FF1F0355A562975072
:105A70000100E78000C697B501009385654B17B517
:105A80000100130565D097900100E780806F17B57E
:105A90000100130525EE97900100E780806E2945EF
:105AA00097900100E780C072930730F817E7FF1F57
:105AB000230AF76697E7FF1F83D7C75D17E7FF1F26
:105AC000A302F76617E5FF1F1305C565A1838D4582
:105AD00017E7FF1F2309F76497400000E780C047DE
:105AE00013450401A5B393F70502D1C797B501008B
:105AF0009385054417B50100130505C9979001006A
:105B0000E780206817B50100130505E997900100AB
:105B1000E7802067294597900100E780606B930735
:105B200040F817E7FF1F230FF75E97E7FF1F83D7A4
:105B3000A75417E7FF1FA307F75EA18317E7FF1F0F
:105B40002303F75E854717E7FF1FA30EF75C97E770
:105B5000FF1F2393075297400000E780A09517E5A9
:105B6000FF1F1305255C914597400000E780C03E6C
:105B700013450402E1B993F70504FDC397B501008D
:105B80009385053B17B50100130505C097900100EB
:105B9000E780205F17B50100130585E197900100AC
:105BA000E780205E294597900100E780606297E7D3
:105BB000FF1F83C727571307700A6386E70613077B
:105BC000800A638CE7081307600A6393E70493076E
:105BD00060F817E7FF1F2307F75497E7FF1F83D7E6
:105BE000C75217E7FF1FA30FF752A18317E7FF1F45
:105BF000230BF752854717E7FF1FA30AF752B1455A
:105C000017E5FF1F1305055297400000E780C034D9
:105C100097400000E780008A1345040497E7FF1FC0
:105C20002395074E25B1930770F817E7FF1F230B45
:105C3000F74E97E7FF1F83D7474D17E7FF1FA303D3
:105C4000F74EA18317E7FF1F230FF74C854717E790
:105C5000FF1FA30BF74C994565B7930780F8F1B781
:105C600093F705080145E38307BE97B501009385C7
:105C7000252C17B50100130525B197900100E78089
:105C8000405017B50100130525D497900100E78017
:105C9000404F294597900100E78080539307A0F873
:105CA00017E7FF1F2300F74897E7FF1F83D78746B3
:105CB00017E7FF1FA308F746A18317E7FF1F230479
:105CC000F746854717E7FF1FA30FF74497E7FF1F26
:105CD0002392074497300000E780C07D17E5FF1F3F
:105CE00013054544914597400000E780E0261345A1
:105CF0000408A9BE411106C697E0FFFFE780C00B6C
:105D00000DC197E7FF1F83D7473A850717E7FF1FA6
:105D1000231DF73897E7FF1F239AA738B2404101A8
:105D2000828097E7FF1F83D78738850717E7FF1F14
:105D3000231FF736E5B78546170300006700C3FB4E
:105D4000411122C491462A8417E6FF1F1306864B91
:105D50009D652D4506C697D0FF1FE78080A8B7F741
:105D6000070003C70701A5476313F70001A09306C7
:105D7000001001469D65254597D0FF1FE78060A66E
:105D800097E7FF1F238087482244B240914617E6D9
:105D9000FF1F130626479D652945410117D3FF1FA5
:105DA000670023A41171CED7B7E9040083A7C90403
:105DB000CAD917E9FF1F1309E936A2DD2E8686DF4F
:105DC000A6DB2E84AA854A85829797E7FF1F83C7A3
:105DD00067351307700A6385E710636DF7001307D3
:105DE000600A6385E704FE506E54DE544E59BE5976
:105DF000116182801307800A6385E7161307900AF2
:105E0000E393E7FE8D476306F41C97B50100938585
:105E1000E55017B501001305259797900100E7801D
:105E2000403617B501001305A54C25A08D47630C1E
:105E3000F40297B501009385654E17B5010013056F
:105E4000A59497900100E780C03317B501001305B2
:105E5000654397900100E780C03229459790010083
:105E6000E780003749B7854717B50100130545435B
:105E700017E7FF1F230AF72297900100E7804048A9
:105E8000B7750200B76602000146054597D0FF1FAF
:105E9000E7802095930760F817E7FF1F2304F72892
:105EA00097E7FF1FA38107289307002617E7FF1F27
:105EB000232CF726E5779387072117E7FF1F231782
:105EC000F726B14597E7FF1F2383072697E7FF1FB4
:105ED000A38FA7244A8597000000E780E01621B72A
:105EE000914763E3870297B501009385254317B572
:105EF00001001305658997900100E780802817B598
:105F000001001305E53BB1B797E4FF1F83C4C4212B
:105F100097E7FF1F83C73721A204DD8C83A7C9043D
:105F20006D14228697E5FF1F938515202800829720
:105F30008E0493160401B7750200C1823000A69545
:105F4000094597D0FF1FE780C089930770F817E7CE
:105F5000FF1F2309F71C994597E7FF1FA386A71C7E
:105F600095BF914763E3870297B501009385053B91
:105F700017B501001305458197900100E780602067
:105F800017B5010013054535E9B597E4FF1F83C434
:105F9000A41997E7FF1F83C71719A204DD8C83A7F5
:105FA000C9046D14228697E5FF1F9385F517280015
:105FB00082978E0493160401B7750200C1823000E7
:105FC000A6950D4597D0FF1FE780A081930780F825
:105FD000BDBF17B501001305E53297900100E780BA
:105FE0002032930790F82304F100834719008D4570
:105FF0002800A304F100834729002305F10097003E
:106000000000E78060041305C01297C0FF1FE780FF
:106010004033014597D0FFFFE78000080D4597000A
:106020000000E78020D2294597C0FF1FE78060313C
:1060300097C0FF1FE780C0217DB397E7FF1F23AB09
:10604000A71C828097E7FF1F9387C71C03A3070045
:10605000630303000283174300006700E3EF41116D
:106060004AC097F6FF1F83D6C66B328917D6FF1F2B
:106070000356A63622C426C206C62A84AE849700DA
:106080000000E780E06929C921C8994763F69704B1
:106090008347140003470400A207D98F1397870092
:1060A000A183D98FC2073167C1831307C755639591
:1060B000E70297D7FF1F83D74732A301F400A183DC
:1060C0002302F40097F7FF1F83D7A76591C7A302A8
:1060D000F400A1832303F40097F7FF1F83C707543D
:1060E000A1CB2686A28517D5FF1F0355052F970044
:1060F0000000E78080C4630F090297F7FF1F83C782
:10610000E7518DEB97E7FF1F83C7071185C79DC038
:1061100097E7FF1F83C747F991EF22852244B240DA
:106120000249A68592444101174300006700C3E27B
:10613000E31A09FCB24022449244024941018280A0
:106140000145828097A70100938787549C430111E2
:106150006800914506CE3EC697000000E780C0EE7D
:10616000F240056182808D4763F6B708011126CAA7
:1061700006CE22CC0344350097E4FF1F83C4D40924
:1061800097B501009385451BB337800017E7FF1FC4
:10619000A304F70809C497B501009385A51A17B59C
:1061A00001001305A51A97900100E78080FD97E78D
:1061B000FF1F83C777066386970097000000E7807C
:1061C000404697400000E78020089967938757EE84
:1061D0002316F100680085479145A3078100230736
:1061E000F10097000000E78020E6F2406244D244CC
:1061F000056182808280894763F7B708011122CC4C
:1062000006CE26CA8344250085472A84639DF4046C
:10621000914763F5B70403454500834734002205E1
:106220005D8D97D7FF1F239AA71A97000000E7807C
:1062300000589967938767EE2314F1008347340071
:1062400023059100A305F1008347440095452800EC
:106250002306F10097000000E78000DFF24062446F
:10626000D24405618280FDF89967938767EE231415
:10627000F10097D7FF1F83D74716A305F100230529
:106280000100A183E1B782800111996722CCD51763
:1062900017F4FF1F130484382314F100834704000C
:1062A00026CA97F4FF1F9384C4472305F10083D7C0
:1062B000040028009545A305F100A18306CE23061E
:1062C000F10097000000E78020D803D60400834542
:1062D000040017B501001305650897900100E780D9
:1062E00040EAF2406244D244056182809D67797140
:1062F000D9172316F10097F7FF1F9387273283C71B
:1063000007001305F10006D62307F10097F0FFFF01
:10631000E780A00609E9B7E70400BC47414681458C
:106320001305F10082976800CD4597000000E780D3
:10633000A0D197F5FF1F83C5652E17B50100130582
:10634000E50497900100E780C0E3B2504561828088
:1063500063080516411126C206C622C44AC097E743
:10636000FF1F83C777EB97F4FF1F83C4242B99C3C8
:1063700093E424002A8497100000E780C00119C12B
:1063800093E4040137E90400832789042285130676
:10639000200381458297930750FA2300F400930766
:1063A000A005A300F4008D472301F4009147A30149
:1063B000F4009307D005A302F40097F7FF1F83D7DB
:1063C00047362304F400A183A304F40097D7FF1FEA
:1063D00083D7A700230394002305F4009304C4008B
:1063E000A18323020400A305F400268597F0FFFF94
:1063F000E780A0F819E58327890441468145268571
:10640000829797D7FF1F83D7E7FA230EF400A18363
:10641000A30EF40093070002230FF400930710FA71
:10642000A30FF4009D472300F402A3000402B7E782
:106430000400FC4713052402194697D5FF1F9385D6
:10644000A542829797E7FF1F83D767C62304F4020C
:10645000A183A304F40297E7FF1F83D707C5230591
:10646000F402A183A305F40297E7FF1F938707C4F3
:10647000839707002285930500032306F402C207D1
:10648000C183A183A306F40297D7FF1F938747E335
:10649000839707002307F402C207C183A183A307E0
:1064A000F40297000000E780A0232308A4022181C2
:1064B000A308A402B24022449244024941018280CE
:1064C00082805D71E17793C777FF1305E10086C68F
:1064D0002316F10097000000E780C0E768009305ED
:1064E000400397000000E78020B6B64061618280DB
:1064F0005DC9411122C426C206C6930750FA230083
:10650000F5009307A005A300F50089472301F500D6
:106510009147A301F5009307D005A302F50097F773
:10652000FF1F9387A70F83C707009304C5002A8422
:106530002303F50097E7FF1F938717CE83C7070054
:1065400023020500A303F50097F7FF1F83D7671DFC
:106550002304F500A183A304F50097D7FF1F83D779
:10656000C7E72305F500A183A305F500268597F06D
:10657000FFFFE78080E001E9B7E70400BC47414640
:106580008145268582972285F14597000000E780A6
:106590002015230EA4002181A30EA400B2402244A2
:1065A00092444101828082805D710A8586C6A2C4C0
:1065B00097000000E78000F437E404007C448A85FB
:1065C0000810794682973C441305E103094681454A
:1065D0008297101093050002014597D0FFFFE780D6
:1065E000E011B640264461618280411122C426C276
:1065F0002A84AE848566AA850146254506C697C0CD
:10660000FF1FE780001EA2852244B24026869244E6
:10661000A1462945410117C3FF1F6700831C0111D3
:10662000B7C7A55A22CC9387C73317E4FF1F1304BB
:10663000B4BE3EC4834704002C00196506CE3EC696
:1066400097000000E780A0FA8345040017B5010019
:10665000130545DE97900100E780A0B2F240624446
:10666000056182800111A146300099652D4522CC3B
:1066700006CE97C0FF1FE780C016A24737C4A55AB1
:106680001304C43363958702B24517B5010013059F
:1066900025D2B335B00097E7FF1FA38FB7B6979009
:1066A0000100E78000AEF24062440561828091659E
:1066B000A1463000938505F02D4597C0FF1FE78068
:1066C0004012A247E38287FC97E7FF1FA38607B427
:1066D000814517B501001305E5CFD1B7C1676976CC
:1066E0008146FD1705061397060141836364B700D1
:1066F0003E8582803307D50003470700B98F2147C5
:1067000013F81700858363050800B18FC207C183A2
:106710007D171377F70F6DF78506F1B741C5A547CC
:10672000054763F2B7088347150003470500316842
:10673000A207D98F13978700A183D98FC207C1837E
:106740001308C855054763900707411106C622C4C0
:1067500026C203442500914763F087049307540041
:1067600063ECF502A301C50021822302C500930456
:10677000340091C6A302D500A1822303D5002A8448
:10678000A68597000000E780A0F526942300A400CA
:106790002181A300A4000147B240224492443A85DB
:1067A0004101828005473A8582800111B7C7A55A09
:1067B00022CC9387E7342A842AC62C00156506CE9E
:1067C0003EC497000000E78080E2A28517B5010073
:1067D000130545C897900100E780A09A9700000034
:1067E000E780C0DCF2406244056182800111A1466D
:1067F000300095652D4522CC06CE97C0FF1FE7805F
:1068000040FEA24737C4A55A1304E43463958702B7
:10681000B24517B501001305E5BD97D7FF1F239EAD
:10682000B7BAC205C18197900100E7808095F24018
:106830006244056182809165A1463000938505EE32
:106840002D4597C0FF1FE780C0F9A247E38287FC70
:10685000D14717D7FF1F2312F7B8D14517B501004D
:10686000130545BBC9B70111A146300091652D45FF
:1068700006CE97C0FF1FE780C0F62247B7C7A55ACC
:106880009387073501456313F7003245F2400561F0
:1068900082800111B7C7A55A2AC6938707352C00F5
:1068A000116506CE3EC497000000E78040D4F24058
:1068B000056182804DC5411126C206C622C4AE8440
:1068C000D1C92A8497100000E78080AD97E7FF1FA9
:1068D00083C7879499C7A685228597300000E780F3
:1068E000A06797F7FF1F83C767D3ADC7954763F3CB
:1068F00097068347040013073005639DE70483462A
:106900001400130750046397E6048346240013071A
:1069100010046391E60403473400631DF702034744
:1069200044009307B0046317F7020347540093072A
:1069300090056311F702A2852244B2402686924454
:1069400017D5FF1F035565A98D46410117F3FFFFBA
:106950006700833AB240224492444101828082809F
:1069600001114EC606CE22CC26CA4AC893F715009E
:10697000AE899DCBAD67371700409387A7AA1CC38C
:10698000B7E70400BC4F13060019854517D5FF1F54
:10699000034585A4829713C51900F2406244D2448E
:1069A0004249B2490561828093F725000145F5D738
:1069B00017F7FF1F0357C7D6954763F9E70C014444
:1069C00017F6FF1F1306C6C59306300513055004BE
:1069D000130810049308B004130390059307640090
:1069E0006374F7043A847D5997F4FF1F83C444C34A
:1069F00097F7FF1F83C7D7C2A204DD8CAD679387CB
:106A0000B755638BF41463E3970AA9679387A75577
:106A1000638EF414A28517F5FF1F130565C0970058
:106A20000000E78060E9E9A0B307860083C507009E
:106A3000639AD50483C517006396A50483C5270010
:106A40006392050583C53700639ED50283C5470061
:106A5000639A150383C757006396670222890DE87E
:106A600097F5FF1F83D5C5CBB3852541C20517F523
:106A7000FF1F1305E5BAC1814A9597000000E78022
:106A8000A0E3E1A005044204418089BF3A847D5916
:106A90008547E3EB87F45DC4854517F5FF1F1305B4
:106AA00025B897000000E78020E169A8B1679387C7
:106AB000C7556389F404B5679387D755E39CF4F40D
:106AC000A28517F5FF1F1305A5B597300000E780D5
:106AD000A0488947630EF4009305E4FFC205C18115
:106AE00017F5FF1F1305E5B397100000E780408BF3
:106AF000A68517B501001305A59797800100E780CB
:106B0000406889A097200000E780603A9710000055
:106B1000E780608811C9A28517F5FF1F130545B0EE
:106B200097100000E780C0870546A28517F5FF1F74
:106B3000130505AF97F0FFFFE780A05297200000F4
:106B4000E780E036FD57E31DF9F097F7FF1F239923
:106B500007BC13C5290091B5A28517F5FF1F1305C2
:106B600025AC97F0FFFFE780E05D59B7A28517F5E8
:106B7000FF1F1305E5AA97F0FFFFE780E05C8DBFDC
:106B8000411122C437E404005C5C06C6354697A573
:106B900001009385A54717B501001305251B8297B2
:106BA00011E917B501001305E58D97800100E78015
:106BB000207501A08327041C82972A84054597C06D
:106BC0000000E780602897700100E78080AD977033
:106BD0000100E780808297B00000E780E0392285DD
:106BE000B2402244410182804111054506C622C4BB
:106BF00026C297C0FFFFE78000341305A00497B0BA
:106C0000FF1FE780C04A757585457D1597C0FFFF5A
:106C1000E780A01D7D7585451305F53697C0FFFFFC
:106C2000E7800027371400408327840A8D45130529
:106C3000002093E707202324F40A97C0FFFFE78092
:106C4000C01AB7E4040097C0FFFFE780E05FC858B0
:106C500097800100E780C06A17B501001305050F92
:106C600097800100E780C0698327840C85454145F2
:106C700093E707082324F40C97C0FFFFE780402127
:106C80008D451305000897C0FFFFE780602097C07F
:106C9000FFFFE780404D37A507001305051297C099
:106CA000FFFFE780E048014597C0FFFFE780004F06
:106CB00095450545894717F7FF1F2305F7A697C098
:106CC000FFFFE780404FB7E700E013070006238D82
:106CD000E7403707000423A0E71097D0FFFFE780C5
:106CE000C0D097D0FFFFE780C0E297000000E780A8
:106CF00060E997000000E780209797000000E78098
:106D000020AF97F0FFFFE78060A897000000E780C2
:106D1000606A97000000E780801083A704081705C9
:106D20000000130525C4829797C7FF1F2386A76A13
:106D3000BC4C130600648545829797B0FF1FE7801F
:106D4000206B01458280AD67371700409387A7AA63
:106D50001CC3B7E700E03707400023A0E718010095
:106D60000100B7F7070003C70701A5476316F7003F
:106D70009397450191C301A04111AE860146AA85B2
:106D8000254506C697C0FF1FE780A0A5B240B7E71C
:106D900000E03707400023A0E71041018280411145
:106DA000B2862E86AA852D4506C697C0FF1FE780AE
:106DB00040A3B2400145410182809307000463EC87
:106DC000C7041D71A2CC2A840808A6CACAC886CEE8
:106DD00032C697800100E780602FAD67371700400B
:106DE0009387A7AA1CC3B7E400E03709400023A09B
:106DF000241901000100B2461008A285294597C058
:106E0000FF1FE780009EF640664423A02411D6446D
:106E10004649256182803955828041110D658D4535
:106E200006C697C0FFFFE78040FCB71700408D669D
:106E300023A6D70A17F5FF1F1305058F1387C70A67
:106E40009387870A1CC15CC5856689675CC958C180
:106E500014C518C9B7E70400B24003A3871E410157
:106E600002838145B307B5008387070089E71723AD
:106E700000006700630A8505C205C181E5B74111BD
:106E800006C6B94763EEB70017A5010013050578DC
:106E900097000000E78020FDB24005454101828057
:106EA0008347E500130710036390E702854717F750
:106EB000FF1F230DF79617A501001305657797F7B8
:106EC000FF1F23940796E9B713070003E39EE7FA31
:106ED00097F7FF1F238C079497F7FF1F23970794BB
:106EE00017A501001305457665B7411126C2E9775C
:106EF00097F4FF1F9384C49322C49387A7552E84CD
:106F00002381B4002E86AA8517F5FF1F13058592ED
:106F100006C62390F400A381040097800100E78057
:106F2000E01A93052400C205C18117F5FF1F130560
:106F3000459097F0FFFFE780A07AB3878400238213
:106F4000A7002181A382A700930564002244B240D8
:106F500026859244C205C1814101172300006700C4
:106F6000A3FB09C99307000463E6B70017030000F9
:106F70006700E3F782809306F00F0307060019E726
:106F80009307F00F63F0B7022E8582809387150078
:106F9000C207C183E3E6F6FEAA952380E500050655
:106FA000BE85E1BF2E9523000500F9BF01111C0825
:106FB000B69706CE238A07FE5C00BE9617A801008E
:106FC000130888741377F600429703470700FD16ED
:106FD00011822380E600E397D7FE3E8697000000EB
:106FE000E780A0F9F240056182800111580006CEC9
:106FF00023070100A947BA8829482543B376060329
:10700000FD1793F7F70F93860603A304D700B35633
:1070100006036375C3007D173686EDF33386F800EB
:1070200097000000E78060F5F240056182803971C9
:1070300017A601001306C66506DE22DC26DA2A84BE
:107040004AD84ED697000000E78020F3AA8517E6BD
:10705000FF1F0356066D9146228597000000E780CA
:1070600020F597E7FF1F83C7675BAA8517A6010076
:107070001306865F89C717A601001306665E228580
:1070800097000000E78060EFAA8517A601001306AD
:107090006660228597000000E78020EEAA8517A68B
:1070A00001001306A65F228597000000E780E0EC50
:1070B000AA851146228597000000E78040F3AA8543
:1070C00017B60100130686BC228597000000E780F2
:1070D000C0EAAA8517A601001306C65C22859700A0
:1070E0000000E78080E9AA8517B60100130606BAFA
:1070F000228597000000E78040E8AA851306D005A6
:10710000228597000000E78080EE97D7FF1F83C796
:10711000B710AA8517A601001306865589E717A69A
:10712000010013066655228597000000E780E0E421
:10713000AA8517A60100130626572285970000008E
:10714000E780A0E337A60700AA851306061222856A
:1071500097000000E780A0E9AA8517A601001306A2
:107160002655228597000000E78020E197E7FF1F62
:1071700083C7075DAA8517A601001306665089E735
:1071800017A6010013064650228597000000E780ED
:10719000C0DEAA8517A60100130646522285970075
:1071A0000000E78080DDAA8517A60100130686513E
:1071B000228597000000E78040DCAA8517A6010021
:1071C0001306C650228597000000E78000DB914639
:1071D000AA8517C6FF1F0356E61D228597000000EB
:1071E000E78000DD2AC697500000E780E0A7B2459F
:1071F000AA8417A601001306A64D22859700000059
:10720000E780A0D713D60401AA8589461376F60F26
:10721000228597000000E780A0D9139604019146CB
:10722000AA854182228597000000E78060D8AA8560
:1072300017A601001306464A228597000000E78042
:10724000C0D39146AA8517C6FF1F0356061922858B
:1072500097000000E780C0D5AA8517A60100130695
:107260002648228597000000E78020D19146AA8514
:1072700017D6FF1F0356A6E3228597000000E7807C
:1072800020D3AA8517A6010013060646228597007B
:107290000000E78080CE9146AA8517D6FF1F0356CF
:1072A000C6E0228597000000E78080D0AA8517A657
:1072B00001001306E643228597000000E780E0CB3B
:1072C0009146AA8517D6FF1F035646DE22859700F2
:1072D0000000E780E0CDAA8517A6010013068641CD
:1072E000228597000000E78040C9AA85914617C60D
:1072F000FF1F0356E6FC228597000000E78040CB85
:10730000AA8517A601001306663F22859700000094
:10731000E780A0C6AA85814497C9FF1F9389C954F5
:107320001949B387340103C60700894622859700AF
:107330000000E780E0C78504AA85E39424FF17A630
:1073400001001306263C228597000000E780E0C27A
:107350002AC6080897E0FFFFE7802002B24504082C
:107360001309010283C7040003C614009146A20753
:107370005D8E228597000000E78080C38904AA857E
:10738000E31299FEF2506254D2544259B25921612B
:10739000828017E5FF1F0345A53A828097E7FF1F0C
:1073A00083C7C74889E7172300006700E3B68280D8
:1073B00097E7FF1F83C7274C99EF411106C6972017
:1073C0000000E78040ADB240854717E7FF1F230468
:1073D000F74A4101828082806302054E6380054E38
:1073E0002971B7064000232E1112232C8112232A63
:1073F00091122328211323263113232441132322FE
:10740000511323206113232E7111232C8111232A60
:1074100091112328A1112326B11101475948A5062E
:107420009319070193D9090163F1B902B307E50084
:1074300083C70700D91793F7F70F6368F800B3D72E
:10744000F600858B13061700A1E3B3893541C20905
:1074500093D90901B9472E89AA8463F93703330404
:10746000E500394697A50100938585082285978018
:107470000100E78040C319E9CE852285970000000E
:10748000E78020A025E5F1A4328759BF97E7FF1FC9
:1074900083C7C739638F0724BD6A396C014A17EB6C
:1074A000FF1F130B2B2A938BFA55938CFA66130D3F
:1074B000EC5505A8B387440183C6070097E7FF1F73
:1074C00083D7A736A5E39307A005639BF6008547FE
:1074D00017E7FF1F231BF73497E7FF1F2384D726E7
:1074E000050A93170A01C183E3E627FD8320C11330
:1074F0000324811383244113032901138329C11217
:10750000032A8112832A4112032B0112832BC111FA
:10751000032C8111832C4111032D0111832DC110E6
:1075200031618280854D639BB7039307500A639E48
:10753000F600894717E7FF1F2319F72E930750FA24
:1075400017E7FF1FA300F72061BF9307A005E3899A
:10755000F6F897E7FF1F239A072C59B713871700F0
:107560004207DA9741832380D70017E6FF1F231EC7
:10757000E62A8D47E3F6E7F617E4FF1F0344B41C41
:1075800097E7FF1F83C7271C22045D8C9307F4FF36
:10759000C207C1839306F00DE3EDF6FA930764008A
:1075A000C207C183E31EF7F293052400C205C1811F
:1075B00017E5FF1F1305251997F0FFFFE78040121D
:1075C00033078B008347570003474700A207D98F33
:1075D00017E7FF1F231B07246312F5108149630D72
:1075E000B40197E9FF1F83C92916A20997E7FF1F76
:1075F00083C79715B3E9F900170500001305A59691
:1076000097F0FFFFE780A0A36385790963EF3B0351
:107610006388A9059307EC656383F90697E7FF1F65
:1076200083C7871205476380E70881CB1387A705C7
:107630001377F70F8D4663F9E6081307F007230069
:10764000E100A300F100894595A863899905938716
:10765000FA77E395F9FC97F0FFFFE780C0E611A801
:10766000A28517E5FF1F1305250E97F0FFFFE780A2
:10767000C0AF014597F0FFFFE780609C95B5A285FC
:1076800017E5FF1F1305450C97F0FFFFE780E0B6F5
:10769000CDB797F0FFFFE78060BFE1BF97F0FFFF36
:1076A000E78000C5F9B7930710F813051100230010
:1076B000F10097F0FFFFE780E0E3FD450A859700C2
:1076C0000000E780C08275B7A28517E5FF1F13058C
:1076D000A50797E0FFFFE780206D61BF9307F007E4
:1076E00089450A852310F10097000000E78020807B
:1076F000C5BB15476375270503C604009306500BE9
:107700000147631FD60203C614009306B0053E87E7
:107710006318D602CA85268597F0FFFFE78080A20E
:1077200011C917A501001305A5DD97F0FFFFE7803C
:1077300080736DBB17A501001305C5DDFDB70147BB
:10774000B70640005946A506131407014180636936
:107750002401CA85268597C0FFFFE78060A879B31A
:10776000B389E40083C70900D91793F7F70F63675C
:10777000F600B3D7F600858B0507F9F73304894087
:1077800042044180BD4763FD8706414697A501003D
:10779000938545DA4E8597800100E780C09017A653
:1077A0000100130666DA05C13D4697A501009385E1
:1077B000E5DA4E8597800100E780E08E21E917A683
:1077C00001001306A6DA81450A8597F0FFFFE780DE
:1077D000C07AAA850A8597000000E7808085AA857F
:1077E000179601001306C6590A8597F0FFFFE78038
:1077F000C078AA850A8597100000E780E071FDB186
:10780000E304F4FAB547E3F687F439A8C147E3FB8C
:1078100087FE454697A50100938585D64E859780BE
:107820000100E780408815D5394697A5010093856A
:1078300025CC4E8597800100E780E08601E5A28592
:107840004E852DB9394697A501009385A5D44E855F
:1078500097800100E7802085E30D05EEC147E3FA3C
:1078600087EE414697A501009385C5D34E85978045
:107870000100E7804083E31E05EC83C7090113077D
:107880001003639CE700854717E7FF1F230AF7EA09
:1078900017A50100130545D249BD1307000317A51D
:1078A0000100130565D4E392E7E897E7FF1F2389FA
:1078B00007E817A501001305A5D185BD82804111F8
:1078C00026C2AE848D4522C406C62A8497B0FFFF27
:1078D000E780005CB717004099C803A5C70C418D2D
:1078E00023A6A70CB240224492444101828003A502
:1078F000870C418D23A4A70CF5B7834705000347E8
:107900001500A207D98FC2076177C1871307272007
:10791000639AE7008345250037050400170300003C
:10792000670023FA828017E6FF1F130626F58147BA
:10793000B2861303F00FA9483308F6000348080085
:1079400013F7F70F6307A80C630668008507E39534
:1079500017FF2947B387E6002380A70097E7FF1F9B
:10796000938787F25DA8411113D76500134717006D
:1079700006C693F63500058B954791CA054699478B
:107980006387C60009469D476383C600A14713F677
:1079900045003336C00093F68503050685C2A14530
:1079A000638BB604E145638AB6049305800263885D
:1079B000B604930580036393B600914697E5FF1FD5
:1079C0002389F51297E5FF1F2384C51297E5FF1F52
:1079D000A380D512BE8517A501001305E5D69770C3
:1079E0000100E780007AB240854717E7FF1FA30236
:1079F000F710410182808546D1B78946C1B78D46CF
:107A000075BF17A501001305A5D617730100670000
:107A1000437717E7FF1F130727E7BA972380B700BD
:107A2000E147E302F5F493077002E30CF5FC828072
:107A30002A8723800500814717E5FF1F130505E40A
:107A40001308F00F2946B306F50083C606006396B7
:107A5000E60297E6FF1F938626E3B69783C70700E3
:107A600005452380F5009947636EF7029D4763FD46
:107A7000E700E147630DF700828063850601850713
:107A8000E393C7FC0145C5B7238005008280B73763
:107A9000004003C7370083C7050093F70704D98F59
:107AA0002380F50082805D7152DC56DA5ED6716A01
:107AB00097EBFF1F938B0B158D6AA6C24EDE62D427
:107AC00086C6A2C4CAC05AD866D26AD06ECEC14990
:107AD0005E8C97E4FF1F9384E4DB130A0A20938AE9
:107AE0007ADC17E9FF1F0349E914B3872B0183C729
:107AF000070093F7F70FC9EFB787004003C7670088
:107B0000058BE310077C03C76700118BE30D077E2D
:107B100083C75700918B99E36F10200317E7FF1F6E
:107B20000347671185476304F7006F10400197E72B
:107B3000FF1FA380E7FC97E7FF1F238D07E097E770
:107B4000FF1F238B07EC97E7FF1F238907F897E7B1
:107B5000FF1F238607F897E7FF1FA38D07DE97E730
:107B6000FF1FA38B07EA97E7FF1FA38907F697E795
:107B7000FF1FA38607F697E7FF1FA38D07F697E77A
:107B8000FF1FA38A070AB787004011476F0070776D
:107B90009307190093F7F70F3D476364F70617E75C
:107BA000FF1F2309F70897E7FF1F9387A707CA97C7
:107BB00083C707001307100293F7F703638EE71ECE
:107BC0006366F70405446385871CE38C07620947F5
:107BD000638EE71013070002E384E74EB7E700E087
:107BE0003707400023A0E718010001006299230035
:107BF0000900FD1923A0E71093F9F90FE39309EEAB
:107C0000E5BD97E7FF1F2387070271BF1307300207
:107C10006388E70C63E8E71613074002638CE70A02
:107C200013070003E39CE7FA97E7FF1F938787FE9C
:107C3000CA9703C70700A1471377F70FE31BF71491
:107C400083C7640097E6FF1F238CF6E897E7FF1FC2
:107C500083C7B7C491C7FD5797E6FF1F2382F6E895
:107C600097E5FF1F83C515C397E7FF1FA38AB7E6F4
:107C700097E7FF1F83C707C213FB0708930600049B
:107C800093F70706639FD74C9307A009638DF516FA
:107C900063EAB7129307F0056386F54A9307500924
:107CA0006384F52A014497E7FF1F83C777E31547ED
:107CB000E392E736B7E700E03707400023A0E71874
:107CC00001000100B786004023808602130680FC75
:107CD0006F00500EFD5717E7FF1F2302F7E0FDBDB1
:107CE000FD5717E7FF1F230BF7DECDBD17A50100DA
:107CF000130585B997700100E780806097E7FF1F43
:107D0000938747F1CA9703C40700014B97ECFF1F05
:107D1000938CCCD01374F40F17AD0100130D4DB735
:107D200063478B04294597700100E780604A8547C7
:107D300017E7FF1FA302F7CE17E7FF1F230F87CC1C
:107D400017E7FF1F2308F7DA37E700E0B706400020
:107D50002320D71801000100378600408347A60280
:107D600093F7370F2305F6022320D71085BDB3877D
:107D70006C0183C507006A85050B97700100E780D9
:107D8000404079BF854717E7FF1F2307F7C8B9B5FC
:107D900017E7FF1F130707E84A970347070097E60F
:107DA000FF1FA389F6BA97E6FF1F2386E6BA17E7F7
:107DB000FF1F2301F7D41DB5854717E7FF1F230BCE
:107DC000F7B829BD9307400A6389F5349307200B60
:107DD0006384F5369307100AE396F5EC8387240055
:107DE0000144E3D207EC97E7FF1F83C7D7AA93F6B6
:107DF0003700638A061A0546638AC62209466395D8
:107E0000C61A1D4755A217E5FF1F0345C5A8C94758
:107E100097ECFF1F83CC3CA897E5FF1F83C5C5A740
:107E200017E4FF1F034454A76315F510CD47639271
:107E3000FC1093077008639CF5021307300FB71707
:107E40000E006308E4001307900DB7B70400631435
:107E5000E40817E7FF1F232BF7C8BE8517A501000D
:107E6000130585A397700100E780A03125BD930716
:107E70008008639DF500B307804013F4F70FB777D0
:107E80004600938787CDB3D78702E1B79307900861
:107E9000639AF500B307804013F4F70F9167938757
:107EA000C766D5B79307A008639BF500B30780406A
:107EB00013F4F70FB7173D0093870790E9B79307BF
:107EC000B008639AF500B307804013F4F70F916789
:107ED000938797D04DBF93F5F5078D47639BF500CA
:107EE000B307804013F4F70FB7975B00938707D869
:107EF00059BF8947639BF500B307804013F4F70F20
:107F0000B7770B009387071BBDBF8547639AF500C2
:107F1000B307804013F4F70FDD67938767E3A5B7D6
:107F2000D28785F9B307804093F7F70FB3D7FA02EA
:107F30000DB797000000E780409FA28566859700F7
:107F40000000E780809EB9BB9305610017E5FF1F25
:107F50000345659417E4FF1F0344F4939700000062
:107F6000E78040AD93057100228597000000E7800F
:107F700060AC3C0017E7FF1F2324F7C8834761006C
:107F80002304F10083477100A304F100894717E738
:107F9000FF1F2307F7B48357810017E7FF1F231B39
:107FA000F78E094409B3154793F64700B336D0005E
:107FB00093F78703850685C32146638BC706614611
:107FC000638AC706130680026388C7061306800308
:107FD0006393C700914717E6FF1F230BD6B097E6C0
:107FE000FF1FA387F6B097E7FF1F2384E7B017E7CB
:107FF000FF1F0347678A9376070497E7FF1F83C72E
:10800000B7898DEE1377770C93067008630CD7024F
:108010001377F7078D466312D70CB307F040B79577
:108020005B0093F7F70F938505D849A81947ADBFB3
:10803000854755B7894745B78D4771BF9306700887
:108040006311D7021307300FB7150E006389E702DB
:108050001307900DB7B504006383E7021307700898
:1080600045BF9306800C6311D702B307F040B77584
:10807000460013F7F70F938785CDB3D5E70297E74F
:10808000FF1F23A5B7A6D9BB9306900C631CD7008E
:10809000B307F04093F5F70F91679387C766B3D5A1
:1080A000B702F1BF9306A00C631DD700B307F040E1
:1080B000B7153D0093F7F70F93850590B3D5F502FB
:1080C0007DBF9306B00CE315D7F4B307F04093F5EA
:1080D000F70F9167938797D0D9B78946631BD7006D
:1080E000B307F040B7750B0093F7F70F9385051BA7
:1080F000F1B78546631AD700B307F040DD6593F703
:10810000F70F938565E35DBFD28535FBB305F0407E
:1081100093F5F50FB3D5BA029DB783C72400C18B81
:1081200099C7854717E7FF1F230FF79AA5BE97E763
:10813000FF1F238A079ABDB6854717E7FF1FA30ACB
:10814000F79A8DB63C0017E7FF1F232BF7AA0947C4
:10815000930700032314F10097E6FF1F2382E6989C
:108160002DBD63940756A94763E5B74217970100F1
:108170001307C75A8A05BA959C41BA97828717D4C4
:10818000FF1F03445471894C6306940D63E68C060B
:1081900085476303F4089307F00F17E7FF1F0347B2
:1081A000279463F6E70017E7FF1F230BF79297EC7E
:1081B000FF1F83CCEC929307000413F4FC0F63F4CD
:1081C00097011304000497E7FF1F938767A303AD8C
:1081D000070022862685EA85B38C8C40229D977005
:1081E0000100E780A0EE97E7FF1F238B978F97E7AB
:1081F000FF1F23A7A7A145BC8D47630CF40A99472D
:10820000E31BF4F8979701009387C75717E7FF1F01
:108210002328F79EA94751B717E7FF1F0347A7A1D8
:1082200097E7FF1F9387C78D494697950100938570
:10823000655E63068700979501009385A5593E8585
:1082400097700100E78080E817E7FF1F232AA79AAD
:10825000C947A1B797E6FF1F83C6E69D054797E785
:10826000FF1F9387E7896394E6023E851306700239
:10827000979501009385855797700100E78000E589
:1082800017E7FF1F232EA7969307700239B73E8585
:1082900013063004979501009385854F9770010070
:1082A000E780C0E217E7FF1F232CA7949307300451
:1082B000EDB597D5FF1F83C5055E17950100130522
:1082C000E55E97700100E780C0EB054D97EDFF1F5D
:1082D00083CD6D9697D5FF1F83C5E55B179501008C
:1082E0001305C55C6398AD0B97700100E78060E9EA
:1082F00097D7FF1F83C7275AB5CBE36EF4E81794CF
:10830000010013046455638CB70117940100130432
:10831000245563869701179401001304E4552285C0
:1083200097700100E78000FF1375F50F93071500A4
:10833000860717D7FF1F2305F77C8D4717D7FF1F29
:10834000A300F77C97D7FF1F9387877B0147BE86E3
:108350001376F70F89076365A60297E7FF1F23A12E
:10836000D78A97D7FF1F83C7A77905BD97970100C5
:108370009387874717E7FF1F2324F788914731BD6D
:108380003306E40003460600A380070005072380A8
:10839000C7007DBF97700100E780A0DE97D7FF1F61
:1083A00083C7674FE1D7E368F4DE17940100130435
:1083B000A447638CA70117940100130464476386E4
:1083C0009701179401001304244822859770010037
:1083D000E78040F41375F50F93071500860717D74C
:1083E000FF1F230FF7708D4717D7FF1FA30AF770E2
:1083F00097D7FF1F9387C7700147BE861376F70F85
:108400008907E37CA6F43306E40003460600A38054
:10841000070005072380C700D5B797D5FF1F83C581
:108420008547179501001305254997700100E780DE
:1084300040D597D7FF1F83C7776C93E7470017D7BF
:10844000FF1FA30DF76A83C7240017D7FF1FA305DB
:10845000F76A89B817950100130545479770010021
:10846000E78000EA97D7FF1F9387076983C7070054
:1084700017D7FF1F2300F74217D4FF1F034444669A
:10848000333480000DB017950100130565459770D2
:108490000100E780E0E697D7FF1F83C7376693E7C1
:1084A000070117D7FF1FA30BF76483C7240017D753
:1084B000FF1F2303F7646FF0EFFE1795010013050C
:1084C000654397700100E780A0E303C704007D8B3C
:1084D00051EFB787004003C767021377C70B1367D5
:1084E00027002383E70203C7A7021377C70B13678D
:1084F00027002385E70203C7E7021377C70B13673B
:1085000027002387E70203C727031377C70B1367E7
:1085100027002389E702854717D7FF1F230CF7425F
:1085200017D7FF1F230AF74E17D7FF1F2308F75A45
:1085300017D7FF1F2305F75A97D7FF1FA38C0740B4
:1085400097D7FF1FA38A074C97D7FF1FA388075809
:1085500097D7FF1FA385075897D7FF1FA38C0758EE
:1085600097D7FF1FA389076C6FF0CFF3894763127A
:10857000F70297D7FF1F83C727329146638CD7082E
:1085800063E0F604638EE70C6369F70A05476380CE
:10859000E70EFD5717D7FF1FA304F7543707400016
:1085A000B7E700E023A0E71801000100B78600400C
:1085B0001306F0FC2381C60223A0E7106FF00FE240
:1085C000130720086382E7086362F70213071008A5
:1085D000E391E7FC378700408347670293F7C70BB7
:1085E00093E727002303F7026FF0CFEB1307300860
:1085F0006389E70213074008E39DE7F837870040E7
:108600008347270393F7C70B93E727002309F70254
:108610006FF04FE9378700408347270393F7370709
:10862000F5B7378700408347E70293F7C70B93E717
:1086300027002307F7026FF0EFE6378700408347F4
:10864000E70293F73707F5B7378700408347A7025C
:1086500093F7C70B93E727002305F7026FF08FE42A
:10866000378700408347A70293F73707F5B7378767
:1086700000408347670293F73707ADB717950100AE
:108680001305452897700100E78080C797D7FF1F23
:1086900023820720D5B3179501001305A5279770EE
:1086A0000100E780E0C597D7FF1F2395071E97D7E6
:1086B000FF1F9387E74203C40700894763F38700DE
:1086C00009441374F40F6FF00FDE13070002E392F6
:1086D000E7EC631B0B0A638FF500930720026383AB
:1086E000F508179501001305652697700100E780CE
:1086F00040A945B517950100130585229770010023
:10870000E78000C00144179D0100130DAD22A14C6C
:10871000B387840083C507006A850504977001004C
:10872000E78020A6E31694FF178501001305456B2B
:1087300097700100E780C0BC17D4FF1F0344C41525
:1087400001E897D7FF1F23890712014B6FF0AFD5C0
:108750008947E310F4E4854717D7FF1F230EF7106E
:108760006FF04FD417D6FF1F0346F61297D5FF1FA1
:1087700083C56512179501001305451C977001000C
:10878000E78020A06FF00FD26380F50693071002F8
:10879000E399F5F497D5FF1F83C5051017950100E0
:1087A0001305C51B97700100E780A09D97D7FF1F99
:1087B00023A8974497D7FF1F93874733944383D7C2
:1087C000470017D7FF1F0347C73217D6FF1F2323C2
:1087D000D60C1D4497D6FF1F2390F60C97D7FF1F8A
:1087E000238DE70A6FF02FCC97D5FF1F83C5C50AED
:1087F000179501001305051897700100E780609830
:1088000097D7FF1F238A070697D7FF1F23940708D0
:108810006FF02FF92547638FE7C8994637870040E7
:108820006394D70223008702B7E700E0B706400051
:1088300023A0D71801000100130600FC2301C70282
:1088400023A0D7106FF08FB99306100A639FD7004B
:1088500023008702B7E700E0B706400023A0D7183F
:1088600001000100130680FCD1BF9306A009E3813B
:10887000D7FE9306400AE38DD7FC93062002639D42
:10888000D700B7E700E0B706400023A0D7180100E3
:10889000010023008702F9B78546E384D7FE9307DA
:1088A0000008E300FBFEB7E700E0B706400023A0A6
:1088B000D71801000100130620FC23008702BDBF6A
:1088C00017D7FF1F0347D7216302F71E63E7E702AD
:1088D00095476300F7109947630AF704B78600408D
:1088E00023800602B7E700E03707400023A0E7181F
:1088F000010001001306A0FC75B99307F005630A97
:10890000F700930750096306F70093071002E31777
:10891000F7FCB7E700E03707400023A0E7180100A5
:108920000100B7860040130620FC69B117DBFF1F6A
:10893000034B0B1B930700045A8D63F46701130D5F
:10894000000497D7FF1F9387A72B83AC07001374EE
:10895000FD0F2286E685268597600100E780007777
:10896000B3078B40669417D7FF1F230BF71697D7D3
:10897000FF1F23A78728B7870040630C0B022380C3
:10898000A703B7E600E03706400023A0C6180100A1
:10899000010003C72702134707042381E70203C727
:1089A00027021377C70F2381E70223A0C6106FF0B9
:1089B000EFA22380070237E700E0B706400023203C
:1089C000D71801000100130620FC2381C7026FF0B5
:1089D000AFB9378700408347370097D6FF1F83C65C
:1089E000B61193F70708D58FA301F700B70640002B
:1089F000B7E700E023A0D718010001001306A0FC90
:108A000035BD97D7FF1F9387E720CA9783C7070015
:108A100093F7F70FC1CF97D7FF1F83C7C721D9E7B8
:108A200017D7FF1F0347D70B930700026310F70800
:108A300083AD040017DDFF1F034D0DE697DCFF1F1C
:108A400083CC9CE517DBFF1F034B2BE5E6876A878A
:108A5000DA866E8697D5FF1F83C505E2179501005C
:108A60001305C5F297600100E780A07197D7FF1F3B
:108A700023AEB70797D7FF1F238CA70797D7FF1FF2
:108A8000A388970797D7FF1F2385670797D7FF1FEF
:108A9000A38387DEB7E700E03707400023A0E7188D
:108AA00001000100B78600406FF04FA2B7E700E079
:108AB0003707400023A0E71801000100B7860040F7
:108AC00015BD97D6FF1F83C606170547639CE604AE
:108AD00029472381E70209472383E7022385E70229
:108AE00097D7FF1FA388070097D7FF1FA3850714F9
:108AF000B7870040A381070017D7FF1FA30E07FE0B
:108B000005472383E700B640264496440649F259B8
:108B1000625AD25A425BB25B225C925C025DF24DB9
:108B20006161828029472381E70209472383E702A5
:108B30002385E7022387E7022389E70255B717D782
:108B4000FF1FA30AF7D26FE01FFF854717D7FF1F4C
:108B50002302F7E017D7FF1F2300F7EC17D7FF1FFB
:108B6000230EF7F617D7FF1F230BF7F66FE0BFFEB4
:108B7000854717D7FF1F230FF7DC17D7FF1F230DDC
:108B8000F7E817D7FF1F230BF7F417D7FF1F2308AA
:108B9000F7F417D7FF1FA30F07DA17D7FF1FA30D8F
:108BA00007E617D7FF1FA30B07F297D7FF1FA3886E
:108BB00007F28280411106C697000000E78080FB23
:108BC000B787004023800700130740FC2386E70097
:108BD0001307C004A386E70017D7FF1F130787CB2F
:108BE0002398E70017D7FF1F1307C7CE239AE70084
:108BF00017D7FF1F130747DA239CE70017D7FF1F7C
:108C00001307C7E5239EE70029472381E7020947A9
:108C10002383E7022385E7022387E7022389E7020C
:108C2000A3810700930600F8A380D7009306900263
:108C30002380D700FD562383D7002381E7009306C6
:108C4000000537E700E0230BD740B706400023209C
:108C5000D71003C7170013671700A380E700B240BF
:108C600097D7FF1F239A07E841018280411106C66A
:108C700097000000E78000F0B787004023800700DE
:108C8000130700FC2386E7003147A386E70017D7C8
:108C9000FF1F130727C02398E70017D7FF1F1307ED
:108CA00067C3239AE70017D7FF1F1307E7CE239C5C
:108CB000E70029472381E70209472383E702238549
:108CC000E702A3810700930600F8A380D70093066C
:108CD00090022380D700FD562383D7002381E7002D
:108CE0009306000537E700E0230BD740B7064000A6
:108CF0002320D71003C7170013671700A380E700CE
:108D0000B24097D7FF1F239907DE41018280F167A8
:108D10009387072017D7FF1F232AF7DC854717D72C
:108D2000FF1F2317F7DCA14717D7FF1F2303F7DC2B
:108D300097D7FF1FA38F07DA97D7FF1F238C07DA78
:108D400097D7FF1F238A07B297D7FF1FA38507B2C4
:108D5000814717D5FF1F130565B2FD5517D6FF1FB5
:108D6000130686B22947B306F5002380B600B30682
:108D7000F600238006008507E397E7FE97D7FF1FDD
:108D8000A38107D697D7FF1FA38F07D497D7FF1FBD
:108D9000238A07D497D7FF1F238507D497D7FF1FB0
:108DA000238407D497D7FF1FA38E07D297D7FF1F1F
:108DB000238B07D2814717D6FF1F1306A6E441472E
:108DC000B306F600238006008507E39BE7FE82805A
:108DD00017D7FF1F034727E685476316F7001703DA
:108DE00000006700E3E8170300006700E3DC4111BF
:108DF00022C406C617D7FF1F0347E7E385472E8621
:108E000013F4F50FAA856317F70417D5FF1F130591
:108E1000A5BC97600100E780602B97D7FF1F238DCB
:108E200007BEB787004023848702B7E600E0370615
:108E3000400023A0C6180100010003C7A702137752
:108E4000C70F2385E702B240224423A0C610014584
:108E50004101828017D5FF1F1305C5AB9760010044
:108E6000E780C02697D7FF1F238607AEB78700404D
:108E700023828702B7E600E03706400023A0C61829
:108E80000100010003C767021377C70F2383E702BE
:108E90005DBF411106C697000000E78080E7B24041
:108EA0004101170300006700E3F2411106C697F085
:108EB000FFFFE78080BF97D7FF1F83C7B7A9A1CB6C
:108EC00097D5FF1F83C525A989C917D5FF1F13058E
:108ED000A5A897E0FFFFE780605097D7FF1FA38BFF
:108EE00007A697D7FF1F238707C037E700E0B7061D
:108EF00040002320D7180100010037860040834737
:108F0000660293F7370F2303F6022320D710B240EF
:108F10004101828041C9D9C597D7FF1F83C7C7BD0B
:108F2000D1C3011122CC4AC84EC656C25AC006CE81
:108F300026CA52C42E89AA890144930A0004371B09
:108F4000030063772403B3078940C207C183BE844B
:108F500063F4FA0093040004C204C180130A1BD412
:108F600097D7FF1F83C7079F9DE37D1A631C0A00E5
:108F7000F2406244D2444249B249224A924A024BE8
:108F80000561828097F0FFFFE78020B2D1BF338573
:108F900089002694A685420497000000E78060E5DA
:108FA000418045B7828097D7FF1F938727DB184200
:108FB0009C4383D645000345070083C5C70003567D
:108FC00046006396A50083D5E700638DD5020111A5
:108FD00006CE2386A7002397D700B705CF00DC4B2A
:108FE0009385757D05077D162EC2230001003AC4C6
:108FF0002316C1002317D10099C30A858297F24036
:10900000056182808280411122C417A4FF1F1304CE
:10901000243F5C4C06C691CBC84B01C9B7E704009E
:10902000BC5782975C4C23AA0700B24022444101FE
:109030008280DC4DDC4B81CFB7E70400904503A371
:109040008705914517D5FF1F034585D1028382808F
:10905000B7E7040003A30705A14517D5FF1F034584
:1090600025D002836D713C083EC6B707E500232278
:1090700091103EC8AA843C083285232611103ECAAE
:1090800023248110232021112E8997300000E780AE
:10909000605A2A84979501009385C592177501003F
:1090A0001305856E97600100E780A00DA2851795D6
:1090B00001001305E59D97600100E780800C2945BC
:1090C00097600100E780C010B705CB009385757DE0
:1090D000680097100000E780E05FA2856800973085
:1090E0000000E7808047014781467000CA852685D9
:1090F00097200000E780608305CD2A8497950100C2
:109100009385458C1775010013050568976001006C
:10911000E7802007A2851795010013052598976021
:109120000100E7800006294597600100E780400ABA
:109130008320C110032481108324411003290110CE
:109140005161828097D7FF1F938747C118429C4384
:10915000797122D406D60348070083C807012A8400
:1091600083D64500035546006396080183D827013E
:10917000638DD8022388070105072399D700370894
:10918000CC00DC4B1308787D3ACC1307F5FF42CABC
:1091900023080100231EE100231FD10099C70808FE
:1091A00032C62EC482973246A2452285970000001F
:1091B000E78080EBB250225445618280797131465C
:1091C000977501009385054D280006D6976001002C
:1091D000E780C0EF97A7FF1F83D78722231B0100DB
:1091E000231C0100231D0100231E0100231F010079
:1091F00099E3C167FD17231AF10097A7FF1F83D7D3
:10920000472091EB97D7FF1F938747B59C439C431B
:10921000DC4783D7070097A6FF1F9386661E231B94
:10922000F100D84E83D74600231CF1005C4B91CB54
:1092300097A7FF1F83C7371D81EB97000000E780CA
:10924000C0DCB25045618280FD1717A6FF1FA30C3A
:10925000F61A0356070183C706014C472800230F5F
:10926000F10097300000E780602C97D7FF1F9387AD
:10927000E7AE9C430147978601009386267E88438C
:1092800030004C0897100000E780206A5DD975B760
:1092900099C9B7E7040003A30705A14517D5FF1F28
:1092A000034505AC028382805C4EDC4BB9CFB1CD67
:1092B000411122C4177501001305054D2E849785B1
:1092C00001009385657506C697600100E78060EB35
:1092D000A285178501001305657697600100E78078
:1092E00040EA294597600100E78080EEB7E7040077
:1092F0002244B24003A3870517D5FF1F034545A6A7
:10930000130640069145410102838280411122C427
:1093100017A4FF1F1304840C1C4C06C689C7DC432A
:1093200099C34C488297584CB7E70400BC57484B48
:1093300082975C4CB240224423AA070041018280FC
:1093400017A7FF1F1307870B834707009306F00B30
:10935000850793F7F70F63E9F60097A6FF1F238FA2
:10936000F608034507008280930700F8FDB783578E
:10937000450099E37D558280011122CC17A4FF1F7F
:10938000130404085C4C4AC84EC6DC4B52C406CEDB
:1093900026CA56C2B2892E8A2A898DC7B7E7040029
:1093A000FC5F829797D7FF1F938747999C431307CA
:1093B000301FB307F54071556375F706970000003D
:1093C000E780A0C49307D00D7D5563EC3705B7E463
:1093D000040093878900B858832AC40113950701B4
:1093E0004181029723AAAA00484C584921E7978552
:1093F000010093856560177501001305E5389760D6
:109400000100E78000D8178501001305E56B976020
:109410000100E78000D7294597600100E78040DB25
:109420005D55F2406244D2444249B249224A924ACE
:109430000561828013874900B705CF002319E50035
:109440009385757D310597100000E780A028484C72
:1094500083456900310597300000E7800010484CD3
:109460004E86D285310597300000E780200C71468A
:10947000CA8517A5FF1F1305A5F897600100E780AF
:10948000E0C4FC5C82970326C90097D7FF1F23A77F
:10949000A78A11CABC4C854517D5FF1F0345458CCB
:1094A00082970145BDBF97000000E78060D1D5BF1E
:1094B000411106C622C426C217D4FF1F1304448AD2
:1094C00097000000E78060B4B7E40400FC4C03455B
:1094D00004008545829703450400224403A3C40584
:1094E000B2409244A14541010283411126C297D462
:1094F000FF1F9384A4869C4006C622C44AC0D5C3DD
:10950000DC43C5C35CC12300B5002A8497850100F4
:109510009385C5491775010013050527976001005C
:10952000E78020C6294597600100E78060CA9C401B
:1095300023A4070023A2070097A7FF1F938707EA2A
:10954000DC4FDC4B91C7295597000000E78040DCD9
:1095500097A7FF1F9387C7EADC4FDC4B89C79700AB
:109560000000E78020F537E904008327C905894515
:1095700017C5FF1F0345C57E82978327C9059145FF
:1095800017C5FF1F0345C57D82979C4003A3470174
:109590006309030022852244B240924402494101FA
:1095A0000283B24022449244024941018280011167
:1095B000328506CE22CC26CA2E8497300000E78062
:1095C0006007AA849785010093858541177501007E
:1095D0001305851B97600100E780A0BA030784008C
:1095E0000356640083554400A686178501001305C1
:1095F000654797600100E780C0B829459760010082
:10960000E78000BD97A7FF1F83C7A7DD639D970075
:10961000014597000000E780A0CF81450A859700AB
:109620000000E780C0ECF2406244D24405618280D1
:109630006D7123248110232611102322911093F79A
:1096400045002E84638707143C083EC0B707E50039
:109650003EC23C083EC42317010023180100231911
:109660000100231A0100231B010097A7FF1F83D7C6
:10967000E7D699E3C167FD172316F10097A7FF1FEF
:1096800083D7E7D591EB97C7FF1F9387276D9C433F
:109690009C43DC4783D7070017A7FF1F130707D496
:1096A0002317F100544F835747002318F100DC4A79
:1096B000A1E7978501009385E5361775010013052D
:1096C000A50C97600100E780C0AB1785010013056A
:1096D000254697600100E780C0AA294597600100F0
:1096E000E78000AF134544008320C110032481109C
:1096F000832441105161828097A7FF1F83C777CED3
:109700002555D9C3FD1717A6FF1FA30CF6CC03D60A
:10971000060183470701CC460A85230BF1009730E9
:109720000000E780A0E097C7FF1F938727639C4353
:1097300017A7FF1F130787CA978601009386862FF6
:1097400088430A866C0097100000E780001EAA84F8
:1097500051D9978501009385E52C177501001305F4
:10976000A50297600100E780C0A1A68517850100CA
:109770001305C53C97600100E780A0A029459760CC
:109780000100E780E0A4268597000000E78040B84C
:1097900091BF93F725009DC7B7E70400BC4741463A
:1097A000814528088297255597000000E78040B63C
:1097B00028089305F00F97000000E78040D3134579
:1097C00024001DB793F7150081CB97000000E780B8
:1097D000209F1345140009BF93F78500014589D7E1
:1097E00017A7FF1F034737C297A7FF1F938747C1DC
:1097F0000DC3D84F584B11CF37E70400384F90476F
:10980000854517C5FF1F0345A555029713458400DD
:10981000E1BD97F0FFFFE780407FCDBF5C4D411178
:1098200006C688C317C7FF1F232AF752B7E70400ED
:1098300083A70708170500001305C5DF8297B2400C
:1098400097C7FF1F238EA750014541018280011158
:109850003335A000A307A100B7E7040083A747178B
:1098600006CE1306F1008545130550308297F2406D
:10987000056182808280411122C406C697B7FF1F0E
:1098800083C79799054489EF97C7FF1F83C707D9F7
:10989000014499E717B4FF1F0344049813441400CC
:1098A000228597000000E780C0FA178501001305A4
:1098B000A52F09E417850100130505302244B240A5
:1098C0004101176301006700C38B797122D4A30F94
:1098D000010037E404008327841726D24AD006D635
:1098E000AA842E89130550309305F10132C6829760
:1098F00032468347F10193150601C18185CB0145AD
:109900002EC697000000E780C0F483274417B245B5
:109910004A8626858297054597000000E78060F318
:10992000B2502254925402594561828083274417D1
:109930004A8626858297EDB741119397050122C487
:1099400006C626C2C1872E8463D40702B7E404008A
:10995000FC5417A5FF1F0345A5AD829719C1BC5440
:1099600082972165218DB240224492444101828038
:1099700093F715008DC7B7E7040083A7471A17A60A
:10998000FF1F1306E6A997C5FF1F9385253E17A560
:10999000FF1F0345E5A9829713451400E9B793F724
:1099A00025000145E9D397C7FF1F83C7A73D85E77A
:1099B000B7E7040003A8871A1307401F97A7FF1FE4
:1099C00083C707A7814613064006994517C5FF1FA1
:1099D0000355C53A02981345240071B797C7FF1F76
:1099E00083D7C7396398A70217C7FF1F2319B73852
:1099F00017C7FF1F2316C73817C7FF1F2313D738F2
:109A00002E86178501001305A521BE851753010079
:109A100067002377178501001305052217630100EE
:109A20006700038E0357450097C7FF1F83D707358D
:109A30006318F702C167F91717C7FF1F2320F73410
:109A400097C7FF1F23AE073297C7FF1F2386073232
:109A500097C7FF1F23880732170300006700E3E161
:109A6000178501001305451D176301006700438931
:109A70007D15954763E2A71C17870100130747115F
:109A80000A053A951C41011122CC06CEBA972E84C4
:109A90008287178501001305A51A97600100E780EA
:109AA0002086A1A203C7250099476311F7022E85DE
:109AB00097000000E78040F78345640017850100A8
:109AC0001305051997500100E780A06B97A7FF1FAA
:109AD0002384077417850100130545197DBF03C74B
:109AE000250095476319F702C16717C7FF1F035782
:109AF000E728F91703D5A5006309F702B7E70400C3
:109B000083A7C7178297178501001305251797505C
:109B10000100E780E07E854717A7FF1F230EF76E41
:109B200017850100130505188DBF97C7FF1F2397E1
:109B3000A72483D7E50097C6FF1F2392F62483D777
:109B4000050197C6FF1F239DF62283D7250197C6DF
:109B5000FF1F2398F62297C7FF1F238F0720631B41
:109B6000E502B7E70400BC4F096613060690894575
:109B700017A5FF1F0345C58B82970356E400835545
:109B8000A400178501001305A51097500100E78078
:109B9000405F51B79307700F2316F100B7E7040039
:109BA00083A7870D17A6FF1F034686886C00829740
:109BB0004DF9854717C7FF1F2300F71C5DB71785B1
:109BC00001001305E50ED1BD83C5250091476392C1
:109BD000F502178501001305250F97500100E78056
:109BE000207297000000E78040C9F240624405619E
:109BF000828099476392F502228597000000E780F2
:109C0000A0E28345640017850100130565049750A1
:109C10000100E7800057D1BF9547639AF50083475D
:109C20001400E1F3178501001305450CBDB5178538
:109C300001001305250CE1BF82803757315F97A7DC
:109C4000FF1F93872780130777D598C39356C500C6
:109C500017870100130787F9BA9683C50600935644
:109C60008500BD8ABA9603C6060093564500BD8A94
:109C70003D89BA962A9783C60600034707002384C6
:109C800007002383D700A383E7002382B700A382C2
:109C9000C7009797FF1F9387E77B2383B700A383B2
:109CA000C7002384D700A384E7008280411106C641
:109CB00097000000E780A0F8B7E7040083A78714A7
:109CC0001796FF1F13060678D54501458297B240C7
:109CD0004D469795FF1F9385E57713057030410139
:109CE000170300006700A3BE61712324811A37E4C3
:109CF0000400832704082326111A2322911A232003
:109D0000211B232E311917050000130525C3829747
:109D10001799FF1F1309C971994785442300A900AA
:109D2000231CF10097850100938545EB93074006BE
:109D300017750100130545A5231CF10823089100A0
:109D400097C9FF1F9389E99D97500100E780604301
:109D500083D5090017850100130545E797500100D9
:109D6000E7802042294597500100E780604603D5EF
:109D7000090097000000E78080EC83274417100853
:109D80008545130550308297832744171796FF1F88
:109D90001306466CCD451305703082978327441710
:109DA0001796FF1F13060669B545130560308297A5
:109DB000832744173008894513051031829783277C
:109DC00044173009894513052031829783274415AC
:109DD0009305000A0D458297832744159305000AD1
:109DE00011458297A30591002306910002CD230817
:109DF0000100230C010083278416300991451305C7
:109E000070408297832784161306B1008545130599
:109E10000040829783278416700085451305104003
:109E20008297832784163008854513052040829742
:109E30008327841610088545130550408297832791
:109E400004157D558297832744137D5582977D5550
:109E500097A0FFFFE78060838327440C8297979049
:109E6000FFFFE780C05E832784141796FF1F130649
:109E7000665DD5450145829789471306700F814578
:109E800028092306F1009780FFFFE78040288D47CF
:109E90001306000881452808230CF1089780FFFF6E
:109EA000E780E0269147230CF10097670100938734
:109EB000277F984383C747003AC8230AF10097C019
:109EC000FFFFE780A06E70008545054597A0FFFF66
:109ED000E780C08230099305700F094597A0FFFF06
:109EE000E780C0813008930500080D4597A0FFFF6B
:109EF000E780C0801008954511459790FFFFE780E7
:109F0000E07FC16717C7FF1F130747E7F9171CC397
:109F1000232207001795FF1F130545519790FFFF58
:109F2000E780A07C8327C41D17C5FF1F130585E3A9
:109F300082973C4803450900854582978320C11AD2
:109F40000324811A8324411A0329011A8329C11980
:109F50005D618280C16717C8FF1F035828E2F917A7
:109F60006301F8083DCDB5CD011126CAB7E4040060
:109F700083A7841222CC2E862315B10006CE2A8414
:109F800001478146ED45428582972AC611ED178526
:109F900001001305E5C697500100E7806036F240E6
:109FA0006244D24405618280FC440356A100A2852C
:109FB00082972C0017C5FF1F035545DC9790FFFFC4
:109FC000E780607F69DD178501001305A5C4975000
:109FD0000100E780E03283A7C412ED452800829794
:109FE0007DBF82800DC585471797FF1FA309F744E2
:109FF0009797FF1F2386074435469795FF1F938544
:10A00000654313056030170300006700438C979782
:10A01000FF1FA3860742E9BF97C7FF1F83C787D6E5
:10A02000A9EFC16717C7FF1F035747D5F917630685
:10A03000F7044111854722C417C7FF1F2304F7D433
:10A0400037E404007C4C06C689451795FF1F03457D
:10A05000253E82970323841A2244B2409797FF1F1C
:10A0600083C7073D17C5FF1F035545D11307401F81
:10A070008146314699454101028382806D712324D6
:10A0800081102326111023229110328401CD89479B
:10A09000630AF5028320C110032481108324411038
:10A0A0005161828017850100130585C5AE849750E4
:10A0B0000100E780E024A285268597B0FFFFE780B6
:10A0C00080C2C9BFB7E70400FC4728008297178504
:10A0D00001001305A5C397500100E7806022834764
:10A0E000810039C41307000B6380E7021387A705BB
:10A0F0001377F70F8D4663EDE602A285280097C01F
:10A10000FFFFE78060CA79B78547E3F587F88345A5
:10A110009100177501001305259BB335B00097A773
:10A12000FF1F2383B7F897500100E78080059DB794
:10A1300003479100A207B966D98F1387E655638458
:10A14000E70C636DF7042D671307B755638FE708B6
:10A15000636AF70029671307A755638FE708A2858D
:10A160002800A1BF31671307C7556388E706356725
:10A170001307D755E395E7FE8947E3FD87F097007E
:10A180000000E780A0E99305E4FFC205C181130543
:10A19000A1009790FFFFE780A004EDBD3D67130687
:10A1A000F7556389C706636DF6009386E665E39805
:10A1B000D7FAA285280097C0FFFFE7800004D9BD29
:10A1C0009306F766638DD7041307F777E399E7F8EB
:10A1D00097C0FFFFE780202F75BD0146A2852800AC
:10A1E00097C0FFFFE780E0E775B5A285280097C01C
:10A1F000FFFFE78020F579BDA285280097C0FFFF0B
:10A20000E78080F441BDA285280097C0FFFFE7806A
:10A21000C0F549B597C0FFFFE7804007A5BD97C0CF
:10A22000FFFFE780E00CBDB5C16717C5FF1F0355F1
:10A23000E5B4F9176307F500B7E7040003A3C717F0
:10A240000283828017F3FFFF670023631783FFFFFA
:10A25000E70243E72A8408452E89B28919C900C15B
:10A26000971500009385A586610597300100E7806A
:10A27000600481447D5A97100000E780E03963C78D
:10A28000A404814497100000E780003A63C8A40446
:10A2900097C7FF1F938747AF9C43DC47B307F9403D
:10A2A00091872302F400638309048327C900B3075D
:10A2B000F4409587A302F4001C4C89C79C4799C3BE
:10A2C000228582971783FFFF670003E35C4413979F
:10A2D00014008504BA972390470171BF1C48139757
:10A2E00014008504BA972390070069BF832789006B
:10A2F0000547B307F4409587A302F4008357040091
:10A30000638EE7028DC309476384E7040D47E39535
:10A31000E7FA97870100938727F21CCC9787010003
:10A32000938787F211A897870100938767B81CCCA1
:10A33000978701009387C7B85CC8BDBF97870100A6
:10A34000938707A41CCC97870100938767A4EDB778
:10A3500097870100938707F31CCC978701009387A9
:10A3600067F3D9BF95E51783FFFFE70243D70046A0
:10A3700018448347940075839D8B6317F7009710EB
:10A380000000E78060B448C41783FFFF670063D70D
:10A3900082801783FFFFE702E3D213893500C1648F
:10A3A00042094111AA890144F11413590901054ACE
:10A3B0002EC697100000E7802026B2456348A4000F
:10A3C000014541011783FFFF670003D383A70900FD
:10A3D00013171400BA9783D707006388B7006394F4
:10A3E000970063742A010504E1B70545D9BF1783B7
:10A3F000FFFFE70243CCAA892E89328BB6843A8AC2
:10A40000BE8A97A00000E78000FE71C926859720CC
:10A410000000E780C00C8D4763E7A7007D551783D8
:10A42000FFFF6700C3CC83DB440097100000E78088
:10A43000A0242A8497100000E78040259307740029
:10A4400031443305850263CDA70297100000E780F1
:10A45000A02297100000E78020222A849710000095
:10A46000E780C0229307740031443305850263C33B
:10A47000A70497100000E78020209307450029A833
:10A4800097100000E7808020330585021307F0173E
:10A490009307C017E35FA7FA2D55E3C277F963046A
:10A4A0000B02D6865286A6854A8597200100E78052
:10A4B00000BDB5B797100000E780401D3305850249
:10A4C0009307C5FFD1BF832749001385C90083D5F2
:10A4D000270097000000E78000EC61F581B769551F
:10A4E0003DBF97C7FF1F2393A78A97C7FF1F938777
:10A4F000A789904381470C463307F5004207418303
:10A500006393B70082805446139847008507C2962C
:10A510002390E600D5B797C7FF1F9387E7869C4334
:10A5200003C58700828017C5FF1F035525868280DB
:10A530001783FFFFE702A3BAC1671387D7FF630B37
:10A54000E502636AA700F1176300F502014517836E
:10A55000FFFF670003BB1387E7FF6302E502FD17F8
:10A560001D8D13351500E5B797500000E780A02931
:10A570007D15C5BF97500000E78020FED5BF9750DE
:10A580000000E78040FCEDB71783FFFFE70223B52B
:10A590004111AA8401442EC697100000E780C0082C
:10A5A000B2456348A400014541011783FFFF6700DE
:10A5B00043B59C48131514003E9583570500E38569
:10A5C000B7FE0504C9BF03485500814693F7F60F4F
:10A5D00063E5070181473E85828058459397560081
:10A5E000BA9703D727006316B70003D70700E30421
:10A5F000C7FE8506E1BF8346450001479377F70F05
:10A6000063E4D700814711A81C45131657000507BE
:10A61000B29703D60700E313B6FE3E858280178308
:10A62000FFFFE70223AA93170501C18797BAFF1F0F
:10A63000938A8A75635BF00883A70A00C0479C472A
:10A6400003570400198D420541816368F5000144F8
:10A6500022851783FFFF670023AA12052A94CDBF26
:10A66000DC4713944900014A3E9483474400634108
:10A67000FA02014A834754006349FA028509C20974
:10A6800093D9090183A70A009847E3EBE9FCC1B716
:10A690001C4413195A00A6853E994A85970000006C
:10A6A000E780C0EE05E1050AC9B75C4413195A00FA
:10A6B000A6853E994A8597000000E78020ED19E1C4
:10A6C000050A4DBFE30C09FA61B7AA8481495DBF51
:10A6D0001783FFFFE702A3A01C452A8481E79307A5
:10A6E000C5001CC51C44231204001CC09307F00FB6
:10A6F00063EDB70093F5F50F228597200000E78002
:10A70000C0E51783FFFF6700C39F93940501C167EE
:10A71000C18063F9F500A685228597200000E780B7
:10A72000E0E8C5B7C18193F5F50F228597200000B9
:10A73000E780A0E2A685228597200000E780E0E37D
:10A74000C9B797B7FF1F93872764884382801C454A
:10A7500099C797B7FF1F23A9A762014582807D553E
:10A76000828097B7FF1F93872762984383474500EE
:10A77000484792073E9582801783FFFFE7022396A2
:10A78000617100451C183EC6B70780013EC81C1801
:10A790003ECA8357440002CE02D002CC231EF100F1
:10A7A000834784002A8902D22301F1023C083ED467
:10A7B00002D697000000E78000FB835705002316B0
:10A7C000F10297500000E78040C72307A1025C40D8
:10A7D00003556400F18313F717008347F102520514
:10A7E0005181F99BD98FA307F10297100100E780EF
:10A7F000607839CDAA840355050097A00000E78052
:10A8000060BF83D704002AD26800231CF10083D7DD
:10A810002400231DF1001C4803D647008C439720D9
:10A820000000E780A0D08347B400CA8617760100F5
:10A830001306864E8117A305F4006C00481097207C
:10A840000100E780C0835D611783FFFF6700638BB2
:10A850002155D5BF1C45B1CF03C5A7008946135765
:10A860006500630BD7028D46630ED70285466300F1
:10A87000D702130740063305E50203C7B700418B33
:10A8800015CB83C7B700BD8B3355F5408280137558
:10A89000F5031307803EC5B709671375F503130762
:10A8A0000771D1BF372709001375F5031307077C1C
:10A8B000D9B7014582801783FFFFE702438203A9CE
:10A8C0008500630C09048347B900AE8493F7070E33
:10A8D00085C303459900930520030D810505B30544
:10A8E000B5028844610597300100E780C0AC35A00F
:10A8F0002E8597000000E78020F62A8419CD970066
:10A900000000E780605C8325C900B307B54063FAA7
:10A9100087002E94B305A440E9F51773FFFF670085
:10A92000437E85457DBF1773FFFFE702437B2A8483
:10A9300003D50500011132C636C43AC22EC002CA80
:10A9400002CC02CE97A00000E780C0AA82452ACAA6
:10A9500022852ECC97000000E780E0E00357050039
:10A96000231EE10097500000E78020ADA24632464A
:10A970009247230FA10036874C08B28622850146F4
:10A9800097000000E780E0A605611773FFFF6700EE
:10A9900043771773FFFFE702837461711C183EC68B
:10A9A000B70780013EC81C183ECA3C0800453ED48B
:10A9B000AA8402CC02CE02D002D202D697000000B6
:10A9C000E78060DA8357050035592316F102975066
:10A9D0000000E78080A62307A10209C48357440032
:10A9E00081EB21594A855D611773FFFF6700637131
:10A9F000035564005205518197100100E78080578C
:10AA00002A8965D18347B40093F7070E99C71305C8
:10AA1000840197300100E780409C83574400231E47
:10AA2000F100834784002301F1025C4003550900D3
:10AA3000D98313F7070883471102231CA10093F75A
:10AA4000F707D98FA300F10283572900231DF100D6
:10AA50005C40F18313F717008347F102F99BD98F0C
:10AA6000A307F10297A00000E780C0982AD235D949
:10AA7000834794006800139757008347B400FD8B09
:10AA8000D98FA305F4001C4803D647008C439720B8
:10AA90000000E780A0A9A687177701001307C72742
:10AAA000740005464C10268597000000E7806094EE
:10AAB0002A890DD98347B400A685FD8BA305F40030
:10AAC00097000000E78060DF31BF1773FFFFE702E8
:10AAD0000361832485FE2A844111268597000000A6
:10AAE000E78080D7834734FF93F7070E8DCB2AC6C4
:10AAF000268597000000E78060C809CD834734FFB2
:10AB0000B245FD8BA309F4FE91C522859730010063
:10AB1000E780608A41011773FFFF6700835E7DD97C
:10AB20008327C4FF2685829775F5834734FF93F703
:10AB3000070E91C7228597300100E780008A032520
:10AB400084FE97000000E78000E5E9B71773FFFF78
:10AB5000E702E3559C4141112A8903C70700894751
:10AB60002E84935667006380F6040D466388C604FE
:10AB70009307F0076304F7022E8597200000E78013
:10AB800060ABAA848149C16B130C490097B7FF1FC2
:10AB90009387871F9C43984763E4E9044101177337
:10ABA000FFFF6700835403D745008547E3F8E7FEBE
:10ABB0002E8597200000E78040ADE1B703D7450020
:10ABC000E3FEE7FC2E8597200000E780A0A6AA847C
:10ABD000228597200000E78000A8C204C98C5DB7D9
:10ABE000DC470355A900139A49003E9A93170501C3
:10ABF000C187635DF00083570A006397A70263E78C
:10AC000074038327CA00034D5A002DA0A167216752
:10AC1000A98F1307F7EFE374F7FE63970900970016
:10AC20000000E780209161FD85098DB783278A00A8
:10AC3000034D4A00835DA90003576900216A138B05
:10AC4000C7003AC6814A33CA4D01631E5D0197B7FA
:10AC5000FF1F9387E7139C43E1DBA2866286814551
:10AC600026858297D1B7A1679387F7EF930C4BFFA7
:10AC700063F24703B2455A8597F0FFFFE780A07162
:10AC80000DC103278B00104709CE10436382C40215
:10AC90003107D5BFEE85668597000000E780008FFD
:10ACA00071F993861A0093FAF60F130B0B0271BF1A
:10ACB000835644005C43E3E9F6F622853AC69720C2
:10ACC0000000E7802081A1679387D7042A8A035D6B
:10ACD0004400324763E897008347D90093E707F8B9
:10ACE000A306F9001C4766852286E2858297C16724
:10ACF0000844FD17337AFA00529508C02312A401C4
:10AD000025B797B7FF1F938727089843814715C337
:10AD10001447814763FFD500939745004C47BE9584
:10AD200019C903C7550081476375E600DC4516065F
:10AD3000B2973E85828003C745008147E37BE6FEEC
:10AD400016069C45F5B71773FFFFE702A337AA89DC
:10AD50002E8A814497BAFF1F938A0A0383A70A00A9
:10AD6000984763E6E4001773FFFF6700E338DC47AA
:10AD70001394440001493E9413BB140083474400DC
:10AD8000634BF900014913BB140083475400634F20
:10AD9000F9008504E1B70844931759005287DA8611
:10ADA0000146A2853E9582990509C9BF484493177B
:10ADB00059005287DA860546A2853E958299050993
:10ADC000E9B71773FFFFE7028331814517F5FFFFEE
:10ADD0001305054897B7FF1F239A07FA970000004D
:10ADE000E780A0F61773FFFF6700A33197B7FF1F37
:10ADF000938787F99C4395C31773FFFFE702232EC0
:10AE0000814517F5FFFF1305A54497000000E78073
:10AE1000C0F31773FFFF6700C32E82801773FFFF15
:10AE2000E702432A37E404008327841241112315E3
:10AE3000E100AE893289368A3A8681460147ED457E
:10AE4000AA8482972AC621C90356A100D2859740B9
:10AE50000100E780A0278327C413CE85268582972B
:10AE6000058905C98327440D2314210101462C00BF
:10AE7000268582972A8401C9B7E7040083A7C712F1
:10AE8000ED4528008297228541011773FFFF670077
:10AE9000A3264944D5B76554FDB75C41FD175CC195
:10AEA00082801773FFFFE7028323B7E70400FC5F8C
:10AEB000829795473305F50281450D811773FFFF92
:10AEC000670023241773FFFFE7026321B7E704003D
:10AED000FC5F829795473305F5020D811773FFFFDD
:10AEE000670023221773FFFFE702631FB7E7040021
:10AEF00083A7870B0355050082971773FFFF670031
:10AF000043201773FFFFE702831D035505003287B7
:10AF1000AE861786FF1F0356065A97B5FF1F938507
:10AF200065E797000000E780A0EF1773FFFF670059
:10AF3000431D1773FFFFE702831AB7E7040083A7D7
:10AF4000C71782971773FFFF6700A31B1773FFFFD5
:10AF5000E702E318B7E7040083A7871397B5FF1F3D
:10AF6000938545E3829701451773FFFF67006319D7
:10AF70001773FFFFE702A316B7E7040083A7C71FF5
:10AF800081451785FF1F0355054F82971773FFFFF4
:10AF9000670023171773FFFFE7026314B7E7040086
:10AFA00083A7871397B5FF1F9385C5DF8297014558
:10AFB0001773FFFF6700E3141773FFFFE702231205
:10AFC000B7E7040083A7C71F81451785FF1F0355F7
:10AFD000855082971773FFFF6700A3121773FFFF57
:10AFE000E702E30F2E8597800000E780C0B29780CC
:10AFF0000000E780C0EF1773FFFF6700831017732F
:10B00000FFFFE702C30D97800000E780C0F91773C8
:10B01000FFFF6700030F5C49E1175CC95CC58357FC
:10B020002501A1072319F50083570501A10723185E
:10B03000F5008280F1473305F50297B7FF1F93872C
:10B0400067D89C433E9582808D476315F60803D7E9
:10B050004600854763F0E7081773FFFFE702230800
:10B06000368536842E8997100000E780A05C29C9B8
:10B070008357440093140501C18063E3970422853C
:10B0800097100000E780005BFD14231294009307E3
:10B09000A0026300F5029307B0026307F50293076D
:10B0A0009002631FF500228597000100E780A088C9
:10B0B00001A80146CA85228597A00000E78040B319
:10B0C0001773FFFF6700E303228597100000E780F6
:10B0D0006007FDB7828097B6FF1F9386E6CE9C423D
:10B0E000014599CF9843D44217B6FF1F232EE6CCD3
:10B0F0006396D70097B6FF1F23AAE6CC1385C7FE39
:10B1000082801773FFFFE70283FD97000000E7804E
:10B11000A04B714433058502914597900000E7806C
:10B1200000EC11E565551773FFFF670083FD97B7C6
:10B13000FF1F23A7A7C897000000E780E04833055A
:10B140008502914597900000E78060E961DD97B73F
:10B15000FF1F23A9A7C697000000E780E04697B726
:10B16000FF1F2399A7C497000000E780E04597B729
:10B17000FF1F2392A7C497770100938727BF17B7B4
:10B18000FF1F232DF7C297070000938707E917B722
:10B19000FF1F2323F7C2014579B71773FFFFE702AB
:10B1A00003F4AA8517B5FF1F1305C5C0971000004B
:10B1B000E780605F1773FFFF6700A3F41773FFFF5B
:10B1C000E702E3F197000000E78060FD97100000C0
:10B1D000E780E05E97B7FF1F938707BF9C4391CF3F
:10B1E0001387C7FE19CB83D5C7FF17B5FF1F1305FC
:10B1F00025BE97200100E780001C1773FFFF670042
:10B2000043F01773FFFFE70283ED97000000E7802C
:10B21000C0EC09CD834785002A8493F7070499EB96
:10B220000355E50097000000E78080F91773FFFFE2
:10B23000670023ED8347C5009304450117B9FF1F3D
:10B24000130989B885E3832709005CC997B7FF1FF5
:10B2500023AC97B683274900F1FB97B7FF1F23A7BD
:10B2600097B6E9B7FD172306F50061059780000042
:10B27000E780A0D98307840063CB07048347840059
:10B2800093E707F82304F400B7E704009C5F829774
:10B290004205A94741813375F5028347840093F73E
:10B2A00007FCC98F2304F4008347D4003E951C405B
:10B2B0002318A40089CF984319CB8347C40050407A
:10B2C000814585073305F5024205418102978327B1
:10B2D00009005CC897B7FF1F23A897AE83274900D2
:10B2E00089E797B7FF1F23A397AE8347C4009DDF6D
:10B2F0008355040117B5FF1F130585AD9720010085
:10B30000E780600B25B71773FFFFE70243DD97B7B0
:10B31000FF1F938727D19C4701448583858B85E355
:10B32000AE84B2853A8697100000E780204F2A84C9
:10B3300019C597100000E7806045829408CC2285EB
:10B340001773FFFF6700E3DB1773FFFFE70283D785
:10B3500041112E8932C6AA8997000000E780C031CA
:10B36000324713060502CA86970500009385C5CCAF
:10B3700017B5FF1F130505A497000000E780E0F84C
:10B380002A8425C99304C50097000000E780E041A6
:10B390001946AA85268597100000E7802019854563
:10B3A000268597100000E78000151775010013052A
:10B3B000A5994E9583450500268597100000E780E6
:10B3C000C0195C4831468145A1075CC85CC48357FD
:10B3D0002401E1172319F40083570401E11723180E
:10B3E000F4001C4C3E859770FFFFE78040D2A30419
:10B3F0002501228541011773FFFF6700E3CF177313
:10B40000FFFFE702C3CD4111AA842EC632C49710B4
:10B410000000E780003A004DB24522468347840091
:10B420000CC050C093F7F70393E707042304F4001C
:10B4300023180400268597100000E78020358347F5
:10B440009400A9462317A40013D737000507330734
:10B45000D7029D8B85072306F400A306E40083C76B
:10B460000401D8488507230FF7FE17B7FF1F1307FE
:10B47000A7955843232A04009307440129E317B7EB
:10B48000FF1F2325F79417B7FF1F232FF79217B439
:10B49000FF1F1304E493228597200100E780E0E377
:10B4A0001C44858B5D8D19E581452285972001001F
:10B4B000E78060F041011773FFFF670083C41CC37E
:10B4C00017B7FF1F2324F790D9B71773FFFFE702C1
:10B4D00003C197050000938565B7014597000000FB
:10B4E000E78000B001451773FFFF670083C1177342
:10B4F000FFFFE702C3BE97000000E78080B017732C
:10B50000FFFF670003C08347C500A5E31773FFFF74
:10B51000E702E3BC2A840355E50097000000E780BA
:10B5200000C821C18347840093F7F7FB2304F4008C
:10B530001C4091C7DC4381C74C400145829797006E
:10B540000000E78080B917B5FF1F130565889720B5
:10B550000100E78080E80355E40097000000E780E1
:10B5600020C61773FFFF6700C3B982801773FFFF00
:10B57000E702E3B697B7FF1F93870785970500009B
:10B58000938565C817B5FF1F1305858423A00700A1
:10B5900023A2070097200100E780C0D11773FFFFA7
:10B5A000670023B61C4D91CFDC4381CF1773FFFF9B
:10B5B000E702E3B28345070082971773FFFF670036
:10B5C00043B4828097B7FF1F9387C7829C4303C50C
:10B5D0000700828097B7FF1F9387C7819C4303C5ED
:10B5E0001700828097B7FF1F9387C7809C4303C5CE
:10B5F0002700828097A7FF1F9387C77F9C4303C5BF
:10B600004700828097A7FF1F9387C77E9C4303C58F
:10B610003700828097A7FF1F9387C77D9C4303C590
:10B620005700828097A7FF1F9387C77C9C4303C561
:10B630006700828097A7FF1F9387C77B9C4303C542
:10B640007700828097A7FF1F9387C77A9C4303C523
:10B650008700828097A7FF1F9387C7799C4303C504
:10B660009700828097A7FF1F9387C7789C4303C5E5
:10B67000A700828097A7FF1F9387C7779C4303C5C6
:10B68000B70011E11D45828097A7FF1F938787763A
:10B690009C4303C5C700828097A7FF1F93878775C8
:10B6A0009C4303C5D700828097A7FF1F93878774A9
:10B6B0009C4303C5E700828097A7FF1F938787738A
:10B6C0009C4303D50701828097A7FF1F938787724A
:10B6D0009C4303C52701828097A7FF1F938787712B
:10B6E0009C4303D54701828097A7FF1F93878770EC
:10B6F0009C4303D56701828097A7FF1F9387876FBD
:10B700009C4303D58701828097A7FF1F9387876E8D
:10B710009C4303C5A701828097A7FF1F9387876D6E
:10B720009C4303C5B701828097A7FF1F9387876C4F
:10B730009C4303C5C701828097A7FF1F9387876B30
:10B740009C4303C5D701828097A7FF1F9387876A11
:10B750009C438857828097A7FF1F9387A7699C43C4
:10B7600003D5C702828097A7FF1F9387A7689C43D2
:10B7700003D5E70219E11305800C828097A7FF1F0C
:10B78000938747679C4303C50703828097A7FF1FE2
:10B79000938747669C43C85B828097A7FF1F938768
:10B7A000E7648843828097A7FF1F93876764884375
:10B7B000828019E17D558280F5DE984265DFFDD9F2
:10B7C00017B7FF1F130707861847AA877155058B00
:10B7D000631D072403C507001547E37DA7FC03C7C6
:10B7E00037001305F0057D171377F70FE364E5FCC9
:10B7F00003C35700E30003FC83C86700E38C08FA27
:10B8000003C77700494579171377F70FE364E5FA23
:10B8100003C7A70011481305F7FF1375F50FE36B76
:10B82000A8F803CE97000D481305FEFF1375F50F1A
:10B83000E362A8F803C8B700630908006518137825
:10B84000F80F1305600DE36705F703C5C7007948D6
:10B8500079151375F50FE36FA8F403C8D7000D45EC
:10B860007D181378F80FE36705F503D80701930EE9
:10B8700040175118420813580801E3ED0EF303C8AE
:10B88000E7007D181378F80FE36605F303C8270176
:10B890007D181378F80FE36F05F103C88700C54ED4
:10B8A00075181378F80FE3E70EF103D86701856E7A
:10B8B000938EBEE06D18420813580801E3EC0EEFBA
:10B8C00003D847016D18420813580801E3E40EEF4E
:10B8D00003D887017918420813580801E36C05ED75
:10B8E00003C8A7017D181378F80FE36505ED03C5BC
:10B8F000B7011D487D151375F50FE36DA8EA03C563
:10B90000D701714879151375F50FE365A8EA03D5DA
:10B91000E7011308E00F7D1542054181E36CA8E8BB
:10B9200003C50702494879151375F50FE364A8E8C4
:10B93000C85301C937C834005915130858BFE36B01
:10B94000A8E603A8870237C53400130555BF591868
:10B95000E36205E717A5FF1F232CC54803C60501B1
:10B9600017A5FF1F2328F5480545E375C5E403D84F
:10B970002501D04933760603E31E06E203C615010E
:10B98000E30A06E217A6FF1F2322B64683C5270057
:10B9900001466387A50003C61700F1453306B602CA
:10B9A00083C707039305C00272971A071307C705D9
:10B9B00016031A9796084697B387B70241553E97E4
:10B9C0003297420741836362E8061763FFFFE7028D
:10B9D0000371368597800000E780806B9700010037
:10B9E000E780004B2A8497A00000E780605D2A94DE
:10B9F00097F00000E78040292A9497900000E780A4
:10BA000080842A9497F0FFFFE780E06F2A949740A4
:10BA10000000E78000972A9497700000E780809FDD
:10BA200022951763FFFF6700C36D82801763FFFFD6
:10BA3000E702E36A4111A307A10097A00000E78095
:10BA400080C89305F100170500001305E5B597F0D0
:10BA5000FFFFE780802F014541011763FFFF67006B
:10BA6000436A1763FFFFE702036517A4FF1F130470
:10BA7000645B0328840079599368180097A4FF1F1A
:10BA800023A6145B1378180063100802BA84BE89D9
:10BA9000368B328A2E89AA8A97F0FFFFE780E0A7CB
:10BAA0007D15269519E531594A851763FFFF670013
:10BAB000036497F0FFFFE78040A67D152695A167F8
:10BAC000E353F5FE97B7FF1F9387C78C98433E8CCF
:10BAD000814B01CB014597F00000E7800047933B85
:10BAE00015004A85DA865686D28597900000E78051
:10BAF000A0502A8911CD1C44F99B17A7FF1F2327AB
:10BB0000F75283270C00CDD3E3800BFA829769BFED
:10BB1000268597A7FF1F23A9075097F0FFFFE7800F
:10BB2000809C4146CE8517A5FF1F130525599730E8
:10BB30000100E780A05997D00000E780209C0325F2
:10BB4000040B97D00000E780E09F054597D00000E8
:10BB5000E780E0A6054597000000E78060EDA9B703
:10BB600097A7FF1F9387074C9C47858BEDC71763EB
:10BB7000FFFFE702C35617A5FF1F1305655297A7DE
:10BB8000FF1F23A1074A97A7FF1F23AF074897A7C7
:10BB9000FF1F23AD074897200100E78000849750DE
:10BBA0000000E780C0F897100100E780804F9710F1
:10BBB0000100E780805597A7FF1F938727459C4387
:10BBC00091C7054597800000E780202397A7FF1FB6
:10BBD0009387872D9C4399C741657D159770000019
:10BBE000E78020A597F00000E780C04097D00000D4
:10BBF000E780609297A7FF1F9387C7579C431397CF
:10BC000017016356070097F00000E780E0AF97A7A1
:10BC1000FF1F23A5074A97A7FF1F23A3074A97A73C
:10BC2000FF1F23A1074A97A7FF1F23AF07489700CD
:10BC30000000E780008C97000000E780A07597F077
:10BC4000FFFFE780401897F00000E78020D91763D6
:10BC5000FFFF6700034B828097A7FF1F9387873CF6
:10BC60008843828097A7FF1F9387C73BC843828082
:10BC7000B7E7B0009387075063E1A70297A7FF1FBC
:10BC80009387473AD843FD576367E50097A7FF1F9F
:10BC900023ACA73881473E858280B957EDBF176333
:10BCA000FFFFE702C34397800000E780A0749780FE
:10BCB0000000E78000771763FFFF67008344176386
:10BCC000FFFFE70223402A849304140201112E850A
:10BCD000B289A685214636C63A8997300100E780A9
:10BCE000803C0DE9B24638082686CE8513059404BB
:10BCF00097500000E780A04021462C084A859730E5
:10BD00000100E780403A1335150005611763FFFF16
:10BD10006700833E0145D5BF1763FFFFE702233C61
:10BD20009305450617A5FF1F1305050D9710010084
:10BD3000E78060681763FFFF6700A33C1763FFFF9E
:10BD4000E702E33941112EC697F0FFFFE780C017E5
:10BD5000B24588C141011763FFFF6700833A17634B
:10BD6000FFFFE7022336AA842E8497800000E78035
:10BD7000406BAA898545228597000000E780E07D19
:10BD800083C7E4011389940899E313890403CE85DA
:10BD9000228597000000E780407C21469305190228
:10BDA000228597000000E780607897A7FF1F9387A0
:10BDB00067278C43228597100000E780C0822146C8
:10BDC00093858402228597000000E7802076176320
:10BDD000FFFF670063321763FFFFE702C32D39716E
:10BDE00097F00000E78020B49305400661E9978052
:10BDF0000000E780405F6302051497A7FF1F83C719
:10BE0000670113B7170097A6FF1F2385E6000144BB
:10BE100099CFC16417A9FF1F1309C9209309400EC8
:10BE2000FD1497000000E78020836342A40A97F086
:10BE3000FFFFE78060094169B7290900096AFD7AB7
:10BE40002A8B81447D199389F97B130A0A71938A9D
:10BE50008AC797000000E780208063D7A4041304FA
:10BE6000400EB387840217A7FF1F1307A71B0324E5
:10BE7000070B3E948357C4016382270B1840330796
:10BE8000EB4063EAE900834744008507B387470333
:10BE9000D6976365F70801468145094597F0FFFF8E
:10BEA000E780C04AAA8B29E597400000E780C0825E
:10BEB00085476317F50689659385057117A5FF1FEB
:10BEC000130585F397100100E780E04E95A0B307B6
:10BED00034030327090BBA9703D7C70163089700F8
:10BEE00003C75700A38207002382E700050415BF9C
:10BEF0009305C500228597000000E78080E65E85F7
:10BF0000228697650100938565E597F0FFFFE7803E
:10BF1000404F5E8597100000E780608A850415BF5A
:10BF200097A7FF1F938707109C478D83858BC1F7C9
:10BF300021611763FFFF6700831B014685450945A3
:10BF400002D002D202D402D697F0FFFFE780004071
:10BF5000AA8479DD97F00000E780209C1389C40053
:10BF60002A8481454A8597000000E780005F0C40E5
:10BF700041464A8597000000E780405B83294400E2
:10BF80006385090C4E8502D802DA02DC02DE9730A6
:10BF90000100E78020382ACE141005462C08081826
:10BFA0004ECC97500000E780200A1375F50F51ED35
:10BFB0008355840093E525004A8597000000E780BB
:10BFC000E05E11460C104A8597000000E78000569D
:10BFD0000146976501009385E5D8268597F0FFFF18
:10BFE000E7802042268597000000E780407D5C4086
:10BFF000A1D3014685450D4597F0FFFFE780003549
:10C00000AA841DD548401389C40097300100E780F9
:10C0100060302AC64A8597000000E780404C3246CF
:10C02000636FC5004C404A8597000000E7800050D0
:10C0300001468145268597F0FFFFE780803C2685F5
:10C0400097000000E780A077E5B583558400ADB781
:10C050001763FFFFE702A30897A7FF1F938787FCDB
:10C060009C471DC193E7870017A5FF1F1305C5D87F
:10C0700017A7FF1F232CF7FA97100100E7808031E4
:10C080001763FFFF6700E307DD9B17A7FF1F232F41
:10C09000F7F897300000E78020647DF117A5FF1FB7
:10C0A000130585D597100100E7802033D1BF1763B2
:10C0B000FFFFE70243004169AA892E8AB28A368BC4
:10C0C000BA8B814417ACFF1F130CCCF5930C400EB8
:10C0D0007D1997F0FFFFE780205863C4A400014456
:10C0E0003DA03384940383270C0B3E948357C401F3
:10C0F000638627055A87D6865286CE8513050403A4
:10C1000097000000E780E0BB01C923800B00228577
:10C110001763FFFF6700A3FD8347F40185C35A87B8
:10C12000D6865286CE851305940897000000E780D6
:10C1300040B909C585472380FB00D1BF850451BFA5
:10C14000835745006380071E1763FFFFE70283F7ED
:10C1500001112A8497000000E780C04D09C9854776
:10C160006309F50605611763FFFF6700E3F897E0D1
:10C170000000E780407B7DF5835744004947ED9BF5
:10C18000E392E7FEC145228597000000E780403337
:10C19000AA84228597000000E780204F03574400BF
:10C1A00002CE91472A89631AF70022859700000082
:10C1B000E780A0513C082ACC3ECE97E00000E78003
:10C1C000C0755C55C5D374084A86A6850545829717
:10C1D00051BF03574400D147E3F6E7F8032A0400B0
:10C1E000C169014997AAFF1F938ACAE3130B400E46
:10C1F000FD1997F0FFFFE7802046634FA90E2285C7
:10C20000032A040097000000E780C042A1452A8964
:10C21000228597000000E780A02AAA842285970043
:10C220000000E780804A14402A86AA89780826857B
:10C23000CA8597000000E780C0E7AA8405D503C738
:10C24000F40189476315F7008347C10181DF554633
:10C25000D2851385640097300100E78020E701450F
:10C2600097800000E780001901C583D7C401A5E7C6
:10C2700097A7FF1F938707DB9C4793551900858974
:10C2800013D73700058B01CF8983858B6399B7005E
:10C2900001452EC697000000E780C0DBB2454E8501
:10C2A00097800000E780A01E0346C1012A84937591
:10C2B0001900268597900000E780203935C1268532
:10C2C00097800000E7802018268511C001459780DF
:10C2D0000000E780404B97300000E780E03F854753
:10C2E000E312F5E883C754001307F00FE38CE7E689
:10C2F0008507A382F400BDB5B304690383A70A0BC5
:10C30000BE9483D7C401638B37015546D28513850C
:10C31000640097300100E78000D955DD0509D1BDE3
:10C320005DD86DB782801763FFFFE702A3D99780BE
:10C330000000E780400B05C1C164014417A9FF1F3D
:10C34000130949CE9309400EFD1497F0FFFFE780D3
:10C35000A030634EA40017A5FF1F1305E5A9971091
:10C360000100E78020031763FFFF6700E3D8330570
:10C3700034038327090B3E958357C50163889700D3
:10C380002312050097800000E780E00B050475BFCD
:10C3900097A7FF1F938707C99C478D83858B8DE3E4
:10C3A0001763FFFFE702A3D317A5FF1F1305C5A45B
:10C3B00097100100E78060021763FFFF670063D4F6
:10C3C00082801763FFFFE70283D197050000938502
:10C3D000C5A017A5FF1F130525A297100100E78030
:10C3E00060ED1763FFFF6700C3D11763FFFFE7022C
:10C3F00003CF8841B7E70400BC5B050542054181D6
:10C40000829709C585472300F50005051763FFFFDF
:10C41000670023CF83C7F5FF2E858507A38FF5FE21
:10C42000828083C7F5FFFD1793F7F70FA38FF5FE03
:10C4300099EF1763FFFFE70283CAB7E70400BC5711
:10C440001385F5FF82971763FFFF670083CB828018
:10C450001C41035745008D8FBA951CC12312B500AE
:10C460003E85828093D78500A2051441DD8D8357D8
:10C4700045001387E6FF18C189072312F50013D67C
:10C4800085004111238FB6FEA38FC6FE4101828035
:10C4900018419307F7FF1CC18357450085072312F6
:10C4A000F500A30FB7FE8280835745008D8F2312BE
:10C4B000F5001C41BE950CC12E858280AA8703D74A
:10C4C000470008410D8FAA952392E7008CC3828014
:10C4D000184108453305A74082808357450003571C
:10C4E00065001D8F1C4108453385A7403305A740D3
:10C4F00082801763FFFFE70283BE41112EC62A84A4
:10C5000097000000E780A0FDB2456373B50001A06D
:10C51000835744000840BE952312B4003E95410164
:10C520001763FFFF6700E3BD1763FFFFE70223BB4D
:10C5300041112E84B28532C697000000E780A0FB2F
:10C540003246A28597300100E78040B84101176369
:10C55000FFFF670003BB1763FFFFE70243B82E84AA
:10C56000854597000000E78000F9230085001763E8
:10C57000FFFF670003B91763FFFFE70243B64111EE
:10C580002317B100894597000000E780C0F6834774
:10C59000E1002300F5008347F100A300F50041010D
:10C5A0001763FFFF6700E3B51763FFFFE70223B3DD
:10C5B00093D78500A2054111DD8D2317B100894570
:10C5C00097000000E78020F38347E1002300F50097
:10C5D0008347F100A300F50041011763FFFF6700E7
:10C5E00043B21763FFFFE70283AF1397850193D729
:10C5F0008501C166938606F0D98F13D78500758FA4
:10C60000D98FA2053707FF00F98D4111DD8D2EC6A8
:10C61000914597000000E78000EE6C0011469730CE
:10C620000100E780A0AA41011763FFFF670063AD27
:10C630001763FFFFE702A3AA1C41854503C4070057
:10C6400097000000E78080E622851763FFFF670000
:10C6500043AB1763FFFFE70283A81C4141118945E3
:10C6600003C7070083C717002307E100A307F100F2
:10C6700097000000E78080E30355E1004101176364
:10C68000FFFF670003A81763FFFFE70243A51C41F4
:10C690004111894503C7070083C717002307E1003D
:10C6A000A307F10097000000E78040E08357E10016
:10C6B000410113D58700A2075D8D420541811763B3
:10C6C000FFFF670003A41763FFFFE70243A10C41CC
:10C6D00041112A841146680097300100E780009FCD
:10C6E0009145228597000000E78040DCB247C16693
:10C6F000938606F01397870113D58701598D13D7B9
:10C700008700758F598DA2073707FF00F98F5D8D60
:10C7100041011763FFFF6700C39E1C45BE950CC116
:10C720008280AE87944391E6584101EF0CC15CC111
:10C73000828003C7570013671700A382E700B687FC
:10C74000D5B70CC3EDB7AA87084119CD1841D4431A
:10C7500098C36313D500D8C32A870346570093763E
:10C76000160081E6232007008280944381CA8C4210
:10C7700003A847008CC363930601CCC3799A14C302
:10C78000A302C7003687D1BF1C45DC471D8DB77794
:10C79000DBB6938777DB09853305F50242054181D6
:10C7A0008280F147B385F50248452E958280834704
:10C7B000450085072302F50082801763FFFFE7022B
:10C7C00003922A8409E41763FFFF6700839383477A
:10C7D0004400F5DBFD1793F7F70F2302F400E5F7AC
:10C7E0001C4403D7270005072391E700DC4399C3C6
:10C7F000228582974C4889CD83475400898B99E7DD
:10C800001C4422859C479C439C478297232A040012
:10C810000040232004007DB71763FFFFE702238C4D
:10C820008357250041112EC681EB01442285410129
:10C830001763FFFF6700E38C035705008147F1464C
:10C84000E305F7FEB385D702404585072E9483455F
:10C85000440008C4F5F5B247AA8481E7232A0400FE
:10C8600009A81C456C0022859C439C43829748C8BC
:10C870004DDD85472312F400B2472320040023181E
:10C8800004002319F4005C485CC483D72400FD171E
:10C890002391F40061BF1763FFFFE702438497977A
:10C8A000FF1F93876757884323260500232405002D
:10C8B000410597100100E78040B21763FFFF670052
:10C8C00043841763FFFFE70283811794FF1F13045C
:10C8D000A4541C40411199CF9C472300B5002AC69F
:10C8E0005CC197000000E78040FB1C40DC4399C31B
:10C8F0003245829741011763FFFF6700838003473A
:10C90000450029E3584DAA877D551DCF1753FFFFDA
:10C91000E702E37C1CC3DC479796FF1F23AEE64E7D
:10C92000F156130507012390D70097050000938562
:10C93000050297100100E780E09701451753FFFFBC
:10C940006700237C7D55828082801753FFFFE702BA
:10C95000037901116146814528009750FFFFE78068
:10C96000007B9797FF1F9387274B9C4328009305D5
:10C97000F00FDC473EC697000000E780C0F4056179
:10C980001753FFFF6700E3779797FF1F9387C74809
:10C990009C43D847A1679387C702631EF70A397182
:10C9A00006DE22DC26DA80004AD84ED652D456D291
:10C9B0003285B28497000000E780C0C7AA89268527
:10C9C00097000000E78020C92318A4FC2685970063
:10C9D0000000E78040C82319A4FC268597000000CA
:10C9E000E78060C783D744000A8A231AA4FC8583A2
:10C9F00093F7F70F230EF4FC8607BD0793F7073F65
:10CA00003301F1408A8A01498347C4FD6367F90213
:10CA1000CE85130584FC232C54FD97000000E7808D
:10CA200080EA5281130104FCF2506254D2544259FC
:10CA3000B259225A925A21618280268597000000BD
:10CA4000E78060C193171900D69705092390A700C6
:10CA50001379F90F55BF82809797FF1F9387C73BC4
:10CA60009C43D847A1679387A702631AF70A3971D5
:10CA700006DE22DC26DA80004AD84ED652D456D2C0
:10CA80003285B28497000000E780C0BAAA89268563
:10CA900097000000E78020BCFD572318A4FC2685E2
:10CAA0002319F4FC97000000E780E0BA83D7440024
:10CAB0000A8A231AA4FC858393F7F70F230EF4FC4C
:10CAC0008607BD0793F7073F3301F1408A8A014982
:10CAD0008347C4FD6367F902CE85130584FC232CCC
:10CAE00054FD97000000E78000DE5281130104FC32
:10CAF000F2506254D2544259B259225A925A216188
:10CB00008280268597000000E780E0B49317190023
:10CB1000D69705092390A7001379F90F55BF828096
:10CB20009797FF1F9387472F9C43D847A167890793
:10CB30006310F70A397106DE22DC26DA80004AD853
:10CB40004ED652D456D23285328997000000E78003
:10CB500060AEAA894A8597000000E780C0AF83577E
:10CB600049000A8A2318A4FC858393F7F70F230C46
:10CB7000F4FC8607BD0793F7073F3301F1408A8A2B
:10CB80008144834784FD63E7F402CE85130584FC6A
:10CB9000232A54FD97000000E780E0D25281130160
:10CBA00004FCF2506254D2544259B259225A925A59
:10CBB000216182804A8597000000E780C0A9939791
:10CBC0001400D69785042390A70093F4F40F55BF63
:10CBD00082809797FF1F938727249C43D847A1679C
:10CBE0009387E704631EF70A397106DE22DC26DA32
:10CBF00080004AD84ED652D456D23285B28497009D
:10CC00000000E78020A3AA89268597000000E7801E
:10CC100080A42318A4FC268597000000E780A0A329
:10CC2000231AA4FC268597000000E780C0A283D7C2
:10CC300044000A8A2319A4FC858393F7F70F230E77
:10CC4000F4FC8607BD0793F7073F3301F1408A8A5A
:10CC500001498347C4FD6367F902CE85130584FC4F
:10CC6000232C54FD97000000E780E0C5528113019A
:10CC700004FCF2506254D2544259B259225A925A88
:10CC800021618280268597000000E780C09C931771
:10CC90001900D69705092390A7001379F90F55BFFE
:10CCA00082809797FF1F938727179C43D847A167D8
:10CCB0009387C704631AF70A397106DE22DC26DA85
:10CCC00080004AD84ED652D456D23285B2849700CC
:10CCD0000000E7802096AA89268597000000E7805B
:10CCE0008097FD572318A4FC2685231AF4FC97008F
:10CCF0000000E780409683D744000A8A2319A4FCE9
:10CD0000858393F7F70F230EF4FC8607BD0793F78F
:10CD1000073F3301F1408A8A01498347C4FD6367B5
:10CD2000F902CE85130584FC232C54FD97000000E6
:10CD3000E78060B95281130104FCF2506254D2546E
:10CD40004259B259225A925A21618280268597000F
:10CD50000000E780409093171900D69705092390AB
:10CD6000A7001379F90F55BF82809797FF1F93870C
:10CD7000A70A9C43D847A167DD076317F704175339
:10CD8000FFFFE702C33579713285328497000000D6
:10CD9000E780408A2AC6228597000000E780A08BA2
:10CDA0002311A102228597000000E780A088B245E8
:10CDB0002300A102280897000000E780C0B0456169
:10CDC0001753FFFF6700E33382809797FF1F938716
:10CDD000A7049C43D847A167938787046317F70488
:10CDE0001753FFFFE702A32F797132853284970032
:10CDF0000000E78020842AC6228597000000E78093
:10CE000080852311A102228597000000E78080829F
:10CE1000B2452300A102280897000000E780A0AADD
:10CE200045611753FFFF6700C32D82809797FF1F4F
:10CE3000938787FE9C43D847A1679387A704631213
:10CE4000F7021753FFFFE7028329011128008145EC
:10CE500097000000E78020A705611753FFFF6700D8
:10CE6000432A82809797FF1F938707FB9C43D847ED
:10CE7000A167938757026319F7021753FFFFE70271
:10CE800003260111328597F0FFFFE780A07A23087F
:10CE9000A1008145280097000000E780C0A205613D
:10CEA0001753FFFF6700E32582809797FF1F938743
:10CEB000A7F69C43D847A1679387E702631BF70453
:10CEC0001753FFFFE702A32101113285328497F047
:10CED000FFFFE7804078AA84228597F0FFFFE78074
:10CEE0008077854709E9228597F0FFFFE780807406
:10CEF0004205B337A00028008145231891003ECA9F
:10CF000097000000E780209C05611753FFFF670032
:10CF1000431F82809797FF1F938707F09C43D84752
:10CF200099476313F7081753FFFFE702431B797113
:10CF30003285328497F0FFFFE780C06F2AC62285D2
:10CF400097F0FFFFE78020712310A102228597F060
:10CF5000FFFFE780206E2301A102228597F0FFFFEB
:10CF6000E780406DA301A102228597F0FFFFE780D3
:10CF7000606C2302A102228597F0FFFFE780806B9F
:10CF80002313A102228597F0FFFFE780A06AB24534
:10CF90002314A102280897000000E780C092456191
:10CFA0001753FFFF6700E31582809797FF1F938752
:10CFB000A7E69C43D847A1679387C7036313F70885
:10CFC0001753FFFFE702A31179713285328497F07E
:10CFD000FFFFE78020662AC6228597F0FFFFE780E3
:10CFE00080672310A102228597F0FFFFE780A066EB
:10CFF0002311A102228597F0FFFFE780A06323029F
:10D00000A102228597F0FFFFE780C062A302A10280
:10D01000228597F0FFFFE780E0612303A1022285CC
:10D0200097F0FFFFE7800061B245A303A102280843
:10D0300097000000E780208945611753FFFF6700D4
:10D04000430C82801753FFFFE702630901112A8412
:10D0500097F0FFFFE780005EAA84228597F0FFFF2C
:10D06000E780605F228597F0FFFFE780C05E03578F
:10D0700044008D4763F7E700228597F0FFFFE780C4
:10D08000805D228597F0FFFFE780E05C2800A685A1
:10D0900097000000E780208305611753FFFF6700BA
:10D0A00043069797FF1F938727D79C43D847A167CD
:10D0B000FD07631FF7001753FFFFE70243023285A6
:10D0C00097000000E78040F81753FFFF67006303F5
:10D0D00082809797FF1F938727D49C43D847A167E7
:10D0E000E5076315F7081753FFFFE70243FF797160
:10D0F0003285328497F0FFFFE780C0532AC622852D
:10D1000097F0FFFFE7802055228597F0FFFFE7802B
:10D1100080542310A102228597F0FFFFE780A053DF
:10D12000520551812311A10222852302010297F0A9
:10D13000FFFFE7802050A302A102228597F0FFFFA6
:10D14000E780404F2303A102228597F0FFFFE7808D
:10D15000604EB245A303A102280897F0FFFFE780C5
:10D16000807645611753FFFF6700A3F98280979788
:10D17000FF1F938767CA9C43D847A1679387E7033C
:10D18000631FF7001753FFFFE70263F5328597002F
:10D190000000E78060EB1753FFFF670083F6828093
:10D1A0009797FF1F938747C79C43D847A1679387EB
:10D1B0004704631EF7021753FFFFE70243F279713A
:10D1C0003285328497F0FFFFE780C0462AC6228569
:10D1D00097F0FFFFE7802048B245280897F0FFFF4F
:10D1E000E780606E45611753FFFF670083F182801F
:10D1F0009797FF1F938747C29C43D847A1679387A0
:10D2000087026310F7041753FFFFE70243ED7971BC
:10D210003285328497F0FFFFE780C0412AC622851D
:10D2200097F0FFFFE7800041B2452300A1022808E4
:10D2300097F0FFFFE780206945611753FFFF670004
:10D2400043EC82801753FFFFE70263E9011197F077
:10D25000FFFFE780203EAA85280097F0FFFFE780C8
:10D26000806605611753FFFF6700A3E99797FF1FCB
:10D27000938787BA9C43D847A167D107631FF700FC
:10D280001753FFFFE702A3E5328597000000E78010
:10D29000A0FB1753FFFF6700C3E682809797FF1F2D
:10D2A000938787B79C43D847A167C507631FF700DB
:10D2B0001753FFFFE702A3E2328597000000E780E3
:10D2C000A0F81753FFFF6700C3E382809797FF1F03
:10D2D000938787B49C43D847A167B907631FF700BA
:10D2E0001753FFFFE702A3DF328597000000E780B6
:10D2F000A0F51753FFFF6700C3E082809797FF1FD9
:10D30000938787B19C43D847A167AD07631FF70098
:10D310001753FFFFE702A3DC328597000000E78088
:10D32000A0F21753FFFF6700C3DD82809797FF1FAE
:10D33000938787AE9C43D84789476318F7021753F2
:10D34000FFFFE702C3D90111328532C897F0FFFF12
:10D35000E780402EAA85280097F0FFFFE780A056BF
:10D3600005611753FFFF6700C3D982809797FF1F9E
:10D37000938787AA9C43D847A1678D076311F70459
:10D380001753FFFFE702A3D501113285328497F0CE
:10D39000FFFFE780202A13066100AA844C00228543
:10D3A00097300000E78000232800A68597F0FFFF54
:10D3B000E780605105611753FFFF670083D48280C7
:10D3C0009797FF1F938787A59C4381CFDC4391CB21
:10D3D0001753FFFFE702A3D082971753FFFF6700A1
:10D3E00043D282801753FFFFE70263CF79713C0875
:10D3F000AE843ED2A165B7070A002A843ED4481005
:10D400003C08DD053ED636C432C63AC297D0FFFF8F
:10D41000E780402C12474810BA8597F0FFFFE7805D
:10D42000C01332464810B28597F0FFFFE780E01442
:10D43000A2464810B68597F0FFFFE7800012501013
:10D4400001478146A685228597D0FFFFE780E04D02
:10D4500045611753FFFF6700C3CA1753FFFFE70279
:10D4600003C801117C000329C501AE843ECAA16531
:10D47000B70707002A843ECC48087C00C5053ECE8D
:10D4800097D0FFFFE78000258345D900480897F033
:10D49000FFFFE780800C500801478146A685228562
:10D4A00097D0FFFFE780604805611753FFFF6700D3
:10D4B00043C51753FFFFE70283C283C7950093F765
:10D4C000F707A384F50097000000E78040F91753A1
:10D4D000FFFF670003C31753FFFFE70243C07971E3
:10D4E0003C08AE843ED2A165B70709002A843ED429
:10D4F00048103C08938545043ED632C636C497D0C2
:10D50000FFFFE780201DA2464810B68597F0FFFF79
:10D51000E780A00432464810B28597F0FFFFE7800D
:10D52000C005501001478146A685228597D0FFFF90
:10D53000E780A03F45611753FFFF670083BC175387
:10D54000FFFFE702C3B983C7950041112A8493F70F
:10D55000F707A384F50032852EC697F0FFFFE7801A
:10D56000800F85672AC46370F50297700000E7801A
:10D5700060E82246B24509ED1147814622859700B1
:10D580000000E78060E641011753FFFF670063B7C3
:10D5900001478346F501DDB71753FFFFE70283B26A
:10D5A00001113C003ECAB7070A003ECC3C003ECE0B
:10D5B00083C79500AA89328593F7F707A384F500FE
:10D5C0002E8497F0FFFFE78000098567637DF504EF
:10D5D000A165AA8493858504480897D0FFFFE7805A
:10D5E000600F268597700000E780C0E02A8929E156
:10D5F0009145480897F0FFFFE78020F6A685480888
:10D6000097F0FFFFE78060F7CA85480897F0FFFFB3
:10D61000E780A0F4014781465008A2854E8597D047
:10D62000FFFFE780803005611753FFFF6700C3AC41
:10D630008145480897F0FFFFE78020F2034909027F
:10D6400075BF1753FFFFE702E3A779711C103ECAAD
:10D65000B7070F003ECC404D1C10AA84AE89480885
:10D66000994532C636893ECE97D0FFFFE7808006C7
:10D6700032464808B28597F0FFFFE78000EE630C62
:10D680000902A545480897F0FFFFE780C0E6254658
:10D69000CA8597200100E78060A3500801478146B2
:10D6A000CE85268597D0FFFFE78020284561175358
:10D6B000FFFF670063A48355C402480897F0FFFF8B
:10D6C000E780A0EB0355E402814505C58547854504
:10D6D0006301F502C167FD179305F00F630BF500B9
:10D6E0007D1597700000E780608D9305150093F518
:10D6F000F50F480897F0FFFFE78020E68345040315
:10D70000480897F0FFFFE78040E583451403480889
:10D7100097F0FFFFE78060E483552403480897F003
:10D72000FFFFE78080E583554403480897F0FFFF3B
:10D73000E780A0E49DB71753FFFFE702439A83C732
:10D7400095008146014693F7F707A384F5009700FB
:10D750000000E78040EF1753FFFF6700839A1753DD
:10D76000FFFFE702C39779713E841C103ECA2E89E1
:10D77000B7070F00A1653ECCFD051C10AA84480820
:10D7800042C03AC23ECE36C432C697D0FFFFE780D1
:10D7900060F432464808B28597F0FFFFE780E0DB8F
:10D7A000A2464808B68597F0FFFFE78000DD1247E4
:10D7B0004808BA8597F0FFFFE78020DC0248630C39
:10D7C00008029145480897F0FFFFE780C0D2114654
:10D7D000A28597200100E780608F500801478146AD
:10D7E000CA85268597D0FFFFE7802014456117532F
:10D7F000FFFF670003918945480897F0FFFFE78026
:10D8000080CF834704002300F50083471400A30062
:10D81000F500E1B71753FFFFE702C38A83C79500FE
:10D8200001112A8A93F7F707A384F5003285AE84A5
:10D8300032C697F0FFFFE78000E232462A89328540
:10D8400097F0FFFFE78000DF85676373F902AA891D
:10D850004A8597700000E780E0B92A8419ED1147E6
:10D8600081464A86A685528597000000E780C0B7AA
:10D8700005611753FFFF670023889387E9FF93F73C
:10D88000F70F0547E366F7FE8347F50195EB8947F8
:10D89000E380F9FE8346F401528501474A86A68556
:10D8A00097000000E78040B4A167D90748083ECC44
:10D8B000230A010002CE97000000E780A0B04DBF10
:10D8C000639EE7008947639EF90093071020231F9A
:10D8D000F50097700000E78000B76DBF0947E39B34
:10D8E000E7FA8D47E398F9FA228597700000E78000
:10D8F000C0DE9787FF1F938767719C4399E79787DF
:10D90000FF1F9387675A9C4399C703D504009780EC
:10D910000000E780E0CD231F040022855DBF174390
:10D92000FFFFE702C37B01113C003ECAB7070B00B3
:10D930003ECC3C003ECE83C795002A89328593F7C2
:10D94000F707A384F500AE8497F0FFFFE780A0D02F
:10D9500093170501C187635AF006A1652A84938550
:10D96000E502480897D0FFFFE780C0D6A2854808A7
:10D9700097F0FFFFE78060C09787FF1F9387C7522C
:10D980009C43A9EB01449375F40F480897F0FFFFFF
:10D99000E780A0BC9355844093F5F50F480897F0B5
:10D9A000FFFFE78080BB9355044193F5F50F4808CE
:10D9B00097F0FFFFE78060BA014781465008A685CF
:10D9C0004A8597D0FFFFE78040F605611743FFFFC8
:10D9D00067002373416585460546A2857D159750EE
:10D9E0000000E780A0BC59DD510597000100E780E9
:10D9F000C08E130440063344850271B71743FFFFFE
:10DA0000E702E36D0111B70706003EC683C7950024
:10DA100021642A8993F7F707A384F500AE842800D0
:10DA20009305A4040AC40AC897D0FFFFE78080CA00
:10DA3000300001478146A6854A8597D0FFFFE780E1
:10DA4000C0EE97E0FFFFE780E0111304940448085C
:10DA500022CC230A010002CE97000000E7808096C6
:10DA600005611743FFFF6700C3691743FFFFE70224
:10DA70006365C1642A8901449789FF1F9389895A84
:10DA8000130A8002FD1497E0FFFFE780E0BD6347C3
:10DA9000A40001451743FFFF67000366B307440373
:10DAA00003A7C90ABA9703D707006306970083D76D
:10DAB0002700638427010504F9B70545E1BF174333
:10DAC000FFFFE70223602A8A2E8999C123A005005F
:10DAD00081498144978AFF1F938A8A34614B97E07A
:10DAE000FFFFE780A0BE63C7A4004E851743FFFF7A
:10DAF000670083603384640383A70A003E948357DE
:10DB0000040099E763040900232089008504C1BF4C
:10DB10004146D2851305440097100100E780A058C4
:10DB200075F5A289E5B71743FFFFE702A3593971DD
:10DB30007C083ED4B7070A003ED67C083ED883C78F
:10DB400095002A8A328593F7F707A384F5002E897A
:10DB500032C697F0FFFFE78000B085676373F50872
:10DB60003246AA84328597F0FFFFE780A0AC854754
:10DB7000AA8963E8A706A16593858504281097D034
:10DB8000FFFFE78020B5268597700000E78080863C
:10DB90002A8429ED9145281097F0FFFFE780E09B4C
:10DBA000A685281097F0FFFFE780209DCE852810DE
:10DBB00097F0FFFFE780609A014781463010CA85E1
:10DBC000528597D0FFFFE78040D6A16793877704FF
:10DBD00048183EDC230A010202DE97F0FFFFE780CF
:10DBE000607E21611743FFFF6700035181452810C4
:10DBF00097F0FFFFE7806096A685281097F0FFFF5B
:10DC0000E780A0979787FF1F938787789C4381CBF6
:10DC100022856389090097D00000E780802383452F
:10DC2000040271B797D00000E7800022CDBF1743F0
:10DC3000FFFFE702234983C795004111AA8993F7A3
:10DC4000F707A384F5003285AE84328A97F0FFFF90
:10DC5000E78060A08567637FF5022A8997600000EE
:10DC6000E78040792A84914631C58347F50105470D
:10DC70006387E70291C70D476366F704AD461DA8A9
:10DC80009305050303250A00414697100100E7802C
:10DC900080410DE941011743FFFF6700E34593050C
:10DCA000950803250A00414697100100E780A03F30
:10DCB000814669F54A86A6854E8597000000E78073
:10DCC000C081C9BF83250A0013059408977000001E
:10DCD000E780E02819C1C146F1BF9787FF1F9387EE
:10DCE000E7329C4399E79787FF1F9387E71B9C4385
:10DCF00099C7228597800000E780608969FD854784
:10DD0000A30FF400228597B00000E780A08322854E
:10DD100097600000E78020734E8581464A86A6857D
:10DD200097F0FFFFE780607BA16793875704480067
:10DD30003EC42302010002C697F0FFFFE78080681F
:10DD400091BF1743FFFFE702033783C795004111D7
:10DD5000AA8993F7F707A384F50032852E89B28A42
:10DD600097F0FFFFE780208F85676374F50EAA8424
:10DD700097600000E78000682A840DED416B014A3E
:10DD8000978BFF1F938B0B2A130C400E7D1B19A83A
:10DD900033048A0383A70B0B3E948357C401638328
:10DDA0006705050A97E0FFFFE780008BE342AAFEC4
:10DDB00095460DA08357C501639697029305050309
:10DDC00003A50A00414697100100E780C02D99463F
:10DDD00011E181462686CA854E8597F0FFFFE780D0
:10DDE000C06F85A883A50A0013050403977000007F
:10DDF000E780E016C14679FD2285231E940097A096
:10DE00000000E7802074228597600000E780A0630F
:10DE10009787FF1F9387C7579C43A9C3230004021A
:10DE2000228597D00000E78080EF4E8581462686C8
:10DE3000CA8597F0FFFFE780406AA16793870704D0
:10DE400048003EC42302010002C697F0FFFFE780AE
:10DE5000605741011743FFFF67006329894723008B
:10DE6000F402E1B7397106DE22DC4AD8800052D4D0
:10DE700056D25AD026DA4ED65ECE2E8A32892A8BD8
:10DE800097D0FFFFE780407A0605710541998A8A9D
:10DE90003301A140232224FC231404FC97D0FFFF6C
:10DEA000E780807883479A000605350593F7F707E2
:10DEB0002315A4FCA304FA004A85232624FC97E03A
:10DEC000FFFFE780407993170501C1876340F002A7
:10DED0005681130104FCF2506254D2544259B25993
:10DEE000225A925A025BF24B21618280AA844A85AF
:10DEF00097E0FFFFE7802076AA894A8597E0FFFF39
:10DF0000E7806075A1659385C5022A89130544FCE5
:10DF100097C0FFFFE780007C268597C0FFFFE78062
:10DF20004070854511C94A86CE8597C0FFFFE780BE
:10DF3000C069AA8B21E98945130544FC97E0FFFFDE
:10DF4000E780A061A685130544FC97E0FFFFE7800A
:10DF5000C062CE85130544FC97E0FFFFE780E061D7
:10DF6000CA85130544FC97E0FFFFE7800061014785
:10DF70008146130644FCD2855A8597D0FFFFE7807F
:10DF8000C09AB9B78145130544FC97E0FFFFE780CD
:10DF9000C05CA685130544FC97E0FFFFE780E05DC9
:10DFA000CE85130544FC97E0FFFFE780005DCA853E
:10DFB000130544FC97E0FFFFE780205C814497D085
:10DFC000FFFFE7806066E3D4A4FA83A70B011397F1
:10DFD0001400BA9783D5070099C5130544FC97E050
:10DFE000FFFFE78080598504D9BF797106D622D416
:10DFF0004AD000184ECE52CC56CA26D25AC8AE8944
:10E000003289AA8A97D0FFFFE7800062060569057A
:10E0100041990A8A3301A140232A24FC231C04FCD1
:10E0200097D0FFFFE780406083C7990006052D0564
:10E0300093F7F707231DA4FCA384F9004A85232E38
:10E0400024FC97E0FFFFE780006193170501C1877B
:10E05000634FF0005281130104FDB25022549254D8
:10E060000259F249624AD24A424B45618280AA84EF
:10E070004A8597E0FFFFE780005EA1659385A502D2
:10E080002A89130544FD97C0FFFFE780A064268519
:10E0900097C0FFFFE780E058854509C9CA8597C04A
:10E0A000FFFFE78080552A8B29E18945130544FD50
:10E0B00097E0FFFFE780604AA685130544FD97E0DF
:10E0C000FFFFE780804BCA85130544FD97E0FFFF03
:10E0D000E780A04A01478146130644FDCE85568558
:10E0E00097D0FFFFE7806084B5B78145130544FDF5
:10E0F00097E0FFFFE7806046A685130544FD97E0A3
:10E10000FFFFE7808047CA85130544FD97E0FFFFC6
:10E11000E780A046814497D0FFFFE780E050E3DB33
:10E12000A4FA83270B0113971400BA9783D507002D
:10E1300099C5130544FD97E0FFFFE780004485047F
:10E14000D9BF1743FFFFE70283F983474500404DDE
:10E15000D5EFFD575DC48346940009476363D70A32
:10E160000346B400854663EEC6088306E40063CA2E
:10E1700006085C45F9562390D7009787FF1F83C791
:10E1800067CA99E3A304E4009787FF1F9387C7D169
:10E190009C4381E78947A306F4009787FF1F938775
:10E1A000271F9C4381E789472306F4009705000059
:10E1B00093854506AA841305040197F00000E780C3
:10E1C000600FFD57231AF40281471CDC0148978732
:10E1D000FF1F23A587C49787FF1F938767C4232E3C
:10E1E000040304C0804397D0FFFFE780204E6146C0
:10E1F0003306C502814522859740FFFFE78020F165
:10E2000081473E851743FFFF6700A3EFFD57D5BF4A
:10E210001743FFFFE702A3EC2A84035545029760EA
:10E220000000E780201D19E5231E04001743FFFFAF
:10E23000670023ED8357E401F5DB930504FF1745E1
:10E2400001001305E5EB97E00000E7802014F9BF1B
:10E250001743FFFFE702A3E82E89A16541119385CB
:10E26000E5032A8436C432C6BE843AC297C0FFFF93
:10E27000E780404612472285BA8597E0FFFFE78096
:10E28000C02D32462285B28597E0FFFFE780E02E61
:10E29000A2462285B68597E0FFFFE780002E630344
:10E2A00009029145228597E0FFFFE780C0241146CF
:10E2B000A68597100100E78060E141011743FFFF49
:10E2C000670023E48945228597E0FFFFE780A022CD
:10E2D00083C704002300F50083C71400A300F500E2
:10E2E000E9BF1743FFFFE70283DF83C79500444D73
:10E2F000054793F7F707A384F5001C42411183C734
:10E3000007006367F7062E842A89B1C003C7D400CB
:10E31000630FF7021787FF1F130707B9184305C3D9
:10E32000A386F40097A00000E780804983C7D4004B
:10E3300099E741657D1597400000E780802F83D7DE
:10E340002403918B89C797E00000E78000134A857A
:10E35000A28597F0FFFFE7808010A167C107480002
:10E360003EC42302010002C697F0FFFFE78080054C
:10E3700041011743FFFF6700C3D81743FFFFE702C0
:10E3800003D603D745008D47AA8441112E843289D4
:10E390002E8563E3E70297E0FFFFE780C02BAA85A5
:10E3A00023000900268597C0FFFFE7800025410173
:10E3B0001743FFFF6700E3D497E0FFFFE780A02942
:10E3C0002AC6228597E0FFFFE780E028B24585470F
:10E3D0002A862300F900268597C0FFFFE780E01E0C
:10E3E000F9B7397106DE22DC26DA80004ED652D427
:10E3F00056D24AD85AD05ECEAE89B284AA8A97D075
:10E40000FFFFE780602106051305250241990A8A6E
:10E410003301A140232224FC231404FC97D0FFFFE6
:10E42000E780801F83C7990006054D0593F7F7071E
:10E430002315A4FCA384F9002685232624FC97E059
:10E44000FFFFE780402193170501C1876340F00279
:10E450005281130104FCF2506254D2544259B25911
:10E46000225A925A025BF24B21618280AA8B03AB43
:10E47000040097C0FFFFE780C01A51E583D744002E
:10E4800001498544F11793B71700A301F4FC8347B2
:10E4900034FCA165C9C79385E504130544FC97C006
:10E4A000FFFFE7802023A685130544FC97E0FFFFCC
:10E4B000E780A00ADE85130544FC97E0FFFFE780B4
:10E4C000C00B834734FC114691E30946DA851305F6
:10E4D00044FC97E0FFFFE78060058144630A090080
:10E4E000416B7D1B97D0FFFFE780001363CCA40234
:10E4F00001478146130644FCCE85568597C0FFFF31
:10E50000E780A042B1B7A685130634FC970000004F
:10E51000E780E0E6933415002A8986048DBF938551
:10E52000C504A5BF8327C90013971400BA9783D5E4
:10E53000070063886501130544FC97E0FFFFE7804F
:10E54000C003850445B71743FFFFE702C3B67971DF
:10E550001C103EC4B7070F003EC61C103EC883C740
:10E560009500AA8A328593F7F707A384F500AE8950
:10E57000328497E0FFFFE780000E93170501C18703
:10E58000635AF0062A8A228597E0FFFFE780A00CF5
:10E590002A895285032B040097C0FFFFE78060089B
:10E5A00039ED8357440081440544F11793B71700B0
:10E5B000A303F10083457100DA872287CA86528659
:10E5C000280097000000E780E0C80147814630003E
:10E5D000CE85568597C0FFFFE7802035A1679387DA
:10E5E000D70348083ECC230A810026CE97F0FFFFD0
:10E5F000E78040DD45611743FFFF670043AFA28519
:10E600001306710097000000E78060D7AA840944D0
:10E6100055D13544E30055FB4A8597F0FFFFE7806D
:10E6200000450D4441D9014497D0FFFFE780C0FE6B
:10E63000634DA400C16B0144FD1B97D0FFFFE78031
:10E64000A0FD634EA4001544B5B7DC4413171400B5
:10E65000BA9783D70700638327030504F1B7D8442B
:10E6600093171400BA9703D70700631B7701239011
:10E670002701268597A00000E780C0DA01441DBF6E
:10E68000050465BF1743FFFFE702C3A383C79500D7
:10E6900041112A8A93F7F707A384F50032852E8962
:10E6A000328497E0FFFFE78000FB93170501C187E5
:10E6B0006353F006AA89228597E0FFFFE780A0F95F
:10E6C0002311A1004E85832A040097C0FFFFE78035
:10E6D00040F539E58357440085440144F11793B769
:10E6E0001700A300F1000348110003572100D6874B
:10E6F0005285CE862686CA8597F0FFFFE7806006A2
:10E70000A167F10748003EC42302910022C697F09A
:10E71000FFFFE78020CB41011743FFFF6700C39D48
:10E72000A2851306110097000000E78040C52A84E7
:10E73000894455D98357210011678544BA97C20788
:10E740001167C1831307F7EFE36FF7F89787FF1F90
:10E750009387C78B9C4381CB854513052100975038
:10E760000000E7806074835521002285814497C0B2
:10E77000FFFFE780A0E125D923100500228597A09F
:10E780000000E78080CC85B71743FFFFE702A39224
:10E7900083C7950041112A8B93F7F707A384F500EF
:10E7A00032852E8A328497E0FFFFE780C0EA931714
:10E7B0000501C1876351F006AA8A228597E0FFFF11
:10E7C000E78060E92A895685832B040097C0FFFF04
:10E7D000E78020E531E58357440081440544F11783
:10E7E00093B71700A301F10003483100DE875A8573
:10E7F0004A87D6862286D28597F0FFFFE78060F6AB
:10E80000A167ED0748003EC42302810026C697F0A9
:10E81000FFFFE78020BB41011743FFFF6700238D07
:10E82000A2851306310097000000E78040B5AA8456
:10E8300009445DD99167CA97C2071167C18313075D
:10E84000F7EF0544E362F7FACA8597C0FFFFE78058
:10E85000E0D3014451F9814997D0FFFFE780C0DC44
:10E8600063DBA900984893971900BA9703D707006C
:10E8700005EF2390270197D0FFFFE780E0DA1544EA
:10E88000E384A9F6268597A00000E78000BC97776F
:10E89000FF1F9387A7779C430144B9D74A859750B8
:10E8A0000000E780005889B785097DB71743FFFF4F
:10E8B000E702438179713E847C083EC82E8AB707FF
:10E8C0001400A1653ECAE5057C08AA89080836C47B
:10E8D000428932C6BA8AC6843ECC97C0FFFFE78021
:10E8E00060DFCA85080897E0FFFFE78000C732466F
:10E8F0000808B28597E0FFFFE78020C8A246630AB8
:10E9000009049D45080897E0FFFFE780C0BE1D464B
:10E9100081459730FFFFE780807F63890A08914532
:10E92000080897E0FFFFE78000BD1146A685970025
:10E930000100E780A079100801478146D2854E8505
:10E9400097C0FFFFE78060FE45611733FFFF670058
:10E95000A37AB685080897E0FFFFE78000C21C4055
:10E960000808D8439355C701858912075183B2051A
:10E97000D98D97E0FFFFE78040C01C40080883C5A1
:10E98000870097E0FFFFE78040BD1C40080883C573
:10E99000A70097E0FFFFE78040BC1C40080883C544
:10E9A000970097E0FFFFE78040BB85BF89450808D7
:10E9B00097E0FFFFE78020B483C704002300F50041
:10E9C00083C71400A300F500BDB71733FFFFE702AC
:10E9D000636F83C795004111AA8993F7F707A38452
:10E9E000F5003285AE84328497E0FFFFE780A0C651
:10E9F00093170501C187635DF0042A89032A040087
:10EA000097C0FFFFE780E0C119E98357440005483C
:10EA1000F11793B71700A307F100814631A8130639
:10EA2000F100A28597000000E78060951DC51C4598
:10EA30009DC783D6470001480347F100930785002F
:10EA4000D2884A86A6854E8597000000E78040E67A
:10EA500041011733FFFF6700236A09487DBF1D4846
:10EA60006DBF1733FFFFE702E36565715C083EC4C5
:10EA7000B7077B013EC65C083EC883C795002A8A5B
:10EA8000328593F7F707A384F500AE8997E0FFFF7F
:10EA9000E78040BA8357E100E1C78945280097C065
:10EAA000FFFFE78020C38145280097E0FFFFE78054
:10EAB000C0AA97C0FFFFE78000C99787FF1F938711
:10EAC000278D9C431774FF1F0344C435AA84333435
:10EAD000800099C3136424009777FF1F9387C73C76
:10EAE0009C4399C3136444009777FF1F9387075291
:10EAF0009C4399C31364840083D504002800014912
:10EB000097E0FFFFE78060A783D52400280097E007
:10EB1000FFFFE78080A683D54400280097E0FFFF31
:10EB2000E780A0A597D0FFFFE78000AB9315050114
:10EB3000C181280097E0FFFFE78020A4A28528007C
:10EB400097E0FFFFE78060A39C446360F902014700
:10EB500081463000CE85528597C0FFFFE780E0DC1C
:10EB600059611733FFFF67002359DC441314490030
:10EB700028003E9497E0FFFFE780609683474400BB
:10EB80000347540089070607BA978607E36AF5FC2E
:10EB9000835524002800814A97E0FFFFE780E09D2D
:10EBA00083454400280097E0FFFFE780009B8345F2
:10EBB0005400280097E0FFFFE780209A8347440035
:10EBC00063C9FA00814A8347540063C1FA02050908
:10EBD000A5BF1C4413975A002800BA9783D5070095
:10EBE000850A97E0FFFFE7804099C9BF032BC40067
:10EBF00093975A0028003E9B83552B00850A97E087
:10EC0000FFFFE780809783550B00280097E0FFFF08
:10EC1000E780A0964DBF1733FFFFE702434C5C49E6
:10EC200093E717005CC997A00000E78060B5173331
:10EC3000FFFF6700034D1733FFFFE702434A2E84AF
:10EC4000814597F0FFFFE780C0E705C583570500C2
:10EC5000FD172310F50009C4835725002310F40085
:10EC600097000000E78060FB01451733FFFF670056
:10EC7000434931457DD823100400C5BF1733FFFF3A
:10EC8000E702434483C7950041112A8A93F7F707A7
:10EC9000A384F50032852E89328497E0FFFFE78058
:10ECA000809B93170501C1876356F006AA89C14569
:10ECB000228597E0FFFFE780A0802A8B4E85832A7C
:10ECC000040097C0FFFFE780C09531E983574400F7
:10ECD000231101000544F11793B71700A300F100B9
:10ECE00081440348110003572100D6875285CE8600
:10ECF0002286CA8597F0FFFFE780A0A6A1679387C9
:10ED0000170248003EC42302810026C697E0FFFF99
:10ED1000E780406B41011733FFFF6700E33D1306B7
:10ED20001100A28597F0FFFFE7806065AA8409E5DE
:10ED300023110100094475B7930521005A859700F6
:10ED40000000E78080EF835721002A84D9DB977782
:10ED5000FF1F9387A72B9C4381CB8545130521007B
:10ED600097500000E78040148355210026853144E8
:10ED700097C0FFFFE78080812DD5231005002685F1
:10ED800097900000E780606C0144A1BF1733FFFF3C
:10ED9000E702E33441112E896C00AA8402C697F081
:10EDA000FFFFE78000D20DC10357050005072310C0
:10EDB000E50097000000E78040E681473E8541017D
:10EDC0001733FFFF6700E3333247954765DBCA859A
:10EDD000268597300000E780800CC147E34005FEA0
:10EDE0003244854741462310F40083570900A68525
:10EDF000130544002311F40097000100E780002D63
:10EE0000228545BF1733FFFFE702C32B83C7950059
:10EE10004111AA8A93F7F707A384F5003285AE89DA
:10EE2000328497E0FFFFE780008393170501C187D5
:10EE30006356F0062A8AC145228597D0FFFFE780F6
:10EE40002068AA845285032B040097B0FFFFE78057
:10EE5000407D31E983574400231101008544F117B7
:10EE600093B71700A300F1000144034811000357B2
:10EE70002100DA875685D2862686CE8597F0FFFF59
:10EE8000E780208EA1679387070248003EC42302D3
:10EE9000910022C697E0FFFFE780C052410117337F
:10EEA000FFFF67006325A2851306110097F0FFFF9F
:10EEB000E780E04C2A8409E523110100894475B7F5
:10EEC00026859305210097000000E78060ECAA8466
:10EED00049FD83552100228597B0FFFFE780006B35
:10EEE00049F5014997C0FFFFE7800074635DA90001
:10EEF000184893171900BA9703D707000DEF035767
:10EF000021002390E70097C0FFFFE780E0716306D0
:10EF100025039777FF1F9387670F9C4399C7035576
:10EF2000210097500000E780C0EF228597900000F5
:10EF3000E780A0511DBF050975B795443DB705C1D0
:10EF40009307F00F630FF500C547630CF5009307B7
:10EF5000F5FF05453315F5004205418182800145E5
:10EF6000828041657D158280B9E91733FFFFE70292
:10EF7000031703450603328497000000E78060FC16
:10EF80009305803EB305B502C205C18181CD03570B
:10EF9000E402854763F8E7001305040197E00000E9
:10EFA000E78060418357E40241677D176385E7008E
:10EFB000FD172317F4021733FFFF670083148280C5
:10EFC0001733FFFFE702230F004283C79500444D2C
:10EFD0000349140093F7F707A384F500834704005F
:10EFE000220911673369F900A167B347F90041119C
:10EFF0002A8BAE8A63ECE70E834724001307C00E0A
:10F00000B91793F7F70F6373F71003473400C1473D
:10F0100063EEE70E834744001307E00793C7070832
:10F020006371F70C8349840083477400A209B3E934
:10F03000F900856763F7F90A034A640083475400BF
:10F040004E85220A336AFA0097500000E780803A22
:10F0500061C123962403834B3400137AFA00239A68
:10F060003403238874032399440393890401631CA4
:10F07000090023A60402239804024E8597E00000AD
:10F08000E780A0353DA0034924004A859700000091
:10F09000E78020EB2397A402834744004E85A38892
:10F0A000F402E38D0BFCE30B09FC97E00000E78022
:10F0B000602E97900000E780407281460146D68519
:10F0C0005A8597E0FFFFE7800058A1679387970371
:10F0D0003EC423020100480002C697E0FFFFE7801C
:10F0E000602E41011733FFFF670063008544A2864D
:10F0F0002686D6855A8597E0FFFFE780C054A16732
:10F10000938797033EC423029100F1B7BD44C5B76E
:10F110009144F1BF1733FFFFE702C3FA01111C0846
:10F12000404D3EC2B7070F003EC41C083EC62A89A8
:10F13000AE8997C0FFFFE78000D7585C1C5C634630
:10F14000B70E6394E50063E2A70E3385A740B3B71B
:10F15000A700B305B7401306803E81469D8D9700FA
:10F160000100E780C0B693140501C180A1659385B5
:10F17000C503480097B0FFFFE780C05581454800B0
:10F1800097D0FFFFE780603D83550404480097D087
:10F19000FFFFE780803E83552404480097D0FFFF9F
:10F1A000E780A03D814589CCC167FD179305F00F2D
:10F1B0006388F400268597500000E78020E0AA8548
:10F1C000480097D0FFFFE78040390355440481454C
:10F1D00001CDC167FD179305F00F6307F500975048
:10F1E0000000E780A0DDAA85480097D0FFFFE780F8
:10F1F000C03683456404480097D0FFFFE780E035C0
:10F2000083457404480097D0FFFFE7800035500025
:10F2100001478146CE854A8597B0FFFFE780E070C1
:10F2200005611733FFFF670023ED814481B7173372
:10F23000FFFFE702C3EA83C7950093F7F707A384AC
:10F24000F50097000000E78020ED1733FFFF67000F
:10F2500043EB1733FFFFE702E3E683C79500411155
:10F26000404D93F7F707A384F5002A8A3285B284CC
:10F27000AE8997D0FFFFE780003E2A8B268597D086
:10F28000FFFFE780403D2A89268597D0FFFFE78072
:10F29000603A93170B0163CA0702E177CA97C20766
:10F2A000C183116763E3E70293070910C207C183B3
:10F2B0001307B00F637BF70093170901C187AA8A70
:10F2C000634AF000C54763FE570141011733FFFF52
:10F2D000670083E297B0FFFFE7802025E31725FF53
:10F2E000D5B763080B0263060902814463890A02E9
:10F2F000B7077F0023106405231124057CC05685C1
:10F3000097000000E780E0C39304803EB3049502B9
:10F3100039A0B7077F00232004047CC08144035533
:10F32000240497E00000E780E0A2A1C497C0FFFF9B
:10F33000E78060B7269593D7F44133379500AE97B1
:10F34000BA9708DC5CDCCE85528597000000E78028
:10F35000A0DC99E023220404A1679387B703480047
:10F360003EC42302010002C697E0FFFFE78080054C
:10F37000A9BF814701481CDC232E0403E9B71733DA
:10F38000FFFFE702C3D597C0FFFFE7802034E147C6
:10F390003305F502914597500000E78040C4E557DA
:10F3A00011C59777FF1F23ADA7A681473E85173369
:10F3B000FFFF670003D51733FFFFE70243D29777BC
:10F3C000FF1F9387A7A580433DC083570404639024
:10F3D000A70683572404639CB7043689B28497C078
:10F3E000FFFFE78040AC5C5C63C3B7046395B70084
:10F3F0001C5C63EEA7028347640463F3F400A687F2
:10F400002303F4048347740463F39700A687A303DC
:10F41000F4048357440441677D176385E70085073B
:10F420002312F4043C4481C7CA852685829717338A
:10F43000FFFF670003CD9777FF1F9387279E9C43AD
:10F44000014599C303C5870082801733FFFFE70298
:10F4500003C90111B70707003EC683C79500584D81
:10F460000AC493F7F7070AC8A384F5002A89AE8473
:10F4700011CB1C4283C707002304F70097900000BC
:10F48000E7800034216493055402280097B0FFFF01
:10F49000E780402497000000E78020FAAA85280032
:10F4A00097D0FFFFE780600B300001478146A685BB
:10F4B0004A8597B0FFFFE78040471304440248089D
:10F4C00022CC230A010002CE97E0FFFFE78080EF05
:10F4D00005611733FFFF6700C3C21733FFFFE70261
:10F4E00003C001117C003ECAB70707003ECC7C0078
:10F4F0003ECE83C795002E84AA8493F7F707A38492
:10F50000F500A16593855502480897B0FFFFE78095
:10F51000601C97000000E78040F2AA85480897D059
:10F52000FFFFE7808003500801478146A2852685BA
:10F5300097B0FFFFE780603F05611733FFFF67006B
:10F5400043BC9777FF1F9387678D9C43094599C3F9
:10F5500003C5970082809777FF1F9387278C9C4372
:10F56000094599C303C5D70082809777FF1F93870A
:10F57000E78A9C43014599C303C5A70082801733DE
:10F58000FFFFE70223B40111B70708003EC683C797
:10F590009500404D0AC493F7F7070AC8A384F50005
:10F5A0002A89AE8429C41442854703C7060063E054
:10F5B000E70A83479400094681496380C702B3077D
:10F5C000F740A304E400B339F00083C71600230515
:10F5D000F40097900000E780A01E03572403058BDA
:10F5E00019C76386090097D00000E78000E921640D
:10F5F00093058402280097B0FFFFE780A00D9700D5
:10F600000000E78040F4AA85280097D0FFFFE7803C
:10F61000C0F497000000E78080F5AA85280097D005
:10F62000FFFFE78080F3014781463000A6854A85C9
:10F6300097B0FFFFE780602F13047402480822CCC4
:10F64000230A010002CE97E0FFFFE780A0D7056103
:10F650001733FFFF670043AA1733FFFFE70223A812
:10F6600001117C003ECAB70708003ECC7C003ECEAC
:10F6700083C795002E84AA8493F7F707A384F50027
:10F68000A16593858502480897B0FFFFE780800455
:10F6900097000000E78020EBAA85480897D0FFFF7D
:10F6A000E780A0EB97000000E78060ECAA8548089F
:10F6B00097D0FFFFE78060EA500801478146A285A6
:10F6C000268597B0FFFFE780402605611733FFFFCF
:10F6D000670023A39767FF1F938747749C430145E7
:10F6E00099C303C5B70082801733FFFFE702239F4A
:10F6F0000111B70707003EC683C79500404D0AC4F5
:10F7000093F7F7070AC8A384F5002A89AE8405C8D1
:10F710001C42054783C707006368F7060347B40028
:10F72000630FF700A305F40097900000E7804009FD
:10F730008347B400B9CF97D0FFFFE78000BF2164B3
:10F740009305B400280097B0FFFFE780A0F897006A
:10F750000000E78060F8AA85280097D0FFFFE780C7
:10F76000C0DF014781463000A6854A8597B0FFFF7C
:10F77000E780A01B2904480822CC230A010002CEFE
:10F7800097E0FFFFE78000C405611733FFFF6700C4
:10F79000439797D0FFFFE780E0BF55B71733FFFFD0
:10F7A000E702E39301117C003ECAB70707003ECC95
:10F7B0007C003ECE83C795002E84AA8493F7F7077A
:10F7C000A384F500A165AD05480897B0FFFFE78069
:10F7D00060F097000000E78020F0AA85480897D0E5
:10F7E000FFFFE78080D7500801478146A285268524
:10F7F00097B0FFFFE780601305611733FFFF6700D5
:10F8000043909767FF1F938767619C43094599C39E
:10F8100003C5C70082801733FFFFE702438C011145
:10F820007C00AE843ECAA165B70707002A843ECC9F
:10F83000D1057C0048083ECE97B0FFFFE78080E905
:10F8400097000000E78020FCAA85480897D0FFFFBA
:10F85000E780A0D0500801478146A685228597B051
:10F86000FFFFE780800C05611733FFFF67006389A6
:10F870001733FFFFE702A38683C7950093F7F707C7
:10F88000A384F50097000000E78020F91733FFFFFD
:10F89000670023871733FFFFE702C38283C7950002
:10F8A0000329C501411193F7F707A384F5001C4212
:10F8B00083C90700854763E637079777FF1F93875C
:10F8C00027AD9C432E84AA8485CF97000000E78053
:10F8D00080F389476306F502630409028347C90080
:10F8E000638037032306390197900000E78040EDDD
:10F8F00083572903898B89C797D00000E780E0B739
:10F900002685A28597000000E78020F1A167CD073A
:10F9100048003EC42302010002C697E0FFFFE780D3
:10F9200060AA41011723FFFF6700037D9767FF1F50
:10F930009387C74E9C431D4599C303C5E70082804A
:10F940001723FFFFE702A3790111B70707003EC69F
:10F9500083C79500584D0AC493F7F7070AC8A384D4
:10F96000F5002A89AE8415C71C4283C70700939609
:10F970008701E18663C4060685466381D706834610
:10F98000E7006388F6002307F70097900000E78000
:10F9900020E321649305E400280097B0FFFFE7808F
:10F9A00060D397000000E780A0F8AA85280097D0D0
:10F9B000FFFFE78080BA014781463000A6854A856F
:10F9C00097B0FFFFE78060F63504480822CC230A91
:10F9D000010002CE97E0FFFFE780C09E056117237C
:10F9E000FFFF670003721723FFFFE702436F011158
:10F9F0007C003ECAB70707003ECC7C003ECE83C7E2
:10FA000095002E84AA8493F7F707A384F500A165D7
:10FA1000B905480897B0FFFFE780C0CB970000000A
:10FA2000E78000F1AA85480897D0FFFFE780E0B2A1
:10FA3000500801478146A285268597B0FFFFE780E1
:10FA4000C0EE05611723FFFF6700A36B1723FFFFBD
:10FA5000E7024367AA8401441769FF1F1309493C61
:10FA6000E14997C0FFFFE78060C66344A4000145F9
:10FA700019A833053403832709003E9583572500D1
:10FA80006397970011051723FFFF6700E3660504DE
:10FA9000C9BF032E8500630A0E121763FF1F1303ED
:10FAA000E356032303006315030029436390061202
:10FAB00003234E01631503001D43639907101723A9
:10FAC000FFFFE702435FC689428A3E89BA8AB6844D
:10FAD000328BAE8B2A84B5E103554E0019E5014304
:10FAE0001A851723FFFF67008360A167A98F11673D
:10FAF00063FBE70097000000E78080F5814597F001
:10FB0000FFFFE78080130844B70700E05841F98FF2
:10FB100018455CC1B707001FF98F1CC55C4991C728
:10FB2000610597E00000E780408BE38A09FA2285AF
:10FB300097900000E78060C65DB7328597C00000EF
:10FB4000E78040430D4349DD1C44116703D547005E
:10FB5000A167A98F63FBE70097000000E78040EFF3
:10FB6000814597F0FFFFE780400D03238400931643
:10FB70004B01D1828347B300035663008588FD8B18
:10FB8000A305F300FD777D8E558EFD76FD16B2043C
:10FB9000F18E83274301C58E231273012313D300F3
:10FBA0002304530123052301A3044301BDDF228560
:10FBB00097B0FFFFE78040CAAA850844B5D1610528
:10FBC00097D00000E780207F8DB71D431A85828083
:10FBD0001723FFFFE702034F0569AA84AE89328A23
:10FBE0000144FD5A7D1997C0FFFFE780E0A26347FB
:10FBF000A40001451723FFFF67000350D844931763
:10FC00001400BA9703D70700631F370323905701E7
:10FC100063070A00268597900000E780A0809C4437
:10FC20009DC383D76700B3F72701639E3701D2884E
:10FC30000148814701478146014681452685970055
:10FC40000000E78040E5050479BF1723FFFFE702C6
:10FC5000634779711C103EC4B7070F003EC61C10E5
:10FC60003EC883C79500AA8A328593F7F707A38415
:10FC7000F5002E89328497D0FFFFE780C09D93174F
:10FC80000501C187635AF006AA89228597D0FFFF34
:10FC9000E780609C2A8A4E85032B040097B0FFFF03
:10FCA000E780209839ED8357440081440544F117DB
:10FCB00093B71700A303F10083457100DA87228709
:10FCC000D2864E86280097E0FFFFE780A0580147C4
:10FCD00081463000CA85568597B0FFFFE780E0C4B3
:10FCE000A1679387F70348083ECC230A810026CEFC
:10FCF00097D0FFFFE780006D45611723FFFF670086
:10FD0000A33FA2851306710097E0FFFFE7802067FD
:10FD1000AA84094455D1528597E0FFFFE78020D59A
:10FD20000D4459D90546D285268597000000E78005
:10FD300060EA2A8451B71723FFFFE702433A83554D
:10FD400007000346270041112A842E8532C62EC49F
:10FD500097E0FFFFE780A0D101C93246A245228586
:10FD600097000000E78000E741011723FFFF6700CD
:10FD700043391723FFFFE702033483C7950041117E
:10FD8000AA8A93F7F707A384F5003285AE893284F7
:10FD900097D0FFFFE780208C93170501C187635739
:10FDA000F00AC1452A8A228597C0FFFFE78040718B
:10FDB0002A8D228597D0FFFFE780E0892A89228556
:10FDC00097D0FFFFE7800087930705F893F7F70FB9
:10FDD0001307E007AA8B637BF706228597D0FFFF06
:10FDE000E78040852A8C228597D0FFFFE7808084BA
:10FDF000AA8C5285032B040097B0FFFFE780608236
:10FE000039E983574400231101008144F11793B766
:10FE10001700A300F1000544034711008356210099
:10FE2000938784005685DA8822885286CE8597F09B
:10FE3000FFFFE780E0A7A167E90748003EC423026F
:10FE4000810026C697D0FFFFE780C05741011723E6
:10FE5000FFFF6700C32913061100A28597E0FFFF8B
:10FE6000E780E051AA8409E52311010009446DB738
:10FE7000930521006A8597F0FFFFE78060F12A84EF
:10FE800041FD835521009356C90013164901854849
:10FE90006688E2875E87858A518226859700000002
:10FEA000E78060BF2A848DBF1723FFFFE702A320EE
:10FEB00083C7950041112A8B93F7F707A384F500B8
:10FEC0003285AE89328497C0FFFFE780C0789317F0
:10FED0000501C1876352F00A2A8A228597C0FFFF75
:10FEE000E7806077AA8A228597C0FFFFE780A07627
:10FEF0002A89228597C0FFFFE780C073930705F822
:10FF000093F7F70F1307E0072A8C6377F70622852C
:10FF100097C0FFFFE7800072AA8C228597C0FFFF81
:10FF2000E78040712A8D5285832B040097A0FFFF44
:10FF3000E780206F39E58357440085440144F11779
:10FF400093B71700A301F100034731009307840022
:10FF50005A85DE882688D6865286CE8597F0FFFFA2
:10FF6000E78000958D4748003EC42302910022C6D9
:10FF700097D0FFFFE780004541011723FFFF67008F
:10FF80000317A2851306310097E0FFFFE780203FAB
:10FF90002A84894455D99356C900131649018548C6
:10FFA0006A88E6876287858A5182D6859700000035
:10FFB000E78060AEAA8449BF1723FFFFE7028310E2
:10FFC0002A8981440144617A916A176BFF1F130BE0
:10FFD000EB0397B0FFFFE780206563C7A40022858D
:10FFE0001723FFFF6700431183270900939914002B
:10FFF000CE9703D507003307450142074183636469
:020000040001F9
:10000000570305C103270B0019C785453E85974057
:100010000000E78060E9832709000504CE9723905C
:10002000070085047DB797000000E78060A2832762
:1000300009000504CE972390070065D5814597F008
:10004000FFFFE78080BFF1BF1723FFFFE7028307B1
:1000500083C7950041112A8A93F7F707A384F50017
:1000600032852E89328497C0FFFFE780C05E9317E8
:100070000501C187635AF004AA89832A040097A066
:10008000FFFFE780005A31E583574400854401446F
:10009000F11793B71700A301F10003483100D68789
:1000A00052850147CE862686CA8597D0FFFFE78016
:1000B000406BA167F50748003EC42302910022C6A9
:1000C00097D0FFFFE780003041011723FFFF670053
:1000D000A302A2851306310097E0FFFFE780202AE4
:1000E0002A8489445DD99767FF1F938727F29C4331
:1000F00081CF044997B0FFFFE7800053AA8526858A
:1001000097400000E78040DA1305040197000000E3
:10011000E780C0EA228597800000E78000338144B1
:10012000ADBF1723FFFFE70203F983C79500411115
:10013000AA8A93F7F707A384F5003285AE89328443
:100140002311010097C0FFFFE780E05093170501DE
:10015000C1876354F0062A8AC145228597C0FFFFF4
:10016000E7800036AA8B5285032B040097A0FFFF7F
:10017000E780204B21E98357440085440144F1176F
:1001800093B71700A300F1000348110003572100A3
:10019000DA875685D2862686CE8597D0FFFFE78000
:1001A000405CA1679387270248003EC42302910068
:1001B00022C697D0FFFFE780E02041011723FFFF11
:1001C0006700E3F2A2851306110097E0FFFFE780C6
:1001D000001B2A8489444DD99767FF1F938707E343
:1001E00098433E8901CF044997B0FFFFE780C043A1
:1001F000AA85268597400000E78000CB13050401FF
:1002000097000000E78080DB97B0FFFFE780C041E8
:1002100095443DD9930521005E8597F0FFFFE78067
:1002200020B7AA8435F11C4803572100228523906A
:10023000E70097800000E780402183270900A9D7C5
:100240000355210097400000E780A0BD35BF17236C
:10025000FFFFE70243E683C795004111AA8A93F79F
:10026000F707A384F5003285AE89328497C0FFFF7B
:10027000E780603E93170501C1876351F0062A8A23
:10028000228597C0FFFFE780003D2A895285032B16
:10029000040097A0FFFFE780C03831E58357440092
:1002A00085440144F11793B71700A301F1000348F7
:1002B0003100DA8756854A87D2862686CE8597D042
:1002C000FFFFE780004AA167F90748003EC4230208
:1002D000910022C697D0FFFFE780C00E410117238F
:1002E000FFFF6700C3E0A2851306310097E0FFFF20
:1002F000E780E0082A8489445DD99167CA97C207DC
:100300001167C1831307F7EF8544E362F7FA976734
:10031000FF1F9387A7CF9843BE8B01CF044997B0A7
:10032000FFFFE7806030AA85268597400000E780C0
:10033000A0B71305040197000000E78020C897B01C
:10034000FFFFE780602E95443DD11C482285814403
:100350002390270197800000E780200F83A70B00E0
:10036000B9D74A8597400000E780A0AB89B717232B
:10037000FFFFE702C3D62A844105B284970000003C
:10038000E780C0C311C5228597800000E780E00B9D
:1003900081460146A685228597800000E780C04EF1
:1003A0001C4C89C7DC4799C3228582971723FFFF1E
:1003B000670023D59767FF1F938747A69C43014596
:1003C00099C31385070182809767FF1F938707A54D
:1003D000884382801723FFFFE70263D09317C6008C
:1003E000DD8DC2054111C1812A8432C697C0FFFF4D
:1003F000E780A0183246228511829375F60F97C0C8
:10040000FFFFE780801541011723FFFF670063CFDF
:100410001723FFFFE70203CB79713C083ED2B707F1
:100420000C003ED43C083ED683C79500AE842A8992
:1004300093F7F707A384F500A16593853504481069
:1004400097A0FFFFE7800029C165FD150144176AE9
:10045000FF1F130A2ABD930A400EAE892E8B2EC6AB
:1004600097B0FFFFE780401F4205931704014181C9
:10047000C183B24563E9A702C167FD176387F50031
:10048000481097C0FFFFE780400F5010014781469A
:10049000A6854A8597A0FFFFE7802049456117237D
:1004A000FFFF670063C53307540383270A0BBA971E
:1004B00003D6C701630A3601638A350148109700E5
:1004C0000000E78060F1DA85050451BFB285EDBF19
:1004D0001723FFFFE70223BE79717C083EC8B707E8
:1004E00011003ECA7C083ECC83C79500AA8932859C
:1004F00093F7F707A384F5002E8997C0FFFFE780E5
:10050000801585676378F504A165AA8489050808C4
:1005100097A0FFFFE780001C268597400000E7803A
:1005200060ED133415000A04A285080897C0FFFF88
:10053000E780A002A685080897C0FFFFE780E003D8
:1005400025CC014781461008CA854E8597A0FFFF3C
:10055000E780A03D45611723FFFF670043B9B3075C
:1005600054030327CA0ABA9703D70700631C9700EE
:1005700003D6270063806505080897000000E78020
:10058000A0E5DE8505042EC697B0FFFFE780C00D0D
:100590004205931704014181C183B245E3E1A7FC01
:1005A000C167FD17E38FF5F8080897C0FFFFE780E4
:1005B000C0FC41BFB285F9B7C165FD150144176A9A
:1005C000FF1F130A2AA6930A80022E8BAE8B65BFEB
:1005D0001723FFFFE702A3B01841834717008346A4
:1005E0000700A207D58FD207D1832390F500834758
:1005F0002700034717008D45A207D98F9183231049
:10060000F60097C0FFFFE78060EA1723FFFF67004F
:1006100043AF1723FFFFE702E3AAC1640144176950
:10062000FF1F130929A093098002FD1497B0FFFF53
:10063000E78080036347A40001451723FFFF67009D
:10064000A3AB330534038327C90A3E9583570500BE
:10065000E38597FE0504D9BF1723FFFFE70283A6B2
:100660002A8AAE89B284B68A97400000E78080D893
:1006700019E591473E851723FFFF6700E3A72A8905
:100680004E8597C00000E780E08E2A84638E0A04BE
:100690008D476DD103570500C547E31D47FD03474F
:1006A000F9018546AD47E317D7FC8347450081CF65
:1006B0004146A6855D0597F00000E780C09E814712
:1006C00055D9AD4745BF130965012302E500CA8529
:1006D000268597100000E780606231C1A547E38B53
:1006E0000AF82302040079B705C183570500E39295
:1006F00047F94146A685190597F00000E780A09AC2
:1007000081472DD99947BDB74E8597000000E780F6
:1007100080F02A84954739DD130955004DBF4146C5
:10072000A68523104401231134011305190097F005
:100730000000E780A099228597800000E780A0EA6A
:1007400081470DBF1723FFFFE702639979717C0092
:100750003ECCB7070A003ECE7C003ED083C7950052
:10076000B2842E8493F7F707A384F5001306A10043
:100770002A892C00268597000000E780A0E5A16566
:1007800028088D0597A0FFFFE780C0F490408355AF
:10079000A10003558100854697000000E78000EC2A
:1007A000AA84AA85280897C0FFFFE78000DB0356CC
:1007B000A10083558100280897000000E780C0C190
:1007C000300801478146A2854A8597A0FFFFE78050
:1007D000C015854748103ED42302910202D697D017
:1007E000FFFFE78020BE45611723FFFF670063918D
:1007F0001723FFFFE702A38E79717C003ECCB70779
:100800000A003ECE7C003ED083C79500B2842E8481
:1008100093F7F707A384F5001306A1002A892C009B
:10082000268597000000E780E0DAA16528088D059D
:1008300097A0FFFFE78000EA90408355A100035591
:100840008100814697000000E78040E1AA84AA85E4
:10085000280897C0FFFFE78040D00356A1008355CA
:100860008100280897000000E78000B730080147A2
:100870008146A2854A8597A0FFFFE780000B4810BC
:100880002302910202D402D697D0FFFFE78080B303
:1008900045611723FFFF6700C3861723FFFFE702A9
:1008A000038497000000E78060DB1723FFFF6700E9
:1008B00043859757FF1F9387A75688438280172346
:1008C000FFFFE702C381835725004111AE842A84CC
:1008D0002307B10017F5FFFF130525466C0023160B
:1008E000F10097A0FFFFE780404691C422859780E2
:1008F0000000E780E0D6FD572310F4001306200225
:100900008145130554009720FFFFE7804080410197
:100910001713FFFF6700E37E1713FFFFE702837AD9
:1009200079717C003ECCB7070A003ECE7C003ED0F9
:1009300083C79500AA89AE8493F7F7073285A3840D
:10094000F5001306A1002C0097000000E78080C886
:1009500003558100114497400000E780A0A915C508
:100960000355A100014497B00000E780A06011CDBD
:10097000035705008357810045446318F7008545F8
:1009800097000000E780E0F30144216993053900F6
:10099000280897A0FFFFE780E0D3A285280897C02A
:1009A000FFFFE78080BB0356A10083558100280824
:1009B00097000000E78040A2300801478146A685E5
:1009C0004E8597A0FFFFE78040F648104AD42302E7
:1009D000810202D697D0FFFFE780C09E45611713C2
:1009E000FFFF670063711713FFFFE702A36D9757BF
:1009F000FF1F9387A7422A8488432E8915C5035772
:100A000045038357C4016311F70223260502231807
:100A10000502410597D00000E780209C630609008D
:100A200097800000E78060DB81449759FF1F93891E
:100A3000695F130A800297B0FFFFE780E0C263C4DA
:100A4000A4049757FF1F938727469C4399C70355D4
:100A5000C40197200000E780C0BD6307090022851C
:100A600097800000E780C0A01306400E81452285D4
:100A70009710FFFFE780A069FD57231EF4001713AE
:100A8000FFFF670063673385440383A7C90A3E9568
:100A9000035705008357C4016317F700CA85970001
:100AA0000000E78000E2850479B71713FFFFE70233
:100AB000636183C795004111AA8993F7F707A3845F
:100AC000F5003285AE8497C0FFFFE780C0B8856728
:100AD0006378F5042A8997400000E780A0910144DB
:100AE00001CD83D7040031446388270185459700F1
:100AF0000000E78080EF01444E85A2864A86A685E5
:100B000097D0FFFFE780609DA16793871704480097
:100B10003EC42302810002C697D0FFFFE780808A8F
:100B200041011713FFFF6700235D1713FFFFE70263
:100B300063599757FF1F9387672E804329C4014548
:100B400097C00000E780002181470148C1641CDC98
:100B5000232E0403232004041759FF1F1309894C73
:100B600001449309400EFD1497B0FFFFE780C0AE2B
:100B7000634FA400814517F5FFFF1305857F97A0FC
:100B8000FFFFE780801C1713FFFF6700E356330564
:100B900034038327090B3E958357C501638797006C
:100BA000854597000000E78040E4050475BF935732
:100BB000050113D78700A380F50093170501C183B2
:100BC000A1832380E5002381F500A381A500828015
:100BD0001713FFFFE702A3502300050083C715008A
:100BE000A300F50083C725002301F50083C7350066
:100BF000A301F50083C745002302F50083C7550014
:100C0000A302F50083C7650093059500A3030500C3
:100C10002303F50023040500328597000000E780D8
:100C200040F91713FFFF6700C34D1713FFFFE702DB
:100C300063494111E9540DCD85CD93F9C5FF2E844B
:100C40002A89AA84338AA900B7EA040063189A02A1
:100C50000D88854411CCB7E704009C5F82972AC6B3
:100C600022866C003305390197E00000E7800046DA
:100C7000268541011713FFFF6700034883A78A03F6
:100C80009104829793170501C183A183A38EF4FE7B
:100C900093570501238FF4FEA183238EA4FEA38F17
:100CA000F4FE6DB763E6D5021713FFFFE702234397
:100CB000B28741113686BE8536C697E00000E780D0
:100CC000E040B246410136851713FFFF67006343DA
:100CD000814636858280838705001387F5003D05B0
:100CE000FD8793F77708834607007D158606B58F45
:100CF000A300F5006307B7007D17834717009D83A6
:100D0000DDB782801713FFFFE702633DB7E70400FA
:100D100083A7070932872A863A85829713351500FB
:100D20001713FFFF6700E33D15C181478DC11713FE
:100D3000FFFFE702C33A414697E00000E780003931
:100D400085473E851713FFFF6700A33B81473E851C
:100D500082801DCD1713FFFFE702633841468145AE
:100D60002A849710FFFFE780803A414681451305AA
:100D700004039710FFFFE78080390147C1672322F2
:100D8000040438C87CC805451713FFFF67006337A4
:100D90000145828081473DCDB5CD1713FFFFE702A6
:100DA0000334B2842E891306800581452A84971066
:100DB000FFFFE780C035CA8524C426859700000060
:100DC000E780C0F64146814522859710FFFFE78006
:100DD00000343044A285228597000000E780C0F2ED
:100DE00093040401A285268597000000E780E0EEC9
:100DF000A6851305040297000000E78000EE228517
:100E000097000000E78020F585473E851713FFFF18
:100E10006700232F3E8582801713FFFFE702832A96
:100E20004111E9540DCD85CD93F9C5FF2E842A8952
:100E3000AA84338AA900B7EA0400639844030D88A2
:100E4000814411CCB7E704009C5F82972AC62286B2
:100E50006C003305390197E00000E78020272685E4
:100E600041011713FFFF6700232983A78A03910419
:100E7000829793170501C183A183A38EF4FE935734
:100E80000501238FF4FEA183238EA4FEA38FF4FE1D
:100E90006DB765CD1713FFFFE702C322B28411E6D9
:100EA00005451713FFFF670023252A842E89014576
:100EB000EDD93C487848B3E6E700E5D69386F7FFDE
:100EC000B3B7F6007D17032A4404BA9734C87CC828
:100ED00063050A06C14913050A03B38949412295EE
:100EE000637D3601B2862E86A68597000000E780D6
:100EF000A0DB7C40BE9464C065B7CE862E86CE85CE
:100F000097000000E78040DAC114D2944E99232262
:100F10000404A2879306040103C7070003C607035E
:100F20008507318FA38FE7FEE398F6FE3044A28554
:100F3000228597000000E78020DD2699C14933060D
:100F4000994063EC9900A9DCA686A68513050403E5
:100F500097000000E78040D579BF8147B306F400D1
:100F60003307F6000347070083C5060085072D8F6A
:100F70002380E600E39437FF3044A2852285970062
:100F80000000E78060D8C1145DBF014582800DC1BB
:100F90001713FFFFE702A31413068005814597107E
:100FA000FFFFE780C01605451713FFFF67006315B5
:100FB00001458280814749C5C1C51713FFFFE7027C
:100FC0000312FC4141462E84AA846399C704138608
:100FD0000501A2878146C14503C7070003C5070372
:100FE0008507298F3305D600034505008506298F1F
:100FF000A38FE7FEE392B6FE3044A28526859700D4
:101000000000E78060D0228597000000E78060F84C
:1010100085473E851713FFFF6700A30E138507035F
:101020001D8E814522959710FFFFE780400E7C4082
:10103000130700F813060402A2972388E70251BFA2
:101040003E8582801713FFFFE70263096D712E84CE
:10105000B284AA8590102800368997000000E780A6
:10106000A0D309EDD55725A050400C40280097008B
:101070000000E78040E27DD5FD142104F5F42C004A
:101080004A8597000000E78020F3814761DD3E85B7
:1010900051611713FFFF6700C3061713FFFFE70235
:1010A000030441112EC432C62C00054697000000EF
:1010B000E78080F941011713FFFF670083041713CE
:1010C000FFFFE702C30101112A842EC602C802CA2B
:1010D00002CC02CE97E00000E780C023B2462A8609
:1010E000A285080897000000E78060FB1375F50FE4
:1010F00005611713FFFF6700C3001713FFFFE70227
:1011000003FE7971B2872A8421462308B1001305B2
:101110001101BE853AC436C697E00000E78000FBA7
:10112000B24693059101368597000000E78060A8DC
:101130002285141035460C0897000000E78020F641
:101140002A84224701E921460C103A8597E00000E5
:10115000E780C0F7228545611713FFFF670063FA38
:101160001713FFFFE702A3F77171AE84AA850A8502
:10117000328497000000E78060BB11C90A86A6850B
:10118000228597000000E78020B8814711E1C5471C
:101190003E854D611713FFFF6700A3F61713FFFF8E
:1011A000E702E3F01D712A8AB289BE84354685477D
:1011B000130511012E8CB68A3A8BC28C468D2308FA
:1011C000F10097E00000E78060F010100C085285F5
:1011D000231F010097000000E780C0F82A843DED3E
:1011E000A1476313FD089307900591E0E547354655
:1011F000E2851305110113990A012308F10013591F
:10120000090197E00000E78060EC1357890093978D
:101210008A00D98F90080C085285231FF10097008F
:101220000000E78020F42A8415E9A1E49387FA00FE
:1012300091831379F9003EC6631309004149668B17
:101240008144C14B854DB247639F970C6A868C00E1
:1012500033855C0197E00000E78040E72285256147
:101260001713FFFF670063E893079004C9F0A547D1
:10127000BDBF834701050947C14B2308F1008347E0
:101280001105A58FA308F10093872400814463E131
:10129000FB04014714083386E6008C08B386E4009B
:1012A000BA95DA9683C6060083C505000507AD8E9C
:1012B0002300D600E390E7FE4147639CE7049008D3
:1012C0000C08528597000000E780C0E925D181A075
:1012D000B3069B00BA871008B305F60090083E9647
:1012E00003C506000346060085078506298E238070
:1012F000C500E39277FF998F90080C085285BE9441
:1013000097000000E78000E68947014749D12A8419
:10131000B1B790083E96034606001408BE96238097
:10132000C600850759BFB247850463879714814774
:101330001808B306F70098083E973386F90003476C
:101340000700034606008507318F2380E600E391FE
:1013500077FF90080C08528597000000E78080E036
:101360005DF53546E285130511012308B10197E0CB
:101370000000E780A0D51397040141839397840070
:101380002183D98F10180C085285231FF100970074
:101390000000E78020DD25FD814710183387F90024
:1013A0003E960347070003460600B306FB00850789
:1013B000318F2380E600E39277FF65A81808B30613
:1013C000F70098083E973386F90003470700034665
:1013D00006008507318F2380E600E3E127FFCA87F7
:1013E000639E770990080C08528597000000E780FB
:1013F00060D711FD81479800B306F70090081810D8
:101400003E973E9603470700034606008507318F47
:101410002380E600E39177FF3546E285130511014D
:101420002308B10197E00000E78040CA1397040148
:101430004183939784002183D98F10180C0852851B
:10144000231FF10097000000E780C0D1E31105ECF5
:10145000814710183387F9003E960347070003467B
:101460000600B306FB008507318F2380E600E3E228
:1014700027FFC109410BC1BB814785B79408BE96C0
:1014800083C6060018083E972300D700850789BF4A
:10149000638006321713FFFFE70263C159712A8484
:1014A000BE89B28B85473546130511022E8B468CBB
:1014B0004289BA8A368A2300F10297E00000E78069
:1014C000E0C010180C1022852317010297000000BD
:1014D000E78040C963180512A147631FFC06930704
:1014E000900563930900E5473546DA851305110237
:1014F00093140A012300F102C18097E00000E78005
:10150000E0BC93178A0013D78400D98F90080C1081
:1015100022852317F10297000000E780A0C47DE137
:10152000639209049307FA00BD88918391E0C14456
:10153000C207C183DE8C814A3EC6414DB24763E299
:10154000FA0E6286B3854B01881097E00000E780B1
:1015500080B54DC93D557DA093079004E39609F8E9
:10156000A54759B7834701050947C14C2300F1023C
:1015700083471105B3C7F900A300F102938729003F
:10158000814963E1FC04814618103306D7008C08BA
:101590003387D900B69556970347070083C50500E2
:1015A00085062D8F2300E600E390D7FE4147639028
:1015B000E70690080C10228597000000E78080BAAB
:1015C00035D189A0B3863A01BA871010B305F60069
:1015D00090083E9603C5060003460600850785066B
:1015E000298E2380C500E39297FF3387EC40900853
:1015F0000C102285BA9997000000E780A0B68947B1
:10160000014741D165611713FFFF670003AE9008E2
:101610003E96034606001410BE962380C60085073A
:1016200079B7B247850A93990A01939D8A0093D9A5
:1016300009016391570F85473546DA851305110275
:101640002300F10293D9890097E00000E78000A809
:10165000B3ED3D0190000C1022852317B1039700D4
:101660000000E78020B059FD8147A68963EA97060C
:1016700026860C084A8597E00000E78020A5814770
:101680001810B306F700100898083E973E960347D7
:101690000700034606008507318F2380E600E3E15B
:1016A00097FE639FA90590080C1022859700000003
:1016B000E78040AB21F981479810B306F700900806
:1016C00018183E973E960347070003460600850715
:1016D000318F2380E600E391A7FF4109C10CB9BD1A
:1016E00018089000B306F7003E963387FC000347C6
:1016F0000700034606008507318F2380E600B5B753
:1017000098084E97034707001C10CE972380E700E8
:10171000850941BF85473546DA8513051102230047
:10172000F10293D9890097E00000E780209AB3ED99
:101730003D0190000C1022852317B1039700000093
:10174000E78040A2E31005EC814718089000B3063B
:10175000F7003E963387FC00034707000346060068
:101760008507318F2380E600E391A7FF41460C08EF
:101770004A8597E00000E780609581471810B3061E
:10178000F700100898083E973E9603470700034667
:1017900006008507318F2380E600E391A7FF9008BC
:1017A0000C10228597000000E780C09B1DD599BDD5
:1017B0007D5582801713FFFFE702639201112A848F
:1017C0002E8593055100328902C002C202C402C6AE
:1017D0009304740097F0FFFFE780A03D1D46A685A7
:1017E0001305910097E00000E780408E10088A857D
:1017F0004A8597000000E780E09619ED93071400F2
:10180000180883C607000346070085070507B18E41
:10181000A38FD7FEE397F4FE05611713FFFF670060
:10182000438E1713FFFFE702E3892E848C41411199
:10183000AA89838715003289914463D30700A144A4
:101840009757FF1F9387C7B49C43A1C7C1CA8D4751
:101850002310F10083C725004A852301F10083C7C7
:101860003500A301F10083C745002302F10083C7BF
:101870005500A302F10083C7650093059100A303FF
:1018800001002303F1002304010097F0FFFFE7802C
:1018900040320C404A860A8597F0FFFFE78080338C
:1018A0000328040083564400A6881D088147014789
:1018B000E51642868A854E8597000000E780408EB7
:1018C0002A8919E5A685228597B0FFFFE780A0C287
:1018D0004A8541011713FFFF670003824A860A8584
:1018E00097F0FFFFE780002F6DB71703FFFFE702B8
:1018F000637D2E848C414111AA898387150032892A
:10190000914463D30700A1449757FF1F938747A8CB
:101910009C43A1C7C1C68D472310F10083C7250092
:101920004A852301F10083C73500A301F10083C775
:1019300045002302F10083C75500A302F10083C7CD
:10194000650093059100A30301002303F100230424
:10195000010097F0FFFFE780C0250C404A860A850A
:1019600097F0FFFFE7800027835644000328040018
:101970008A85858EC2061D08C1822312D400A688DE
:1019800081470147E51642864E8597000000E780B3
:1019900060B041011703FFFF670003764A860A859E
:1019A00097F0FFFFE78000234DBF1703FFFFE7021B
:1019B0000373B335B000011185052A891315F601AB
:1019C000336515012308B1009305110136843AC629
:1019D00032C03EC442C297F0FFFFE780801DA2479D
:1019E0001248425593D68700230BF10093059101CD
:1019F00093578800A30AD100A30BF100230C010127
:101A000097F0FFFFE780E01A324702460328040000
:101A1000B337E000835644009207914411C2A144B9
:101A20004A85A68842860C0897F0FFFFE78040773A
:101A30002A8919E5A685228597B0FFFFE780A0AB2C
:101A40004A8505611703FFFF6700A36B1703FFFFBC
:101A5000E702436701113EC68647B335B0008505EE
:101A6000AA891315F6015D8D2308B10093051101B4
:101A700036843A89B28442C446C297F0FFFFE780B9
:101A8000401322489248164593578800A30AF10054
:101A90009305910193D78800230B0101A30BF1005B
:101AA000230C110197F0FFFFE780A0103247104090
:101AB00083564400B337E000920703280900914899
:101AC00091C0A1480C084E8597000000E780809CDB
:101AD000AA8401E9835544004A8597B0FFFFE78057
:101AE00080A1268505611703FFFF6700E360AA95C3
:101AF0009307F00F17070100130707646317B5007A
:101B000013C5F7FF1375F50F828005058346F5FFB2
:101B1000B58FBA9783C70700D5B70357450014415F
:101B20009307F00F17060100130606613697420768
:101B30004183139506014181631BE500AD8FB29788
:101B400003C50700130515F31335150082808506BC
:101B500003C5F6FFA98FB29783C70700D9BF170344
:101B6000FFFFE702C357B28736842E86BA86AA855E
:101B70003E85BA8497F0FFFFE7806052634F05000F
:101B8000228597D00000E780E0782A86A686A28585
:101B9000268597F0FFFFE78080501703FFFF67005F
:101BA00043561703FFFFE702E3515D712A8BAE8AAC
:101BB000170501001305C5552C00B284368ABA8971
:101BC0003E8997F0FFFFE780C04F2A845DE1341023
:101BD0004146DA85280097F0FFFFE780404C2A84D1
:101BE00049E98547A303F100A6C2930771002408C1
:101BF000BEC4A68685470D462C18281002DC02DEDE
:101C0000D6C0BEC697F0FFFFE78000442A8435E1C6
:101C100083477102A6860D4693F7F7072300FA0063
:101C2000C1473EDE2C188947281026DCA303F100AB
:101C300097F0FFFFE78040412A8405ED4146A685E5
:101C40004E8597D00000E78060488D47A6860D46F8
:101C50002C182810A303F10097F0FFFFE780C03E87
:101C60002A8401E94146A6854A8597D00000E7808D
:101C7000E045228561611703FFFF6700E347170313
:101C8000FFFFE702C34597F700009387E7A198435A
:101C900083C7470079712A89AE84170501001305AF
:101CA000A5470C083AC42306F10097F0FFFFE78030
:101CB00040412A8405ED14104146CA85080897F072
:101CC000FFFFE780C03D2A8415E1140815462C006B
:101CD000081097F0FFFFE780803C2A8401E9214645
:101CE0002C08268597D00000E780403E228545617C
:101CF0001703FFFF6700E3401703FFFFE702233EE0
:101D000097F700009387479A9C477971AA842E849D
:101D1000170501001305C5400C083EC697F0FFFFEC
:101D2000E780203A0DE914104146A685080897F08F
:101D3000FFFFE780C03605E1140811466C0008106B
:101D400097F0FFFFE780A03519E58347F10193F78E
:101D5000F7032300F40045611703FFFF6700633AB0
:101D60001703FFFFE702A3373688A14881470147E1
:101D7000E54697F0FFFFE780A0421703FFFF6700EB
:101D800043381703FFFFE70283353688A1488147B0
:101D90000147E54697F0FFFFE780C06F1703FFFF9D
:101DA000670023361703FFFFE702633301112A841C
:101DB0002E850C0832C697F0FFFFE780803009EDD2
:101DC000324797060100938626341008C1452285C4
:101DD00097000000E780E0D805611703FFFF670068
:101DE00043321703FFFFE702832F4111C1472EC083
:101DF00032C48A8509463EC23EC697F0FFFFE7809F
:101E0000A02441011703FFFF6700A32F1703FFFF63
:101E1000E702E32C4111AE8613061009AA850A8554
:101E200002C002C202C402C697F0FFFFE78020276B
:101E300041011703FFFF6700C32C1703FFFFE702F1
:101E4000032A3287970601009386062E2E86930575
:101E5000000297000000E780C0D01703FFFF670073
:101E6000432A1703FFFFE70283277971C1472ACC72
:101E70002ED032D42C080D4628003ECE3ED23ED67F
:101E800002C402C602C802CA97F0FFFFE780C01B67
:101E900045611703FFFF6700C3261703FFFFE70233
:101EA00003240111AA842E84170501001305452877
:101EB0008A8597F0FFFFE780C02015E514084146AA
:101EC000A6850A8597F0FFFFE780601D09ED83472F
:101ED000E1010347F101A207D98FCA07C9836177DE
:101EE000D98F2310F40005611703FFFF67006321FA
:101EF00015CD1703FFFFE702831E9747FF1F938748
:101F0000A7F690439745FF1F938545F61745FF1F9A
:101F1000130585F197D00000E78000C51745FF1F26
:101F2000130585F01703FFFF6700A31D1745FF1F6B
:101F3000130585EF82808DCD1703FFFFE702231A7B
:101F40009747FF1F938747F2944301112E840A8617
:101F50009745FF1F938585F197D00000E78040C625
:101F60000A850294014505611703FFFF67006319A5
:101F70007D5582801703FFFFE702631697D00000AC
:101F8000E78080D19747FF1F23A0A7EE17F5FFFF3B
:101F90001305E5C997B00000E780C0741703FFFF81
:101FA000670023161747FF1F130747EE9317150007
:101FB00008433E95FD572310F50082801703FFFF6D
:101FC000E702E3112A84084009E51703FFFF6700D1
:101FD00043131C4158401CC06313E5005CC0834799
:101FE000550023200500F99BA302F50097A0FFFFF1
:101FF000E780E07CC9BF1703FFFFE702A30C974708
:10200000FF1F9387A7EA98432A8411CB83473500A3
:1020100093F7070289C70355050089450297130501
:10202000440197B00000E780403B8355040003550E
:10203000E40097300000E780A00C485819C597A02D
:10204000FFFFE780C077232A04021305840397006B
:102050000000E780E0F68144B1499790FFFFE780F8
:10206000E06A63CBA402834734002320040493F77F
:1020700027FCA301F40000489790FFFFE780006A67
:1020800013161500814522859700FFFFE780200881
:102090001703FFFF67004306B387340303290403D4
:1020A00085043E994A8597000000E78060F123048B
:1020B000090065B78347350093F7070299E30145A7
:1020C00082808357E500E39CB7FEC167FD17631666
:1020D000F60005458280054599A81703FFFFE70232
:1020E000030093170601C187B2842A84014963590A
:1020F000F002835705009DCB01456367F600034559
:1021000084003E953325A6001375F50F0DA01C48DD
:1021100013171900BA9783D70700E38E97FA0509BA
:102120009790FFFFE780805FE343A9FE0145170317
:10213000FFFF670003FD1703FFFFE702A3F8AE8967
:10214000AA849790FFFFE78020532A8497D0FFFF4F
:10215000E780A02EAA860147130684019705000098
:10216000938585E41745FF1F130585D29790FFFFE0
:10217000E780A0192A8925C98C441304C50022854B
:102180009E0593F5050897A0FFFFE780003DCC4032
:1021900083877400E18163DD070493E505082285E8
:1021A00097A0FFFFE780603B0D46938544002285A2
:1021B00097A0FFFFE780803783D50400228597A092
:1021C000FFFFE780A03E83D52400228597A0FFFF74
:1021D000E780C03D03D6490083A50900228597A06A
:1021E000FFFFE780A0344A851703FFFF6700C3F0B5
:1021F00093F5F5076DB71703FFFFE70243EE0111F3
:102200002A84328532C697A0FFFFE780A0289780F6
:10221000FFFFE7808031835704001747FF1F130734
:1022200067E03246231BF100930700F8A30DF1008D
:102230001C471843231AA1008983858BB307F740F5
:10224000B28548083ECE231C0100230D01009700F3
:102250000000E78080EE05611703FFFF670063EA77
:102260001703FFFFE70203E6004101453DC4930465
:10227000C40026853289AE8997A0FFFFE7808025BC
:1022800095452A8A2685035B040197A0FFFFE78016
:10229000E021268597A0FFFFE780203F8D45AA8A91
:1022A000268597A0FFFFE7806020268597A0FFFF87
:1022B000E780A03D5C48420A135A0A01D2975CC4E9
:1022C00023186401814763983A0146054D8133061E
:1022D00025419337160013F5F70F1703FFFF67002B
:1022E000A3E11703FFFFE70203DD89692A8BAE8BA9
:1022F000328AB68A81440144314CFD199790FFFF20
:10230000E780C04063CDA4009790FFFFE7800043C3
:10231000018D33B5AA001703FFFF670043DD338942
:10232000840383270B003E9963170A0083478900C3
:1023300085043E94E1B703560A00DE854A8533F6EC
:10234000C90097000000E780E0F16DD10545E1B7D5
:102350001703FFFFE702A3D801112A847C0003556D
:10236000E5003ECAB70707003ECC7C003ECE972072
:102370000000E78020082A898545480897A0FFFFCC
:10238000E780E0399945480897A0FFFFE780A0164D
:10239000AA844A8597200000E780A0082380A40033
:1023A0009747FF1F938707C89C434166130606F0B3
:1023B0009396870113D78701558F93D68700F18EA7
:1023C000558FA207B706FF00F58FD98F11462C0055
:1023D000138514003EC497D00000E78020CF50083A
:1023E000A38204008945228597000000E780E0E091
:1023F00019C9AA851305840397A0FFFFE780A032BF
:102400003C4085073CC005611703FFFF670063CFB1
:102410001703FFFFE702A3CC9790FFFFE78000328E
:102420002A8405049790FFFFE78040303305A4021B
:10243000F14791453305F50297200000E78020BA67
:1024400011E565551703FFFF6700A3CB9747FF1FF3
:1024500023A6A7A49790FFFFE780402E2A840504B7
:102460009790FFFFE780802C3305A402894506057D
:1024700097200000E780A0B669D59747FF1F23A7E4
:10248000A7A09790FFFFE780602B2A840504979010
:10249000FFFFE780A0293304A4029747FF1F239979
:1024A000879E9790FFFFE78060292A849790FFFF1F
:1024B000E780C027930714003385A7029747FF1FC3
:1024C0002399A79C970701009387478A1747FF1F07
:1024D0002324F79C0145BDB71703FFFFE70283BE26
:1024E000AA842E8901449749FF1F9389A9B3130A2F
:1024F00080069790FFFFE78060236347A4000145B3
:102500001703FFFF670043BF3305440383A7090296
:102510004A86A6853E9597000000E780E0B919E15C
:102520000504C1BF0545E9BF1703FFFFE702A3B8D4
:10253000AA8A2E8BB28B368C3A8A81440144814917
:10254000974CFF1F938C0CAE130D80069790FFFFE6
:10255000E780C01D63C9A40011E085494E851703BB
:10256000FFFF6700C3B83389A40383A70C025E860C
:10257000D6853E994A8597000000E780E0B31DC1EB
:102580009790FFFFE780801B0544636D4501D2866D
:102590006286DA851305090397000000E780A0D45E
:1025A00011C1854985045DB71703FFFFE70283B1B9
:1025B000C16441112A8901449749FF1F938989A663
:1025C000130A8006FD1436C632C42EC29790FFFF50
:1025D000E780C01592452246B2466348A4000145F3
:1025E00041011703FFFF670023B13305440383A7AD
:1025F00009023E9509C683473500C18B9DC791C628
:102600008347350093F707028DC36306990083570C
:10261000E500639C27010357050001CB63E7E50054
:1026200083478500BA97E3CDF5FA050469BF170320
:10263000FFFFE70223A9C1642A8901449749FF1FCC
:102640009389499E130A8006FD149790FFFFE78047
:10265000E00D6346A4001703FFFF6700E3A93305FD
:10266000440383A709023E958357E500638A9700D8
:10267000630499006396270197000000E780E097C4
:102680000504E1B71703FFFFE70263A289692A8AFD
:10269000AE8A328BB68B8144174CFF1F130C8C987B
:1026A000930C8006314DFD199790FFFFE7800008DD
:1026B00063C6A4001703FFFF670023A333899403B5
:1026C00083270C028355CA015A863E994A85970092
:1026D0000000E780609E31C1814D15A03384AD03B9
:1026E0008327090303D60B00D68533F6C9003E9431
:1026F000228597000000E780E0B609E9850D9790F4
:10270000FFFFE780A000E3CBADFC01A82285970086
:102710000000E780E08A23040400850471B71703F2
:10272000FFFFE70243994169AA8A014A174BFF1F3D
:10273000130B4B8F7D19C14B054C9790FFFFE78022
:10274000E0FE6346AA001703FFFF6700439A930960
:102750008006B3073A0383290B02BE9983D7E900A9
:10276000638E270163842A01639A570103A48903B6
:1027700001E84E8597000000E780C0BD050A75BFDF
:1027800083570401639977099304C400268597A0B1
:10279000FFFFE78020D485452A8D2685835C0401D0
:1027A00097A0FFFFE78080D0268597A0FFFFE780F6
:1027B00060E862056185635905048D45268597A00B
:1027C000FFFFE780A0CE8945268597A0FFFFE78021
:1027D000E0CD8945268597A0FFFFE78020CD854580
:1027E000268597A0FFFFE780A0CD83470500094716
:1027F00093F7F707639AE7009945268597A0FFFFAF
:10280000E78000CCA30285014848337D2D012318C1
:1028100094016A9548C40040A1BF1703FFFFE70277
:10282000038C37E404008327041D82979737FF1F2A
:1028300083C7476C1715FF1F130545CFA300F5008D
:102840008327441C82978327841C81461306F00F3C
:102850008145014582971703FFFF6700838A173779
:10286000FF1F1307275918439735FF1F83C5856836
:102870009737FF1F9387876683468703034697032F
:102880006397D5009737FF1F2386C766828083C56D
:1028900087010347A7036317B6009737FF1F238BF2
:1028A000E764828003C687016317C7009737FF1F5D
:1028B0002382D764828083C687011307500263197D
:1028C000D700930760021737FF1F2305F762828046
:1028D00083C68701130660026315D6009307700252
:1028E000DDB783C7870155BF9737FF1F9387075F02
:1028F000D44B0947638DE60817F3FEFFE702237EFA
:102900001739FF1F1309C95A3E8483470900918B69
:102910009DCFB7E4040083A7041D829783A7441CBE
:102920001735FF1F13054559829783A7841C8146DD
:102930001736FF1F0346465A81450145829721C538
:1029400083470900ED9B1737FF1F2303F756834783
:10295000040093F7F70F85CB91471737FF1F232903
:10296000F75897000000E78080EB97000000E780B1
:1029700040EFB7E70400BC4F414691451735FF1FB4
:1029800003454556829717F3FEFF670083778280E1
:1029900017F3FEFFE702A3748D4741116306F504A8
:1029A000C5476308F50285476310F5029737FF1F97
:1029B0002384A754B7E70400BC4B930500101735D8
:1029C000FF1F034525528297410117F3FEFF670061
:1029D000437385471737FF1F2300F752B7E70400FB
:1029E000BC4B93050020E1BF9737FF1F9387074F2C
:1029F000D44B1147638DE600B7E7040083A7071D9A
:102A00008297B7E70400BC4B930500044DBF05490E
:102A10001737FF1F232E274D83C7070032C62E848A
:102A200093F7F70FD5D3B7E4040083A7041D7D14F3
:102A30001374F40F8297E37689FCB245994703C675
:102A40001500E3F0C7FCFC4409061735FF1F13050A
:102A5000E54A8297BC48930500081735FF1F0345D8
:102A60006548829779BF17F3FEFFE7024367173780
:102A7000FF1F1307A7464047184B1C409736FF1F00
:102A800023A4F6466316E4001737FF1F2320F746FA
:102A9000130584FE9790FFFFE78020A7035564FF8E
:102AA0009780FFFFE780A06F97A0FFFFE78020D10E
:102AB00017F3FEFF6700E36417F3FEFFE7022362EC
:102AC0009737FF1F93878741D84BDC4789C797000B
:102AD0000000E78080F985471737FF1F232AF7405A
:102AE0009737FF1F938707319C43930500021735E3
:102AF000FF1F0345253F83C787031737FF1F230B9E
:102B0000F73EB7E70400BC4B829717F3FEFF670060
:102B1000435F9737FF1F23A5A73C828017F3FEFF73
:102B2000E702435A37E404007C4CA1451735FF1FE8
:102B30000345453B82977C48A1451735FF1F034558
:102B4000653A9734FF1F938464398297DC4489EB9C
:102B500097000000E78080D917F3FEFF6700C35994
:102B600003D567FF9780FFFFE7806063AA896DD177
:102B7000D84891476310F7027C4C91451735FF1FE9
:102B80000345453682977C4891451735FF1F03451D
:102B90006535829703A9490103D409018947B7E93B
:102BA00004001737FF1F2325F73483A7091D2104CD
:102BB0004204829783C784011715FF1F13050597E9
:102BC00061191717FF1FA303F79683A7491C4180BC
:102BD00082979737FF1F2381073283A7C91C81463D
:102BE00009469375F40F4A85829711E99737FF1FBD
:102BF00083C7C74089C79700FF1FE780A0FFB7E7DB
